:020000040800F2
:1000000000040020A51F0008F71F0008F71F0008C4
:10001000F71F0008F71F0008F71F00080000000086
:10002000000000000000000000000000F71F0008B2
:10003000F71F000800000000F71F0008C91F020892
:100040005521020857210208592102085D210208A2
:100050007D2102087F21020881210208A5210208D2
:10006000C9210208ED2102081122020835220208E6
:1000700037220208392202083B2202083D220208E8
:100080003F2202084122020843220208F71F00080B
:10009000F71F0008F71F0008F71F00084522020895
:1000A0009122020893220208952202089722020850
:1000B000992202089D220208C92202083923020857
:1000C0003B2302083D2302083F2302084123020884
:1000D00045230208B5240208DD2302087925020819
:1000E0003D26020801270208032702080527020807
:1000F00009270208712702087327020875270208DA
:1001000077270208792702087B2702087D27020843
:100110008127020855280208572802085928020892
:100120006529020867290208692902086B29020863
:1001300000000000000000000000000000000000BF
:1001400000000000000000000000000000000000AF
:10015000000000000000000000000000000000009F
:10016000000000000000000000000000000000008F
:10017000000000000000000000000000000000007F
:10018000000000000000000000000000000000006F
:10019000000000000000000000000000000000005F
:1001A000000000000000000000000000000000004F
:1001B000000000000000000000000000000000003F
:1001C000000000000000000000000000000000002F
:1001D000000000000000000000000000000000001F
:0401E0005FF8E0F1F3
:1001E800032A70B404460D4626D941EA000313F0E9
:1001F800030F13D020782B78984208BF294606D0E1
:100208001EE014F8010F11F8013F984218D1012A95
:1002180002F1FF32F5D1002070BC70470B4604464E
:1002280051F8045B50F8046BAE4204D1043A04461A
:10023800032A0B46F2D81D461046002ADAD1EBE70E
:10024800C01AE9E7032A2DE9F00109D82AB10023E9
:10025800CC5CC45401339342FAD1BDE8F001704735
:100268000B468218014603E02478013301F8014B5C
:1002780011F0030F1C46F7D113F003055DD06E4251
:10028800C5F1040CED009B594FEACC0C08E004348E
:10029800A7593B4607FA0CF748EA070741F8047BD9
:1002A800571A23FA05F8032FF1DC03E014F8013B91
:1002B80001F8013B8A42F9D8CFE753F8404C41F89E
:1002C800404C53F83C4C41F83C4C53F8384C41F8FE
:1002D800384C53F8344C41F8344C53F8304C41F80E
:1002E800304C53F82C4C41F82C4C53F8284C41F81E
:1002F800284C53F8244C41F8244C53F8204C41F82E
:10030800204C53F81C4C41F81C4C53F8184C41F83D
:10031800184C53F8144C41F8144C53F8104C41F84D
:10032800104C53F80C4C41F80C4C53F8084C41F85D
:10033800084C53F8044C41F8044C561A1D460C4618
:10034800403340313F2EB8DC2B460FE053F8101CE9
:1003580044F8101C53F80C1C44F80C1C53F8081CE7
:1003680044F8081C53F8041C44F8041C161B2146C6
:100378001D46103410330F2EE8DC2B4602E02468AB
:1003880041F8044B551A1C46032D03F10403F6DC0F
:1003980090E700BF032AC9B270B408D82AB103464F
:1003A800121803F8011B9342FBD170BC70478218E6
:1003B800044601E004F8011B14F0030FFAD14FF0D2
:1003C800013303FB01F31FE044F8403C44F83C3C94
:1003D80044F8383C44F8343C44F8303C44F82C3C6D
:1003E80044F8283C44F8243C44F8203C44F81C3C9D
:1003F80044F8183C44F8143C44F8103C44F80C3CCD
:1004080044F8083C44F8043C161B254640343F2E6B
:10041800DADC2C4607E044F8103C44F80C3C44F87D
:10042800083C44F8043C161B254610340F2EF2DC19
:1004380001E045F8043B541B032CFADC01E005F805
:10044800011B9542FBD3B0E710F0030F38B5044603
:1004580012D10368A3F1013222EA030313F0803FAB
:100468000AD1031D184653F8042BA2F1013525EAD9
:10047800020212F0803FF5D003782BB1431C1846D6
:1004880013F8012B002AFAD100F076F9204638BD7E
:10049800C9B2F0B4002950D010F0030F10D003787F
:1004A800002B79D0994246D0431C05E013F8012B64
:1004B800002A3FD091423ED013F0030F1846F5D1E1
:1004C800036841EA01270646A3F1013247EA0747D4
:1004D80022EA030212F0803F1DD187EA0303A3F149
:1004E800013222EA030313F0803F14D1043002E002
:1004F80012F0803F0FD1064650F8043BA3F10135B6
:1005080087EA030225EA0303A2F1013413F0803FCE
:1005180024EA0202ECD033783046002B3CD09942D2
:1005280009D0731C01E0914205D0184613F8012B3D
:10053800002AF8D11046F0BC704710F0030F0CD019
:100548000378002BF7D0431C03E013F8012B002A93
:10055800F1D013F0030F1846F7D102680346A2F151
:10056800013121EA020212F0803F0AD10430034629
:1005780050F8042BA2F1013121EA020212F0803F67
:10058800F5D01A781846002AD5D00133184613F842
:10059800012B002AFAD1CEE71846CCE780EA0102FF
:1005A80012F0030F3AD110F0030220F0030021F0FB
:1005B800030150F804CB08BF51F8043B0DD082F07A
:1005C80003024FEAC2026FF07F4323FA02F251F8A6
:1005D800043B4CEA020C43EA020300BFACF10132CF
:1005E8009C4501BF22EA0C0212F0803F50F804CB70
:1005F80051F8043BF2D04FEA0C604FEA1C2C01285A
:1006080028BFB0EB036F08BF1B0AF4D003F0FF0349
:100618004FEA1060A0EB0300704700BF10F0030F13
:100628000AD010F8012B11F8013B012A28BF9A4281
:10063800F4D0A2EB030070474DF8045D4DF8044D6B
:100648004FF0010242EA022242EA024201F0030CA0
:1006580021F0030150F8044B51F8045BBCF1020F80
:1006680026D04BD824F07F4CBCEB152FA4EB02030B
:1006780023EA04030DD113EAC21308BF51F8045B3F
:100688000AD18CEA040CBCEB056F0CD150F8044B72
:10069800E8E74FEA15255CE033F07F4352D10D7847
:1006A8004FEA146C55E04FEA146C05F0FF0550E072
:1006B8004FEA044CA4EB02034FEA1C4C23EA040360
:1006C800BCEB154F17D113EAC21308BF51F8045BEE
:1006D80007D18CEA040CBCEB054F08D150F8044B49
:1006E800E6E71B042ED10D884FEA144C31E04FEA9F
:1006F80005454FEA144C4FEA15452AE004F0FF0C73
:10070800BCEB156FA4EB020323EA04030DD113EA33
:10071800C21308BF51F8045B0AD18CEA040CBCEB85
:10072800052F0AD150F8044BE8E74FEA156510E0A9
:1007380014F0FF0F06D051F8045B4FEA142C25F093
:100748007F4506E04FF000005DF8044B5DF8045B60
:1007580070470CF0FF0205F0FF00012828BF904207
:1007680004BF4FEA1C2C2D0AF3D0A2EB00005DF861
:10077800044B5DF8045B704780EA0102844612F07E
:10078800030F4FD111F0030F32D14DF8044D11F082
:10079800040F51F8043B0BD0A3F101329A4312F035
:1007A800803F04BF4CF8043B51F8043B16D100BF0E
:1007B80051F8044BA3F101329A4312F0803FA4F19F
:1007C80001320BD14CF8043BA24312F0803F04BF26
:1007D80051F8043B4CF8044BEAD023460CF8013B93
:1007E80013F0FF0F4FEA3323F8D15DF8044B70473D
:1007F80011F0010F06D011F8012B0CF8012B002A7B
:1008080008BF704711F0020FBFD031F8022B12F069
:10081800FF0F16BF2CF8022B8CF8002012F47F4F24
:10082800B3D1704711F8012B0CF8012B002AF9D12C
:10083800704700BF20F0030110F00300C0F1000072
:1008480051F8043B00F1040C4FEACC0C6FF00002A5
:100858001CBF22FA0CF213434FF0010C4CEA0C2C8B
:100868004CEA0C4CA3EB0C0222EA030212EACC126B
:1008780004BF51F8043B0430F4D013F0FF0F1FBF3E
:10088800013013F47F4F013013F47F0F18BF01308C
:10089800704700BFF0B4002A46D041EA000313F0C5
:1008A80003032CD1032A07460E4643D904680D6872
:1008B800AC423FD1043A37D0A4F1013525EA04040B
:1008C80014F0803F18BF18462CD1041D0D1D0EE0F2
:1008D80054F8043B55F8041BA3F101308B4220EA7D
:1008E800030027D1043A1FD010F0803F1ED1032AFD
:1008F80027462E46ECD820462946002A1DD00478E3
:10090800013A0D78AC420CD172B18CB1002302E0EF
:1009180093420BD064B1013310F8014FCD5CAC4267
:10092800F6D0601BF0BC70471046FBE70020F9E7E3
:100938002046F7E738463146E1E724782D78F0E796
:1009480041EA000313F0030F0B4670B414BF0024F0
:100958000124032A94BF002404F001040546D4B9F5
:10096800BAB10E782B46013A03F8016B56B1AC1CAC
:100978007AB111F8015F2346013A04F8015C0134A9
:10098800002DF5D12AB19A18002103F8011B9342D2
:10099800FBD170BC7047194653F8044BA4F10136DB
:1009A80026EA040616F0803FDAD1043A45F8044BEB
:1009B800032A1946EFD8D3E701232DE9F0071D468E
:1009C80000264FF0FF37AC1900EB070C8C420DD214
:1009D8001CF805C010F80480E0452ED201252646F3
:1009E800E31BAC198C4200EB070CF1D34FF0010963
:1009F80000264D464FF0FF3C1360AC1900EB0C0885
:100A0800A1420ED918F8058010F804A0C2451AD9D9
:100A180001252646CCEB0409AC19A14200EB0C08D1
:100A2800F0D80CF101000137B8423CBF994638466E
:100A3800C2F80090BDE8F00770470BD00123374695
:100A48001D46F618BFE709D04FF00109B4464D46D8
:100A58004E44D2E79D4205D00135B4E74D4505D057
:100A68000135CAE72B4626460125ACE7A9462646A6
:100A78000125C2E72DE9F04FADF5826D81B014462E
:100A8800074610460DF580628B460C3219461D4606
:100A9800FFF792FF03AE04A901F57E72331F0090A1
:100AA80043F8045F9342FBD14DB1681E0023E25C1A
:100AB800C11A013303AEAB4246F82210F7D1DDF874
:100AC8000C142046009A6118FFF78AFB002877D19A
:100AD8000099814605F1FF380646C1F101020192ED
:100AE8005A46AB4609EB0B0501F1FF3AB81800214D
:100AF800AA1A00F0E5F900284FD1002D00F0C080B7
:100B08007B1903A913F8013C51F82330002B4CD171
:100B1800009B9E4228BF334698450FD903EB090135
:100B2800E05C7A18795C884205D038E012F8011F39
:100B3800E05C884233D101339845F7D8009A964251
:100B480080F0A48007EB090214F80A10534612F843
:100B58000A20914204BF0AEB0901791807D095E0F1
:100B680014F802C011F8010D844503D113465A1E2A
:100B7800B342F5D101369E4200F28D80DDF80C6457
:100B88002A46B144C6EB0B0609EB0B05B818002141
:100B9800AA1A00F095F90028AFD0002071E0019A58
:100BA8000026914499442A46EEE7002EFAD0DDF853
:100BB8000C2493423CBFC2EB0B0306469944F2E770
:100BC800009E4FF000080099AB1BB34238BF334674
:100BD800C1F101026E1E019201F1FF3A5A4689469F
:100BE800AB460133CDF80C3408EB0B05B8180021DF
:100BF800AA1A00F065F90028CFD1002D40D07B1942
:100C080003A913F8013C51F82330002B30D1B1452A
:100C180013D208EB090314F80910FA18FB5C99427F
:100C280018BF4B4627D14B4604E012F8011FE05C81
:100C3800884220D10133B342F7D3BAF1FF3F53467C
:100C48002CD007EB080C14F80A101CF80A20914263
:100C58000CD10AEB0802BA1804E0E05C12F8011D96
:100C6800884203D1013BF8D260460AE0DDF80C3433
:100C780098442A46B8E701992A4688449844B3E735
:100C8800284605B00DF5806DBDE8F08F009B013654
:100C98009E427FF673AF07EB0900F2E707EB080CFB
:100CA8006046EEE72DE9F04F8346037885B00C46A1
:100CB800002B00F0F9800A78A2B106460131012024
:100CC80002E011F8012B8AB1934214BF002000F012
:100CD800010016F8013F0D46002BF2D12B782BB1FD
:100CE8004FF0000B584605B0BDE8F08F0028F9D149
:100CF8000BF101002178FFF7CBFB2D1BA5F10102B9
:100D0800534243EB0203002808BF43F001030746A0
:100D180083B90BEB0508404594BFC0EB08084FF0BA
:100D280001081F2D08D9414622462B46FFF7A2FE8F
:100D38008346D7E78346D5E7294603AA2046FFF727
:100D48003BFE03996118814620464A46FFF748FA58
:100D580000284FD109F1FF33C9F10102064601927B
:100D680082464246C84699460AEB050BB818002148
:100D7800C2EB0B0200F0A4F80028B1D1BBF1000FC0
:100D8800B0D046452CBF334643469D420FD903EBAE
:100D98000A01E05C7A18795C884205D075E012F89F
:100DA800011FE05C884270D101339D42F7D1B04504
:100DB8007DD907EB0A0214F809104B4612F80920EE
:100DC800914202BF09EB0A01AC46791806D06EE0E1
:100DD800A55C11F8010D854203D113465A1EB34292
:100DE800F6D1654601369E4267D8039E5A46B244FC
:100DF800AE1BB9E7C9F10101C9EB0503424600265C
:100E080009F1FF3A88464B4538BF4B4601330393F7
:100E180006EB050BB8180021C2EB0B0200F050F8E6
:100E280000287FF45DAFBBF1000F3FF45BAF4D4589
:100E380012D906EB090314F80910FA18FB5C994259
:100E480008BF4B4605D026E012F8011FE05C884237
:100E580022D101339D42F7D1BAF1FF3F534628D042
:100E680007EB060C14F80A101CF80A20914217D157
:100E78000AEB0602BA1804E0E05C12F8011D884289
:100E88000ED1013BF8D2E3462CE7019A00269244A2
:100E98005A469A4468E74B4646445A46F618B7E716
:100EA800039B5A46F618B3E70D46012016E743465A
:100EB80098E707EB060CE34614E707EB0A0B11E784
:100EC80010F0030F034670B4C9B211D0002A22D023
:100ED80003788B421DD0013A013005E0DAB110F8F1
:100EE800014B013A8C4218D010F0030F0346F5D19C
:100EF800032A14D87AB1187888420ED0541E5D1C83
:100F080003E015F8016B8E4203D0013C2846F8D265
:100F1800002070BC70471046FBE71846F9E741EA25
:100F2800012646EA0646184653F8044B86EA0404A6
:100F3800A4F1013525EA040414F0803F03D1043AF2
:100F48001846032AEFD80346D4E700BF0000000084
:100F5800C1F30A5C0246ACF57E7C2DE9F84FACF192
:100F68000704132C0B4606460F468946804627DCA5
:100F7800002C52DB4FF6FF7CC0F20F0C4CFA04FA3F
:100F88000AEA0105054317D037A3D3E9002300F087
:100F980075F80022002300F0B3FC002856D0002F7B
:100FA80005DD4FF4801353FA04F407EB040929EA2A
:100FB8000A0900264B46324610461946BDE8F88F06
:100FC800332C07DDB4F5806FF6D100F057F80246F0
:100FD8000B46F1E74FF0FF3BACF11B0C2BFA0CFB77
:100FE8001BEA000FE8D020A3D3E9002300F046F85D
:100FF8000022002300F084FC40B3002F0ADD142CEB
:1010080006D00126C4F13404A64016EB080601D325
:1010180007F1010926EA0B0619E013A3D3E9002317
:1010280000F02CF80022002300F06AFC78B1002FB1
:1010380013DB46EA07054FF000094D45C3F6F07982
:101048000CBF2E46002608BFA94600E0B9464B460D
:10105800324610461946BDE8F88F00264FF0004981
:10106800F5E700BFAFF300809C7500883CE4377E4D
:1010780081F0004102E000BF83F0004330B54FEA41
:1010880041044FEA430594EA050F08BF90EA020FAE
:101098001FBF54EA000C55EA020C7FEA645C7FEA41
:1010A800655C00F0E2804FEA5454D4EB5555B8BF64
:1010B8006D420CDD2C4480EA020281EA030382EAD5
:1010C800000083EA010180EA020281EA0303362D67
:1010D80088BF30BD11F0004F4FEA01314FF4801C3A
:1010E8004CEA113102D0404261EB410113F0004F4C
:1010F8004FEA03334CEA133302D0524263EB430303
:1011080094EA050F00F0A780A4F10104D5F1200EA0
:101118000DDB02FA0EFC22FA05F2801841F10001FB
:1011280003FA0EF2801843FA05F359410EE0A5F1CF
:1011380020050EF1200E012A03FA0EFC28BF4CF000
:10114800020C43FA05F3C01851EBE37101F00045B6
:1011580007D54FF0000EDCF1000C7EEB00006EEBC3
:101168000101B1F5801F1BD3B1F5001F0CD349084D
:101178005FEA30004FEA3C0C04F101044FEA4452A4
:1011880012F5800F80F09A80BCF1004F08BF5FEA2B
:10119800500C50F1000041EB045141EA050130BD0B
:1011A8005FEA4C0C404141EB010111F4801FA4F1AE
:1011B8000104E9D191F0000F04BF01460020B1FA03
:1011C80081F308BF2033A3F10B03B3F120020CDA3B
:1011D8000C3208DD02F1140CC2F10C0201FA0CF019
:1011E80021FA02F10CE002F11402D8BFC2F1200C7E
:1011F80001FA02F120FA0CFCDCBF41EA0C01904034
:10120800E41AA2BF01EB0451294330BD6FEA04047C
:101218001F3C1CDA0C340EDC04F11404C4F1200267
:1012280020FA04F001FA02F340EA030021FA04F379
:1012380045EA030130BDC4F10C04C4F1200220FAD0
:1012480002F001FA04F340EA0300294630BD21FA0E
:1012580004F0294630BD94F0000F83F4801306BFD4
:1012680081F480110134013D4EE77FEA645C18BFC8
:101278007FEA655C29D094EA050F08BF90EA020F5F
:1012880005D054EA000C04BF1946104630BD91EA57
:10129800030F1EBF0021002030BD5FEA545C05D15A
:1012A8004000494128BF41F0004130BD14F5800499
:1012B8003CBF01F5801130BD01F0004545F0FE410D
:1012C80041F470014FF0000030BD7FEA645C1ABF42
:1012D800194610467FEA655C1CBF0B46024650EA79
:1012E800013406BF52EA033591EA030F41F40021A5
:1012F80030BD00BF90F0000F04BF0021704730B52B
:101308004FF4806404F132044FF000054FF00001FF
:1013180050E700BF90F0000F04BF0021704730B5C0
:101328004FF4806404F1320410F0004548BF404295
:101338004FF000013EE700BF42004FEAE2014FEAEA
:1013480031014FEA02701FBF12F07F4393F07F4FC5
:1013580081F06051704792F0000F14BF93F07F4FF7
:10136800704730B54FF4607401F0004521F000413A
:1013780020E700BF50EA010208BF704730B54FF0C0
:1013880000050AE050EA010208BF704730B511F0C5
:10139800004502D5404261EB41014FF4806404F1FD
:1013A80032045FEA915C3FF4DCAE4FF003025FEA7F
:1013B800DC0C18BF03325FEADC0C18BF033202EB07
:1013C800DC02C2F1200300FA03FC20FA02F001FA61
:1013D80003FE40EA0E0021FA02F11444C1E600BF00
:1013E80070B54FF0FF0C4CF4E06C1CEA11541DBFB3
:1013F8001CEA135594EA0C0F95EA0C0F00F0DEF87E
:101408002C4481EA030621EA4C5123EA4C5350EA62
:10141800013518BF52EA033541F4801143F48013B3
:1014280038D0A0FB02CE4FF00005E1FB02E506F044
:101438000042E0FB03E54FF00006E1FB03569CF099
:10144800000F18BF4EF0010EA4F1FF04B6F5007F9F
:1014580064F5407404D25FEA4E0E6D4146EB060611
:1014680042EAC62141EA55514FEAC52040EA5E509A
:101478004FEACE2EB4F1FD0C88BFBCF5E06F1ED844
:10148800BEF1004F08BF5FEA500E50F1000041EB7B
:10149800045170BD06F0004646EA010140EA020028
:1014A80081EA0301B4EB5C04C2BFD4EB0C0541EA4A
:1014B800045170BD41F480114FF0000E013C00F35F
:1014C800AB8014F1360FDEBF002001F0004170BD83
:1014D800C4F10004203C35DA0C341BDC04F114049C
:1014E800C4F1200500FA05F320FA04F001FA05F228
:1014F80040EA020001F0004221F0004110EBD370F5
:1015080021FA04F642EB06015EEA430E08BF20EA20
:10151800D37070BDC4F10C04C4F1200500FA04F3C3
:1015280020FA05F001FA04F240EA020001F0004155
:1015380010EBD37041F100015EEA430E08BF20EAC8
:10154800D37070BDC4F1200500FA05F24EEA020E10
:1015580020FA04F301FA05F243EA020321FA04F03F
:1015680001F0004121FA04F220EA020000EBD370F6
:101578005EEA430E08BF20EAD37070BD94F0000FF6
:101588000FD101F00046400041EB010111F4801F2A
:1015980008BF013CF7D041EA060195F0000F18BFDB
:1015A800704703F00046520043EB030313F4801F17
:1015B80008BF013DF7D043EA0603704794EA0C0FD1
:1015C8000CEA135518BF95EA0C0F0CD050EA4106E7
:1015D80018BF52EA4306D1D181EA030101F0004164
:1015E8004FF0000070BD50EA410606BF104619468C
:1015F80052EA430619D094EA0C0F02D150EA013698
:1016080013D195EA0C0F05D152EA03361CBF1046D8
:1016180019460AD181EA030101F0004141F0FE4177
:1016280041F470014FF0000070BD41F0FE4141F4FB
:10163800780170BD70B54FF0FF0C4CF4E06C1CEAFB
:1016480011541DBF1CEA135594EA0C0F95EA0C0FB0
:1016580000F0A7F8A4EB050481EA030E52EA03356B
:101668004FEA013100F088804FEA03334FF080558C
:1016780045EA131343EA12634FEA022245EA1115B9
:1016880045EA10654FEA00260EF000419D4208BF6A
:10169800964244F1FD0404F5407402D25B084FEA17
:1016A8003202B61A65EB03055B084FEA32024FF4C3
:1016B80080104FF4002CB6EB020E75EB030E22BF20
:1016C800B61A754640EA0C005B084FEA3202B6EBE0
:1016D800020E75EB030E22BFB61A754640EA5C008F
:1016E8005B084FEA3202B6EB020E75EB030E22BF1F
:1016F800B61A754640EA9C005B084FEA3202B6EB20
:10170800020E75EB030E22BFB61A754640EADC00DE
:1017180055EA060E18D04FEA051545EA16754FEA40
:1017280006164FEAC30343EA52734FEAC2025FEA5E
:101738001C1CC0D111F4801F0BD141EA00014FF0ED
:1017480000004FF0004CB6E711F4801F04BF0143BE
:101758000020B4F1FD0C88BFBCF5E06F3FF6AFAEDA
:10176800B5EB030C04BFB6EB020C5FEA500C50F16A
:10177800000041EB045170BD0EF0004E4EEA1131ED
:1017880014EB5C04C2BFD4EB0C0541EA045170BDF4
:1017980041F480114FF0000E013C90E645EA060E38
:1017A8008DE60CEA135594EA0C0F08BF95EA0C0F66
:1017B8003FF43BAF94EA0C0F0AD150EA01347FF4AE
:1017C80034AF95EA0C0F7FF425AF104619462CE785
:1017D80095EA0C0F06D152EA03353FF4FDAE1046E8
:1017E800194622E750EA410618BF52EA43067FF439
:1017F800C5AE50EA41047FF40DAF52EA43057FF4C9
:10180800EBAE12E74FF0FF3C06E000BF4FF0010CD3
:1018180002E000BF4FF0010C4DF804CD4FEA410C37
:101828007FEA6C5C4FEA430C18BF7FEA6C5C1BD004
:1018380001B050EA410C0CBF52EA430C91EA030F85
:1018480002BF90EA020F0020704710F1000F91EAE2
:10185800030F58BF994208BF90422CBFD8176FEAB0
:10186800E37040F0010070474FEA410C7FEA6C5C7E
:1018780002D150EA013C07D14FEA430C7FEA6C5C85
:10188800D6D152EA033CD3D05DF8040B704700BFB1
:101898008446104662468C461946634600E000BFFF
:1018A80001B5FFF7B7FF002848BF10F1000F01BDD1
:1018B8004DF808EDFFF7F4FF0CBF012000205DF89C
:1018C80008FB00BF4DF808EDFFF7EAFF34BF012021
:1018D80000205DF808FB00BF4DF808EDFFF7E0FFBA
:1018E80094BF012000205DF808FB00BF4DF808ED0B
:1018F800FFF7CEFF94BF012000205DF808FB00BF72
:101908004DF808EDFFF7C4FF34BF012000205DF853
:1019180008FB00BF4FEA4102B2F1E04324BFB3F530
:10192800001CDCF1FE5C0DD901F0004C4FEAC0024E
:101938004CEA5070B2F1004F40EB830008BF20F032
:101948000100704711F0804F21D113F13872BCBFEC
:1019580001F00040704741F480114FEA5252C2F141
:101968001802C2F1200C10FA0CF320FA02F018BF8A
:1019780040F001004FEAC1234FEAD32303FA0CFCDD
:1019880040EA0C0023FA02F34FEA4303CCE77FEA6C
:10199800625307D150EA01331EBF4FF0FE4040F4B6
:1019A8004000704701F0004040F0FE4040F4000065
:1019B800704700BF80F0004002E000BF81F00041A6
:1019C80042001FBF5FEA410392EA030F7FEA226CDD
:1019D8007FEA236C6AD04FEA1262D2EB1363C1BF6D
:1019E800D218414048404140B8BF5B42192B88BFDC
:1019F800704710F0004F40F4000020F07F4018BFFF
:101A0800404211F0004F41F4000121F07F4118BF1E
:101A1800494292EA030F3FD0A2F1010241FA03FCC6
:101A280010EB0C00C3F1200301FA03F100F00043AE
:101A380002D5494260EB4000B0F5000F13D3B0F176
:101A4800807F06D340084FEA310102F10102FE2AE5
:101A580051D2B1F1004F40EBC25008BF20F0010055
:101A680040EA03007047490040EB000010F4000F03
:101A7800A2F10102EDD1B0FA80FCACF1080CB2EB96
:101A88000C0200FA0CF0AABF00EBC25052421843F5
:101A9800BCBFD0401843704792F0000F81F400019A
:101AA80006BF80F400000132013BB5E74FEA41036D
:101AB8007FEA226C18BF7FEA236C21D092EA030FD9
:101AC80004D092F0000F08BF0846704790EA010F53
:101AD8001CBF0020704712F07F4F04D1400028BF80
:101AE80040F00040704712F100723CBF00F5000062
:101AF800704700F0004343F0FE4040F40000704798
:101B08007FEA226216BF08467FEA23630146420243
:101B180006BF5FEA412390EA010F40F48000704756
:101B28004FF0000304E000BF10F0004348BF4042FC
:101B38005FEA000C08BF704743F0964301464FF038
:101B480000001CE050EA010208BF70474FF0000394
:101B58000AE000BF50EA010208BF704711F00043D5
:101B680002D5404261EB41015FEA010C02BF8446A5
:101B78000146002043F0B64308BFA3F18053A3F504
:101B88000003BCFA8CF2083AA3EBC25310DB01FA4B
:101B980002FC634400FA02FCC2F12002BCF1004FCF
:101BA80020FA02F243EB020008BF20F00100704760
:101BB80002F1200201FA02FCC2F1200250EA4C00B4
:101BC80021FA02F243EB020008BF20EADC707047FA
:101BD8004FF0FF0C1CEAD0521EBF1CEAD15392EA08
:101BE8000C0F93EA0C0F6FD01A4480EA010C4002E4
:101BF80018BF5FEA41211ED04FF0006343EA50103E
:101C080043EA5111A0FB01310CF00040B1F5000F7F
:101C18003EBF490041EAD3715B0040EA010062F12E
:101C28007F02FD2A1DD8B3F1004F40EBC25008BF18
:101C380020F00100704790F0000F0CF0004C08BF36
:101C480049024CEA502040EA51207F3AC2BFD2F103
:101C5800FF0340EAC250704740F400004FF0000311
:101C6800013A5DDC12F1190FDCBF00F0004070474B
:101C7800C2F10002410021FA02F1C2F1200200FA89
:101C880002FC5FEA310040F1000053EA4C0308BF50
:101C980020EADC70704792F0000F00F0004C02BFA1
:101CA800400010F4000F013AF9D040EA0C0093F01C
:101CB800000F01F0004C02BF490011F4000F013B76
:101CC800F9D041EA0C018FE70CEAD15392EA0C0FE4
:101CD80018BF93EA0C0F0AD030F0004C18BF31F04F
:101CE800004CD8D180EA010000F00040704790F025
:101CF800000F17BF90F0004F084691F0000F91F0C9
:101D0800004F14D092EA0C0F01D142020FD193EA8E
:101D18000C0F03D14B0218BF084608D180EA010016
:101D280000F0004040F0FE4040F40000704740F0F2
:101D3800FE4040F4400070474FF0FF0C1CEAD052C0
:101D48001EBF1CEAD15392EA0C0F93EA0C0F69D01C
:101D5800A2EB030280EA010C49024FEA402037D087
:101D68004FF0805343EA111143EA10130CF000407E
:101D78008B4238BF5B0042F17D024FF4000C8B426E
:101D880024BF5B1A40EA0C00B3EB510F24BFA3EB4E
:101D9800510340EA5C00B3EB910F24BFA3EB91031E
:101DA80040EA9C00B3EBD10F24BFA3EBD10340EA78
:101DB800DC001B0118BF5FEA1C1CE0D1FD2A3FF6BE
:101DC80050AF8B4240EBC25008BF20F00100704773
:101DD8000CF0004C4CEA50207F32C2BFD2F1FF0316
:101DE80040EAC250704740F400004FF00003013A47
:101DF80037E792F0000F00F0004C02BF400010F4EB
:101E0800000F013AF9D040EA0C0093F0000F01F0FE
:101E1800004C02BF490011F4000F013BF9D041EA20
:101E28000C0195E70CEAD15392EA0C0F08D1420253
:101E38007FF47DAF93EA0C0F7FF470AF084676E726
:101E480093EA0C0F04D14B023FF44CAF08466EE7FF
:101E580030F0004C18BF31F0004CCAD130F00042CD
:101E68007FF45CAF31F000437FF43CAF5FE700BF25
:101E78004FF0FF3C06E000BF4FF0010C02E000BF4E
:101E88004FF0010C4DF804CD4FEA40024FEA4103F0
:101E98007FEA226C18BF7FEA236C11D001B052EAA6
:101EA800530C18BF90EA010F58BFB2EB030088BF6C
:101EB800C81738BF6FEAE17018BF40F001007047DB
:101EC8007FEA226C02D15FEA402C05D17FEA236CBD
:101ED800E4D15FEA412CE1D05DF8040B704700BF04
:101EE800844608466146FFE70FB5FFF7C9FF00289B
:101EF80048BF10F1000F0FBD4DF808EDFFF7F4FFD4
:101F08000CBF012000205DF808FB00BF4DF808ED6C
:101F1800FFF7EAFF34BF012000205DF808FB00BF8F
:101F28004DF808EDFFF7E0FF94BF012000205DF8B1
:101F380008FB00BF4DF808EDFFF7D2FF94BF012062
:101F480000205DF808FB00BF4DF808EDFFF7C8FF5B
:101F580034BF012000205DF808FB00BF42000ED20C
:101F6800B2F1FE4F0BD34FF09E03B3EB126209D4CC
:101F78004FEA002343F0004323FA02F070474FF082
:101F88000000704712F1610F01D1420202D14FF0F7
:101F9800FF3070474FF00000704700BF00F026F890
:101FA8000C4880F30888002103E00B4B5B58435032
:101FB80004310A480A4B42189A42F6D3094A02E009
:101FC800002342F8043B084B9A42F9D318F0E0F991
:101FD8007047000000C0002090580308000000204F
:101FE80060130020601300204C6000207047FEE75B
:101FF80010B586B0002301244FF46022114801A9CE
:1020080001938DF80930039204938DF808408DF8F8
:10201800144023F0A7FA0B48214623F0C9FA0948CF
:1020280023F0D0FA074823F0D2FA0028FAD105485D
:1020380023F0D1FA034823F0D3FA0028FAD106B0E6
:1020480010BD00BF00240140014610B50D48012213
:10205800032323F0D3FA0B48012123F0C5FA7F208C
:1020680024F002F90748022123F012FB0028F6D0D9
:102078000448022123F012FB0248BDE8104023F077
:1020880004BB00BF002401400C4A0C2303FB0123BE
:1020980010B59C880CB9588010BD5B8803F11304F7
:1020A800844204DA142B07D9133B834204DC0C2343
:1020B80003FB012102238B8010BD00BF742E00207A
:1020C8000A4B10B500241C7021464FF4E0720848F2
:1020D800FEF760F9074B43F604501C70064B1C7062
:1020E8000FF0B0FC054B187010BD00BFDC150020C8
:1020F800A8170020F3190020701900207219002079
:10210800074B1978013101F01F011970054B1A7836
:102118008A4203D1013202F01F021A70704700BFD1
:1021280070190020F319002010B50E4A0E2303FB86
:1021380000200D4A014614780C4A03FB042300F1E1
:102148000C0251F8044B914243F8044BF9D10A8828
:1021580000211A800E22FEF71DF9BDE81040FFF796
:10216800CFBF00BFE015002070190020A81700207D
:10217800084B1A5C002352FA03F111F0010FD8B290
:1021880002D00130C0B270470133042BF3D10120D3
:10219800704700BFAB1A002000F07F0000F57450B4
:1021A8002DE9F84309300C46154698460FF04AFCCD
:1021B80000284FD043F63C37002638460FF042FC43
:1021C800C0B25FFA86F988B120280FD04FEA5900CB
:1021D80000F5364037300FF035FCC0B208B10228A0
:1021E80004D10123B340227813432370113743F6F7
:1021F800C43301369F42E0D14BF2DE400FF022FC9F
:10220800C0B280B120280ED02B784BF2CD4043F0DD
:1022180001032B700FF016FCC0B220B1202802D0A9
:10222800012388F800304BF20F500FF00BFCC0B2BE
:1022380080B120280ED02B784BF2CD4043F002031A
:102248002B700FF0FFFBC0B220B1202802D0012371
:1022580088F80030BDE8F883034610465A1E10B5CA
:10226800032A1CD8DFE802F00E0E0207114A527842
:1022780002F0100203E00F4A527802F00802D2B2CC
:1022880072B10BE00C4A927802F04002D2B23AB135
:102298000A4A127802F003029A4200D140B10022A1
:1022A8000748105C984203D00132052AF8D1002172
:1022B800084610BD5C5E0020783A00202B3D0020C7
:1022C800A0170020F8B5064643F63C3500242846FA
:1022D8000FF0B8FBC0B2E7B268B120280BD078087D
:1022E80000F5364037300FF0ADFB012803D1A04090
:1022F80033781843307001341135082CE7D1F8BD14
:1023080003780E2202FB0313084AD3189978002396
:1023180051FA03F010F00100DAB202D0501CC0B23A
:1023280070470133082BF3D1704700BFA81700206E
:102338002DE9F04101248C40284A29490346E4B29A
:10234800107891F800C019E0264F0E2606FB00769B
:10235800F178A9B996F80680B8F1000F10D196F86F
:102368000580B8F1000F0BD196F80480B8F1000F82
:1023780006D1F67926B9013000F01F00054626E09F
:10238800FBB1012B05D0022B06D10E2101FB0077F2
:1023980039790C4218D014E0042B04D10E2101FB2A
:1023A8000077B9790CE0032B04D10E2101FB0077EB
:1023B800797905E0052B07D10E2101FB0077F97922
:1023C80011B11570BDE8F081013000F01F006045C3
:1023D800BAD11570FF20BDE8F08100BFF3190020C5
:1023E80070190020A81700202DE9F043444D454BF3
:1023F8002A780E2101FB0232917A85B0044698466C
:1024080039B101390523594301F56E51443189B277
:1024180001E043F6C431204604220FF024FB2B7858
:102428000E2505FB038393F80B80364E344FB8F125
:10243800000F25D131232371073363713B7801A83D
:102448006B430422F15E06F0D3FA3B7802A805FB41
:1024580003630222997A06F0CBFA3B780DF10A0061
:1024680005FB03650322697A06F0C2FAA01D01A9DB
:102478000922FEF765FA4FF00F0984F8108012E080
:10248800B8F1010F0FD132232371053363713B7803
:102498004FF0080905FB036393F90130E3713B78BA
:1024A8005D43735BA371002320461A4612E010F8BF
:1024B800011BA1F13005EDB2092D04D8EB18302924
:1024C800DBB203D004E037395B1800E00A33DBB233
:1024D8000132D2B24A45EAD10F21B3FBF1F108012A
:1024E800411A5B1AC3F10F03DBB2092BA35401D8BD
:1024F800303300E03733A35405B0BDE8F08300BFA4
:10250800A6170020A8170020024B1A7842F00102F3
:102518001A707047111D002008B50C4B0C4A1B7827
:102528000E2101FB0323D97A21B101290CBF09210E
:10253800002100E0102140221346064806F07CF8EE
:10254800054B1A7842F002021A7008BDA61700203F
:10255800A817002073190020111D0020034B1A78BA
:1025680002F0F8026FF3C3021A707047111D0020C1
:10257800024B1A7842F004021A707047111D0020AD
:10258800024B1A7842F008021A707047111D002099
:1025980038B5114B1C7814F0010502D1FFF7B4FFD0
:1025A80005E004F00405EDB21DB9FFF7E1FF284688
:1025B80038BD04F00805EDB215B9FFF7E1FFF6E7FD
:1025C80004F00204E4B21CB9FFF7A6FF204638BDA8
:1025D800FFF7C4FF012038BD111D0020014B1878FA
:1025E800704700BFDC15002030B51E4B85B01B7846
:1025F8000446002B34D11C4D2B78034113F0010FF6
:102608002ED01A4B1A4A1B780E2101FB0323DA78C5
:10261800024112F0010F1CD11B79034113F0010391
:1026280017D110F0010001F1F1014FEA540206D070
:1026380001320091019302926D20FE3905E00132CA
:102648000091019002923C20012103220B460FF0D9
:1026580077FA012313FA04F42B7823EA04042C7084
:1026680005B030BD7219002069190020F319002047
:10267800A8170020037830B513F0010F144A4FF063
:102688000E0419D104FB01210133012212FA03F3CC
:10269800CD7825EA0303CB7004780D79A41812FAD3
:1026A80004F425EA04040C7103789B189A408B788B
:1026B80023EA02028A7030BD04FB0121013B01229A
:1026C80012FA03F38A7822EA03038B7030BD00BF45
:1026D800A817002010B500230278590052FA01F417
:1026E80004F00304022C05D1013414FA01F122EAA2
:1026F800010202700133042BEED110BD2DE9F04F19
:1027080085B00192BDF838201C46744B0092DA78E7
:10271800054612F020028B4640F0D9808DF80E2035
:102728008DF80F208DF80D20DCB99B7803F040035D
:10273800DBB21BB101238DF80F3020E0684B5B78CA
:1027480003F00203DBB21BB101238DF80E3016E053
:102758000DF10F010DF10E020DF10D03FFF71CFD38
:102768000DE0012C0BD19B7803F04003DBB223B9B9
:102778000DF10F00FFF7A6FD01E08DF80F409DF861
:102788000F3023B99DF80E00002800F0A38044B94B
:1027980005F07F01490001F574510DF10A00663119
:1027A8000AE0012C0BD1E90101F51C4101F5B471D6
:1027B8000DF10A0001EB4B0102220FF054F9BDF9AB
:1027C8000A3013B9002C00F08480009B33B9454BC4
:1027D800454F93F80080FFF793FC08E0434B444FC4
:1027E80093F8008008F1010202F01F021A700DF13F
:1027F8000F00FFF76FFF002C44D1BDF80A3069B213
:1028080040F6B83212EA210238BF4FF47A72D21871
:102818000E2303FB08F3ADF80A20FA529DF80F9037
:10282800224649460120FE18FFF716FD4946F0707A
:1028380022460220FFF710FD86F8029030719DF8BD
:102848000E90224649460420FFF706FD4946B0711E
:10285800824622460320FFF7FFFC05F07F057071D2
:102868003572BAF1000F00D128B1224B1B7813B989
:102878009DF80D3000E00023F37186F809B0019A45
:10288800B2721CE0012C1AD10E2303FB08F3BDF829
:102898000A202046FA529DF80F6000223146FD18A2
:1028A800FFF7DAFC3146E87000220220FFF7D4FC7B
:1028B80000232871AE70AB716B71EB71AB720E2394
:1028C80003FB0877FC72009B0120BB8102E000201B
:1028D80000E0204605B0BDE8F08F00BF783A002040
:1028E8005C5E002070190020A8170020DB1500206E
:1028F800E0150020F61C002073B5154B04461B7824
:102908000E46D3B11348214621F0D3FF0546A0B99E
:10291800012E04F1010606D12046FFF729FC009597
:102928000246812005E02046FFF722FC009502467A
:10293800982031462B46FFF7E1FE2146054821F055
:10294800A2FF0548214602B0BDE8704021F0A6BFAD
:1029580071190020161C00200E1A00202DE9F743DB
:102968007B4B04461B7843B17A4B1B7803F0240356
:10297800042B02D1002900F0E880774B774F1B78B1
:10298800002B00F0C7807648214621F092FF0028EE
:1029980040F0C08007F5C470214621F08AFF8046C8
:1029A800002840F0B7803B1993F880302D2B01D0D8
:1029B800532B3AD16B4E357845B30FF09FFB04F19A
:1029C8000108054650B12046FFF7D2FB337802468E
:1029D8001E33009393204146002307E02046FFF76B
:1029E800C7FB00950246414693202B46FFF786FE1B
:1029F8000FF084FB014628B1337803201E3300937F
:102A0800002101E0009003200A4680E02046FFF7FD
:102A1800AFFB611C02462B4693200095FFF76EFE24
:102A28000095032029462A4671E0542B09D12046F7
:102A3800FFF79EFBCDF800800246611C94204346B8
:102A480066E0462B474D20D12E78BEB10FF056FBDD
:102A580004F10109064648B12046FFF789FB2B78A7
:102A680002461E3300939A20494622E02046FFF78B
:102A78007FFB0096024649469A2025E02046FFF74C
:102A880077FB009602469A2039E02E78002E2CD04B
:102A98000FF034FB04F11C09064660B12046FFF72D
:102AA80067FB2B7802461E3369F07F000093C0B2A3
:102AB800611C434609E02046FFF75AFB024669F0CD
:102AC8007F000096C0B2611C3346FFF717FE0FF077
:102AD80015FB21B2024628B12B7803201E33009340
:102AE800002214E00090032011E02046FFF740FB8D
:102AF800024604F11C0060F07F000096C0B2611C21
:102B08003346FFF7FBFD009603202146324601239A
:102B1800FFF7F4FD124821463F1921F0B4FE97F85B
:102B280080302D2B0AD0532B08D0542B06D0462B9F
:102B380004D00D48214621F0BCFE30B10B48214697
:102B480003B0BDE8F04321F0A9BE03B0BDE8F083AF
:102B5800DE150020041C002071190020A02C002084
:102B6800161C00206E1C0020282E00200E1C0020A1
:102B7800002302780E2101FB0232044901338A182E
:102B88000021062B9170F4D1704700BFA8170020D0
:102B9800064B00201870064B1A78064B1B789A4291
:102BA80002D00146FFF7C4BBFF207047DC150020A8
:102BB80070190020F31900200121814038B5114B0C
:102BC800C9431A78104BC9B202F0030203F5E07446
:102BD800012A04D1DD7801EA0505DD7005E0022A45
:102BE80003D11D7901EA05051D710E33A342EFD10A
:102BF800FFF7FAFC43F604500EF024FF034B18705D
:102C080038BD00BF2B3D0020A817002072190020F6
:102C18002DE9F743A34D8DF807002B78A24C1BB183
:102C28002378C2B29A4204D043F604500EF00AFF49
:102C380028709DF8073023709C4C2278072A00F2F0
:102C48002D81DFE812F008002400360054005D00F2
:102C580072008D00BA00964A3C211170954A1946B7
:102C6800107800F00300FFF763FB934BFF28187000
:102C780000F0368120F01EFB904B002093F8742062
:102C880042F0010283F874208D4B187064E0884B81
:102C98001B78002B00F0248120F0D4FC012840F0A0
:102CA8004D812378142201332370864B01381A7022
:102CB80047E17F4B1B78002B00F01281814E307862
:102CC80008B901234AE020F0BDFC022804D020F016
:102CD800B9FC032840F0328120F0ECFA2378042272
:102CE800013323701D233370774B1A7026E1704B24
:102CF8003C221A707548FFF777FB2378013323705D
:102D08006B4B1B78002B00F0EB806E4B1D78002D71
:102D180040F014811020FFF73BFC002800F01181DF
:102D280023782846013323700BE1614B1B78002B75
:102D380000F0D68005F0EAFC002800F00281614B23
:102D48007D221A705E4B002018705C4B93F874203B
:102D580042F0010283F87420237801332370F0E0F5
:102D6800534B1B78002B00F0BB8020F06BFC012834
:102D7800544E03D020F066FC03280FD19DF807209D
:102D8800012111FA02F2524B197821EA02021A7053
:102D980064233370237801332370CFE03078002820
:102DA80040F0CC80484A032323701378013BDBB200
:102DB8001370002B00F09480C3E0404A414E92F813
:102DC8006A201AB13278002A40F0B88000223270A6
:102DD800013212FA03F3DFF8E0803E4F98F8001052
:102DE8004FF00E0909FB0172DB4392F803E0DBB2F6
:102DF80003EA0E0E907882F803E092F804E003EA02
:102E08000E0E0340937082F804E00DF10700FFF7FF
:102E180031FC98F8003009FB0372D278DFF89490FF
:102E28002AB999F8002002F00302012A0AD00E22DA
:102E380002FB03721279B2B999F8002002F003027A
:102E4800022A10D10E2202FB0377BA785AB9224F10
:102E58003A789A4207D11848FFF78AFE3B7801333F
:102E680003F01F033B7099F800009DF8071000F06D
:102E78000300FFF75DFA144B0422FF281A7088F844
:102E88000000164B42D0987800F04000C0B20028ED
:102E98003CD1032323701A33337052E00020207092
:102EA8004FE000BF72190020DF150020DC1500205C
:102EB8006A1900202B3D0020A6170020B03C0020F6
:102EC800DD150020DA15002068190020731900208C
:102ED80069190020A8170020F3190020783A00206B
:102EE800FFF73CFB0023237020F0E4F92B78013B2B
:102EF800DBB22B702BB1144B9B7803F04003DBB291
:102F0800F3B19DF80700FFF757FE19E09B780E4ACA
:102F180003F04003DBB22BB1136843F400031360E2
:102F2800FFF7CEF8FFF71AFB20F0C4F9002323704F
:102F380043F604500EF086FD287001E0002000E002
:102F4800FF20BDE8FE8300BF783A0020044B1A78C2
:102F58000AB1013A1A701B780BB9FFF72DBE7047FA
:102F680072190020044A054B10781B7803EA5010A8
:102F780000F00100704700BF783A0020DD1B0020F8
:102F8800044B054A1B781078C3F3400303EA10107A
:102F9800704700BFDD1B0020783A0020034B044A2D
:102FA8001B78D078C3F3800318407047DD1B0020DE
:102FB800783A0020044B054A1B78D078C3F3C00345
:102FC80003EA5000704700BFDD1B0020783A00205C
:102FD800044B054A1B78D078C3F3001303EA90002A
:102FE800704700BFDD1B0020783A0020044B18789A
:102FF800044BDB785B005BB2DB1103EAD01070474F
:10300800DD1B0020783A002008B50E2104481CF08A
:10301800B7FB044B5B7803EA000000F0010008BD31
:10302800FC190020DD1B002070B500241BE0304691
:10303800E9B21CF0E3FB80B14FF4366363433422FA
:1030480002FB05330A4AD3181B7A13F0010F04D088
:10305800084B1878C0F3001070BD0135382DE6D143
:103068000134022C02D0E6B20025E0E7002070BD52
:10307800043E0020DD1B002008B51BF0DBFC034BE1
:103088001B7800EA931000F0010008BDDD1B00204A
:10309800044B054A1B78D078C3F3401303EAD000E9
:1030A800704700BFDD1B0020783A00202DE9F74F5C
:1030B800FFF758FF8246FFF763FF8346FFF76EFF6F
:1030C8000190FFF777FF8146FFF782FF0446FFF77D
:1030D800ABFF0546FFF7DCFF8046FFF7CDFF07464D
:1030E800FFF784FF0646FFF78FFF019B45EA0404BC
:1030F8009B0043EA4B0343EA0A0343EAC90343EA52
:10310800481343EA871343EAC61343EA0023E0B2AD
:1031180043EA0010BDE8FE8F044B987800F00F00DA
:10312800A0F10203584240EB030070474B1A0020FD
:10313800044B987800F00F00A0F10102504240EBD8
:10314800020070474B1A0020044B987800F00F00DB
:10315800A0F10301484240EB010070474B1A0020E0
:10316800054B987800F00F00A0F1060CDCF1000088
:1031780040EB0C00704700BF4B1A0020514AF0B5D5
:1031880013781446012B29D003D3022B40F09880E2
:103198005EE04D484D4B047819786FF3C304047012
:1031A80001F0F80158786FF3C301197000F080013D
:1031B800C9B2002900F08480012111709C78062290
:1031C80004F00F04544302464148005D60F30602D0
:1031D8005A701A7861F302021A70F0BD3B494D78B3
:1031E8000B4625F07F00002838D00A7802F0080244
:1031F800D2B222B9344A117841F0080111709A7894
:1032080002F00F02012A04D12F4A117841F001017E
:10321800117015F07F0F53D119789E7801F00700CF
:10322800062206F00F0602FB0606294F5D78BE5DF2
:10323800013066F3060500F007005D7090FBF2F5BB
:1032480002FB150262F30201197002232370F0BD1C
:103258001E494D780B4625F07F0028B98B7860F31E
:1032680003038B701070F0BD174A11786FF3C30118
:103278001170997801F00F01012903D111786FF3CA
:103288000001117015F07F0F1AD119789E7801F09E
:103298000700062206F00F0602FB06060C4F5D78B3
:1032A800BE5D013066F3060500F007005D7090FB17
:1032B800F2F502FB150262F3020119700123237073
:1032C800F0BD00BF9A1A00200D1A00204B1A0020EA
:1032D8001063020810B51F4A1F4B92F9031009B179
:1032E800002231E008B1032119701978032930D878
:1032F800DFE801F00209192C1178002929D01548B6
:1033080081700121197092F90200124920B1134B02
:103318001A786FF3861217E0487808B9032213E089
:1033280088700221197092F902100A4889B90B4A6B
:10333800147861F386141470026861F30F22D1B215
:1033480061F31742026001221A7010BD002111605A
:10335800197010BD701C00200B1A0020043C0020BE
:1033680070B543F6EF23044643F6F020012A08BF60
:1033780018460D460EF066FB2678C0B20640164C7D
:103388000CD001201CF000FC43F6EE200EF05AFB96
:10339800236860F307036FF30F2314E02B781842B8
:1033A80012D030461CF0F0FB0C4B43F6EE201A8886
:1033B80066F34D321A800EF045FB2368C0B260F305
:1033C800070360F30F23236094F9003013B1024B15
:1033D8000F22DA7070BD00BF701C0020041C002092
:1033E80008B543F6FB200EF02DFB014B187008BD05
:1033F8000C1A0020014B1870704700BFE71B002013
:10340800024B1A5C6FF303021A547047F41A002037
:1034180070B50C46C10001F5CE411B48BF310822EA
:103428000EF021FB002518482946EEB221F041FA9A
:1034380008B9237823BB154B2278EB5C1A421FD1BD
:103448003046FFF7DDFFF6084BF2DF5030180EF07C
:10345800F9FA05F00703C0B2184110F0010F0FD1B7
:103468000B48294621F025FA50B12946084821F091
:1034780015FA074B06F5CC40CE30995D0EF0D8FA18
:103488000135402DCFD170BDE91B0020AB1A0020BB
:103498004E1A002038B546F2167540242046FFF72C
:1034A800AFFFA5F5CC43094AD63BD15C11F0100F0C
:1034B80006D06FF30411D154284600210EF0B8FA53
:1034C8000134E4B20135E92CE8D138BDF41A002002
:1034D8003F287FB5054607D800F5E24041300EF099
:1034E800B1FAC3B22BB92AE1994A1478002C00F03A
:1034F8002B81984E725D02F00F014C1C04F00F04F2
:1035080064F303023F2D725533D8002C00F01C8160
:1035180001339C4240F015818F4B5A1992F8802054
:10352800522A725D03D161F30302725509E16FF308
:103538000302EC081B19725593F8902105F0070354
:1035480052FA03F313F0010F40F0FD802946834837
:1035580021F099F9814B04F5CC40195DCE30012456
:103568000EF066FA2D190223009301940295182093
:10357800CEE0002C00F0E880754B1B7801339C42AC
:1035880040F0DF80735D05F5CC406FF30303D63060
:10359800012173550EF04CFA735D43F01003735517
:1035A800A5F14003DBB2032B07D8042200920133B4
:1035B80002320192029319202FE0A5F14803DBB2F1
:1035C800032B07D80422009201330332019202939D
:1035D8001A2060E0A5F15003DBB2012B07D80422C2
:1035E800009201330332019202931B2053E0572DBE
:1035F80007D104230093012403330193029421206B
:1036080086E0A5F15B03DBB2012B09D80422009206
:10361800013302320192029322200121033A8AE007
:103628005D2D06D1042300930193043B02932846A1
:103638007FE05E2D07D10423009301330193053BFE
:1036480002935E2075E0A5F15F03DBB26F2B09D80A
:10365800042200920133921801920293332001212F
:10366800053A68E005F13103DBB2032B07D80422E1
:10367800009201330332019202935F200BE005F1BF
:103688002903DBB2012B09D804220092013303324B
:103698000192029360200121043A4CE0DA2D07D10F
:1036A800042300930124043B0194029361202FE03A
:1036B800D92D07D104230093023B0193023B0293C7
:1036C800622036E0DD2D08D1042300930322043B59
:1036D80001920293632001212DE0DB2D06D1042302
:1036E8000093043B01930293642022E0DC2D06D171
:1036F80004230093043B01930293702019E0DE2D0C
:103708000CD104230093012402330193029468200E
:103718002146032223460EF013FA15E01E35EDB2BA
:10372800012D10D80423009301350233019302952B
:103738006A20012103220B460EF002FA03E01C4620
:1037480002E0002400E00124204604B070BD00BF60
:1037580000000020F41A0020A02C00204E1A00209F
:10376800024B185CC0F30010704700BFF41A002029
:10377800F8B508220E4600210746FCF70BFE46F274
:10378800BF7500243378234113F0010F08D0294670
:10379800064808220EF067F93846044921F041F836
:1037A80001340835042CEDD1F8BD00BFF31B00200F
:1037B800024846F2CE6108220EF055B94E1A002092
:1037C80070B5044600F56A5044300EF03BF90B4DD5
:1037D80006462B7813F0010F02D1CC2021F056FEBB
:1037E8002B8843F001032B80054B1E55054B13F81E
:1037F800242042F0010203F8242070BD041C00209C
:103808002F1A00201E1A0020024B185C084100F0F5
:1038180001007047AB1A002070B505460024094B1B
:10382800E0B2E618E35C4BB12946FFF7EDFF28B19B
:10383800002333700448214621F030F80134402C2D
:10384800EDD170BD261C00203B1A002038B5054676
:1038580000242846E1B2FFF7D7FF10B1044BE35C20
:1038680023B90134042CF4D1002038BD012038BD1F
:103878002F1A002038B505460EF040FCA0B10024F0
:103888002846E1B2FFF7C0FF40B1084B13F82430D7
:1038980013F0010F02D0064BE35C23B10134042C72
:1038A800EED1002038BD012038BD00BF1E1A00200F
:1038B8002F1A0020F8B5114800214022FCF76AFDB4
:1038C80046F2BF75002401270D4829460822A74063
:1038D8000EF0C9F8FFB200260948314620F0E9FF8A
:1038E80020B1064BF25C47EA0202F2540136402E40
:1038F800F2D101340835042CE5D1F8BDAB1A00200B
:10390800F31B00202DE9FF4100263446B0461A4B30
:103918001B78234113F00102184B23D0184F1D5D6B
:1039280017F82430A84538BFA84613F0010F1AD05D
:10393800CDB965F3000307F8243023B20122F71943
:1039480002935B2029462B46009201950EF0F8F869
:103958007B78B878F9781843621C2B460095FEF7F7
:10396800CDFE00E01A5501340436042CCFD1054BA6
:1039780083F80080BDE8FF810C1A00202F1A002070
:103988001E1A00200A1A002010B50C4B1B78A3B190
:103998000B4B1B788BB100240A48214620F089FF85
:1039A80040B10948214620F084FF18B9204601217A
:1039B800FEF7D4FF0134402CEED110BD7119002060
:1039C800DE1500200E1C00209E2300202DE9F04368
:1039D800324C334A238800266FF386136FF3C403EF
:1039E8002380304B304F85B016701E709146984634
:1039F80017F8013B5BB32278D20052B243EAA21215
:103A08002388402E62F3C40343F0400323801ED072
:103A180000253046E9B2FFF7F7FEA8B117F8013CD8
:103A280013F0010F06D00122AA4099F800100A43AA
:103A380089F8002013F0020F06D00123AB4098F854
:103A48000020134388F800300135042DE1D10136F8
:103A5800F6B2412ECCD1237803F04005EDB2D5B9AA
:103A680003F02403042B0BD1FFF78EFFFF230093F1
:103A78004020294601222B46019502950EF060F858
:103A8800238800226FF345136FF382036FF3C40397
:103A98002380064B1A7005B0BDE8F083041C002093
:103AA800A03B0020BD3B0020591A0020E81B002045
:103AB80010B500240548214620F0FBFE08B9044B48
:103AC800E0540134402CF5D110BD00BFDF1B0020AD
:103AD800591A002010B5127804469DF80810DAB17A
:103AE800D3B111B10D4920F091FEACB1082246F2D4
:103AF800CE610B480DF0B7FF2146094820F091FE32
:103B08000749082246F2CE600DF0A7FF0548044990
:103B1800BDE8104020F09BBE10BD00BF382E00202D
:103B2800F41900204E1A002030B5064B04781D7891
:103B380024EA05040C7001781B7823EA010313704A
:103B480030BD00BF0C1A002038B50A4D002415F806
:103B5800013F2D2B09D0532B07D0542B05D0462BD2
:103B680003D00548214620F099FE0134402CEED1BF
:103B780038BD00BF1F2D00200E1C002010B50F48B7
:103B880020F03CFE00240E48214620F092FE80B131
:103B98000C4BE31893F88030482B06D003D82D2B14
:103BA80003D0462B00E0542B03D10448214620F0D3
:103BB8006AFE0134402CE6D110BD00BF9B1A0020DC
:103BC8000E1C0020A02C0020094A0A4B117831B1A4
:103BD800997801F00F01814201D0002111709A7883
:103BE80060F303029A705A7842F080025A70704764
:103BF8009A1A00204B1A00202DE9FF411E466D4BF2
:103C0800DDF82880154604461A780F4600236A49CD
:103C180011F8231011F0010F05D001219940C1F1CD
:103C28000F0101EA02020133042BF0D1634B1A7031
:103C3800002C6FD014F0010F0AD0FF23012100934C
:103C4800FF3B0193029352200A460B460DF078FF82
:103C580014F0020F0AD0FF2301210093FF3B0193C8
:103C6800029353200A460B460DF06AFF14F0040F26
:103C78000AD0FF2301210093FF3B019302935420B4
:103C88000A460B460DF05CFF14F0080F0AD0FF231C
:103C980001210093FF3B0193029355200A460B46EE
:103CA8000DF04EFF14F0100F0AD0FF2301210093EE
:103CB800FF3B0193029356200A460B460DF040FF46
:103CC80014F0200F0AD0FF2301210093FF3B01933A
:103CD800029357200A460B460DF032FF14F0400FAE
:103CE8000AD0FF2301210093FF3B01930293582040
:103CF8000A460B460DF024FF14F0800F0AD0FF236C
:103D080001210093FF3B0193029359200A460B4679
:103D18000DF016FFCFB100243046214620F0C9FD32
:103D280060B1FF230093FF3B0193631C1BB2012189
:103D380002935A200A460B460DF002FF21463046F0
:103D4800013420F0ABFD402CE6D1BDB10024404643
:103D5800214620F0AEFD70B1012D0CD10423009353
:103D6800DB180193631C1BB20293742029460322BB
:103D78002B460DF0E5FE0134702CE8D10F481049B0
:103D8800104AFFF7D1FE104B00221A700132009240
:103D9800063201920832029209490A4A074809F094
:103DA800BBFE0A4B3C2251201A7004B0BDE8F0411A
:103DB8000EF090BA0C1A00201E1A00207C1D00205C
:103DC800651E0020581E0020411D00202E1A0020CC
:103DD80037B5FFF76BF904460E4820F03DFDD0F1EA
:103DE800010538BF00250C480E211BF0C9FC10B195
:103DF80014F4807F03D124B95DB1224602E0012288
:103E080000E00022044B204600932946014BFFF7AF
:103E1800F3FE3EBDEC1A0020FC190020054B03EB15
:103E2800D00393F8903100F0070053FA00F000F047
:103E380001007047A02C002010B50F4B04461B78DA
:103E480013F0010315D0FFF701FD28B90B4B1B191F
:103E580093F88030462B0DD10EF050F918B9204652
:103E6800FFF7DCFF30B10648214620F00CFD0120A9
:103E780010BD184610BD00BF041C0020A02C002057
:103E8800EC1A0020024B1878003818BF0120704740
:103E98002E1A002010B5034C04EB83035870997058
:103EA800DA7010BD1E1A002010B500240948002140
:103EB80000190E220E34FCF76DFAB4F5E07FF5D147
:103EC800054A00231370054A002199520233AA2B90
:103ED800F9D110BDE0150020DB150020DA1E002006
:103EE8007FB5474B04461B780E46AA2B78D0454829
:103EF800214620F0DEFC0546002871D12046FFF758
:103F08009BFF00286DD14048214620F0D2FC50B9D3
:103F18003E48214620F0CDFC054620B92046FFF753
:103F2800D7FA00285DD13A4B1B7823B9394B1B7857
:103F380013F0010F09D1384BDB7803F02003DBB213
:103F48001BB9364B032283F84020012E05D82E4892
:103F5800214620F0AEFC40B142E0022E07D12B48AA
:103F6800214620F0A6FC10B13AE0274800E0274897
:103F7800214620F088FC2A48214620F08FFC022E9A
:103F880015D10125294603222B4600964A20661999
:103F9800019502960DF0D4FD2046FEF7E9F80023BE
:103FA8000246314618200093FEF7A8FB19E0012EBF
:103FB80009D102230093631C029301961220314613
:103FC8000322334609E07EB90121022300936318D6
:103FD80002930191112003220B460DF0B1FD03E07D
:103FE8000025284604B070BD2046FEF7C1F80246F9
:103FF80001200023211800930125FEF77FFBF0E73D
:10400800E71B00204E1A00200E1A0020661C002014
:104018000C1A0020D51E0020783A0020591A0020DA
:10402800161C00202DE9FF4704460D467548214619
:1040380020F03FFC8146002840F0DF80214671488F
:1040480020F021FC7048214620F028FC6F4E0DBB63
:1040580001274FF00208E31902934246032039462C
:104068003B46CDF8008001970DF06AFD327862B1C9
:104078000EF044F8024630B1337840461E330093C0
:1040880021462A4604E0009000E00092404621467E
:104098003B4628E0012D2BD15D4B04F5E240413031
:1040A8001F5D0DF0CFFC07F00F07874209DA631C8C
:1040B800022202930E2029462B46009201950DF00C
:1040C8003FFD327892B10EF019F8024638B14F4BE5
:1040D8000D201B7821461E330093002202E0009039
:1040E8000D2021460123FEF709FB5EE00092F7E769
:1040F800022D0BD101230193E318029314204946A2
:104108002A464B4600950DF01BFD4EE0032D4CD181
:1041180001272A464FF0020804EB070A4D203946CA
:104128003B46CDF800800197CDF808A00DF008FDBA
:1041380035783DB30DF0E2FF024630B133784046A2
:104148001E33009321464A4602E00090214640462D
:104158003B46FEF7D3FA0DF0D1FF671C054648B180
:104168002046FEF705F8337802461E3300931A20DE
:1041780039462CE02046FDF7FBFF009502463946FC
:104188001A202DE021462A463B4640460095FEF778
:10419800B5FA2046FDF7ECFF514602462B461A2099
:1041A8000095FEF7ABFA384628E03578EDB10DF00A
:1041B800A5FF04F11C06054658B12046FDF7D8FFB7
:1041C800124B02461B7830461E330093611C0023B5
:1041D80007E02046FDF7CCFF009502463046611CFB
:1041E8002B46FEF78BFA012008E02046FDF7C0FFBA
:1041F8000095024604F11C00F1E7002004B0BDE878
:10420800F08700BF0E1C0020161C00206E1C00202A
:10421800F41A0020064B1B1893F84001492804D0D3
:10422800452814BF0320022070470120704700BFB3
:10423800A02C00202DE9F041244F00243C70244894
:10424800214620F036FBE5B2224B002837D01E5D10
:104258003B789E4200D303B93E70002E30D13146E0
:104268001C484022FCF796F81B4B1C4803EBD5036F
:1042780093F8888104F0070348FA03F8214608F008
:10428800010820F016FB68B9B8F1000F02D02846E3
:10429800022101E028463146FFF7C4FE28460EF009
:1042A80019F80DE0B8F1000F0AD12846FFF7B2FF60
:1042B8000B4BDB7803F02003DBB20BB9094B185525
:1042C8000134402CBBD1BDE8F08100BF6E1C00203A
:1042D8003B1A0020261C0020A02C00200E1C0020C9
:1042E800783A0020591A00202DE9F04F914B8BB0F5
:1042F8001B7813F0010F06D08F4B1A786FF38612D4
:104308001A7001F09EBA8D498D4A0B7810788D4D40
:10431800984218BF8C49137018BF0B706B7803F064
:104328000803DBB24BB143F6CF200DF08BFB864B75
:1043380018702B886FF3CB232B80844B1B78AA2B08
:1043480008D18349AA3B0B702B8843F080032B804C
:1043580000F0F0BE6A787B4B02F01002D2B27D4CBE
:10436800A2B11A886FF30C321A807B4B1B7823B9E1
:104378007A4B1B7813F0010F08D1E37803F0200380
:10438800DBB21BB9764B032283F840202368754FB4
:104398006FF3186323603A7802F00202D2B232B99E
:1043A8006B494A781AB16B4A43F080731360E67818
:1043B80016F0010648D05D20FFF7D2F900285AD13F
:1043C8006B78DFF8808103F00203DBB22BBB5D3032
:1043D800FFF77EF8064600BBB8F80030012143F429
:1043E8000073A8F80030042303220093019302907D
:1043F8000B460D200DF0A4FB45200DF06BFF314658
:10440800012233460D200096FEF778F9092031463F
:10441800324601230096FEF771F96B7803F0020328
:10442800DBB243B34C4B1B7823B94C4B1B7813F0CE
:10443800010F20D1E37803F02003DBB2DBB9484B4E
:10444800032283F8402016E06B7803F00203DBB206
:104458006BB13146324601230A200096FEF74EF929
:104468008D203146012233460096FEF747F92B8806
:104478006FF349232B802368354A6FF35963236010
:1044880093787BB1D37823B93B7813F00C0F05D11F
:1044980008E03B7803F00C03042B03D0236843F0B7
:1044A80000732360E17801F00201C9B200295BD0F2
:1044B8005E20FFF755F9002865D16B78214F03F08E
:1044C8000403DBB2EBB95E30FFF702F80646C0B969
:1044D8003B88012143F480633B800423009301332C
:1044E8000322019302900B4617200DF029FB45206B
:1044F8000DF0F0FE0D203146012233460096FEF7FE
:10450800FDF86B7803F00403DBB2002B3BD0124BB1
:104518001B7823B9114B1B7813F0010F33D1E378C3
:1045280003F02003DBB273BB0D4B032283F840205A
:1045380029E000BF7D1D0020043C0020F11B002065
:10454800F21B0020041C00206F1C0020E71B002029
:1045580060130020783A00200C1A0020D51E002095
:10456800591A00209E2C00206B7803F00403DBB25C
:104578002BB18D2001220B460091FEF7BFF82B8846
:104588006FF38A232B8023684FF05F0B6FF3DF7381
:104598002360002696E00698F9B21BF02FF9002850
:1045A80075D04FF436637343342202FB0733A749AF
:1045B800A8F15E0ACB1803F108021B7A5FFA8AFA9F
:1045C80013F001034DD02368404643F000432360B5
:1045D8000592FFF7C5F8059A002864D1937813F07F
:1045E800040F20D14046FEF773FF059A8146D0B9E3
:1045F8009378012143F00403937004230093DB189C
:104608000322019332200B46CDF808A00DF098FA4A
:104618004A200DF05FFE0C20514601224B46CDF892
:104628000090FEF76BF84FF436637343342202FBB5
:104638000733864AD3189B7A13F0040F33D0844B80
:104648001B7823B9834B1B7813F0010F2BD1E37828
:1046580003F02003DBB233BB7F4B032283F84020F7
:1046680021E0927812F0040F05D08C2051460122E7
:104678000093FEF743F84FF436637343342202FB8A
:1046880007337249CB189A7A6FF382020AE04FF423
:1046980036637343342202FB07336C4AD3189A7A81
:1046A80060F382029A72013708F10108382F5FFA25
:1046B80088F87FF470AF01360BF1380B022E5FFAE1
:1046C8008BFB04D0F3B20693D846002763E7236830
:1046D800624923F080636FF39E7323600B79002B8C
:1046E80000F0EC835E4ADFF87CB106924FF0CF0809
:1046F80000271BF8011F3E460137002952D02368C6
:1047080008F1710A43F080635FFA8AFA2360504621
:10471800FFF726F800285CD118237343DFF8489187
:1047280019F8032012F0100F23D150460593FEF715
:10473800CFFE059B8246E0B919F80320012142F01B
:10474800100209F8032004230093023301933BB2BB
:10475800032202930F200B460DF0F2F945200DF0CD
:10476800B9FD0D20514601225346CDF800A0FDF7B2
:10477800C5FF1823734319F8033013F0100F28D01E
:10478800334B1B7823B9334B1B7813F0010F20D11F
:10479800E37803F02003DBB2DBB92F4B032283F865
:1047A800402016E018237343DFF8BC9019F8033053
:1047B80013F0100F05D08D2001220B460091FDF754
:1047C8009DFF1823734319F803206FF3041209F8A7
:1047D8000320069A12F8011F0692002946D0236882
:1047E800404643F080432360FEF7BAFF002854D1C7
:1047F8004FF0180909FB06F9DFF86CA01AF8093020
:1048080013F0200F49D14046FEF762FE0646002805
:1048180043D11AF80930012143F020030AF809307E
:1048280004230093033301933BB2032202934B20EA
:104838000B460DF085F950200DF04CFD192031463E
:10484800012233460096FDF759FF26E0043E00207A
:104858000C1A0020D51E0020591A002060130020D1
:10486800103B0020353B00203C3B002018237343BD
:10487800DFF8089319F8033013F0200F05D09920BA
:1048880001220B460091FDF739FF18235E4319F802
:1048980006306FF3451309F8063008F10108042FB4
:1048A8005FFA88F87FF425AFAD4ADFF8D4B20692F4
:1048B8004FF05008043F1BF8011F3E4601370029FE
:1048C80052D02368A8F16E0A43F080635FFA8AFA2F
:1048D80023605046FEF744FF00285CD1DFF8A4921D
:1048E80006EB061319F8032012F0400F23D15046A7
:1048F8000593FEF7EDFD059B8246E0B919F8032004
:10490800012142F0400209F80320042300930233F6
:1049180001933BB20322029369200B460DF010F974
:1049280045200DF0D7FC0D20514601225346CDF805
:1049380000A0FDF7E3FE06EB061319F8033013F0A9
:10494800400F28D0874B1B7823B9874B1B7813F06F
:10495800010F20D1E37803F02003DBB2DBB9834BEE
:10496800032283F8402016E0DFF8189206EB0613BE
:1049780019F8033013F0400F05D08D2001220B46A3
:104988000091FDF7BBFE06EB061319F803206FF341
:10499800861209F80320069A12F8011F06920029C8
:1049A80033D02368404643F080432360FEF7D8FEA7
:1049B800002841D1DFF8CCA106EB06191AF8093016
:1049C80013F0200F38D14046FEF782FD064698BB0B
:1049D8001AF80930012143F020030AF809300423AA
:1049E8000093033301933BB20322029310200B463A
:1049F8000DF0A6F850200DF06DFC1920314601226B
:104A080033460096FDF77AFE16E0DFF8789106EB5C
:104A1800061319F8033013F0200F05D0992001224E
:104A28000B460091FDF76AFE06EB061619F80630EC
:104A38006FF3451309F8063008F10108022F5FFAF1
:104A480088F87FF438AF4A4B1978002946D0236894
:104A5800DE2043F080632360FEF782FE00284CD1FD
:104A6800444B1A78984612F0400F20D1DE30FEF7FA
:104A78002FFD0746D8B998F80030012643F04003C7
:104A880088F800300423009302333146032201934F
:104A98006720334602960DF053F845200DF01AFCB6
:104AA8000D20394632463B460097FDF727FE98F819
:104AB800003013F0400F20D02A4B1B7823B92A4B23
:104AC8001B7813F0010F18D1E37803F02003DBB251
:104AD8009BB9264B032283F840200EE0254E3378FD
:104AE80013F0400F05D08D2001220B460091FDF7F1
:104AF80005FE33786FF3861333701F4B197800293E
:104B080042D02368572043F080432360FEF728FEF5
:104B1800002848D1174E337813F0200F43D157306F
:104B2800FEF7D6FC074600283DD13378032243F030
:104B38002003337004230126009303333146019385
:104B48001F20334602960CF0FBFF50200DF0C2FBED
:104B58001920394632463B460097FDF7CFFD22E043
:104B68007B3A00200C1A0020D51E0020591A00207C
:104B7800A93A0020BC3A0020AE3A00203C3B002075
:104B8800003B0020DF3A0020864E337813F0200FD8
:104B980005D0992001220B460091FDF7AFFD33782F
:104BA8006FF3451333704FF000084FF05B094FF077
:104BB800D70A46467C4B08F10108F15C7B4F002977
:104BC80049D02368484643F080632360FEF7C8FD58
:104BD800002852D113237343FA5C12F0200F22D11C
:104BE80048460593FEF774FC059B8346D8B9FA5CE2
:104BF800012142F02002FA54042300930233019366
:104C08000FFA88F30322029320200B460CF098FF3A
:104C180045200DF05FFB0D20594601225B46CDF87B
:104C280000B0FDF76BFD13237343FB5C13F0200FFB
:104C380023D05F4B1B7823B95E4B1B7813F0010F11
:104C48001BD1E37803F02003DBB2B3B95A4B03223C
:104C580083F8402011E013237343FB5C13F0200F0B
:104C680005D08D2001220B460091FDF747FD132347
:104C78007343FA5C6FF34512FA54504BF15C002908
:104C880033D02368504643F080432360FEF768FD25
:104C980000283ED1132303FB06735A7812F0200F25
:104CA80037D150460593FEF713FC059B834680BB1E
:104CB8005A78012142F020025A70042300930333EA
:104CC80001930FFA88F3032202934C200B460CF051
:104CD80037FF50200DF0FEFA1920594601225B4695
:104CE800CDF800B0FDF70AFD13E0132303FB0673AC
:104CF8005B7813F0200F05D0992001220B46009114
:104D0800FDF7FCFC132303FB06735A786FF3451277
:104D18005A702B4B1322F35C002B53D002FB06F383
:104D280017F803B0CBF3801BBBF1000F22D143F679
:104D3800DE2005930CF086FE059BD8B1FA5C0121B4
:104D480042F04002FA5404230093DB1801930FFA4F
:104D580088F3032202932F200B460CF0F1FE472024
:104D68000DF0B8FA0920414601225B46CDF800B0A3
:104D7800FDF7C4FC13237343FB5C13F0400F32D0E0
:104D88000B4B1B7823B90B4B1B7813F0010F2AD15F
:104D9800E37803F02003DBB22BBB074B032283F835
:104DA800402020E0BC3A00200E3B0020833A00203F
:104DB8000C1A0020D51E0020591A0020033B0020A1
:104DC800B03A00207243BA5C12F0400F05D0892037
:104DD800414601220093FDF791FC13237343FA5CCB
:104DE8006FF38612FA5401360AF1010A09F1010932
:104DF800022E5FFA8AFA5FFA89F97FF4DBAEDFF8F0
:104E080048A24827023E1AF8011FB0460136002979
:104E180037D02368384643F080432360FEF7A0FC70
:104E2800002847D14FF01E0909FB08F9DFF81CB22A
:104E38001BF8093013F0200F3CD13846FEF748FB29
:104E48008046002836D11BF80930012143F02003A1
:104E58000BF80930042300930333019333B2032280
:104E6800029313200B460CF06BFE50200DF032FA23
:104E78001920414601224346CDF80080FDF73EFC4B
:104E880018E01E2303FB08F3DFF8C09119F803307C
:104E980013F0200F05D0992001220B460091FDF751
:104EA8002DFC1E2303FB08F819F808306FF345138F
:104EB80009F808300137042EFFB2A4D1A67806F00D
:104EC8000806F6B2002E40F03581594A06925FFA7C
:104ED80086F8B8F1000F0CBF4023702347F61B413A
:104EE8000993089149F61E59002447464FF4E07A81
:104EF8000AFB06FA4E4A2146524410465FFA84F8E5
:104F080007921FF0D6FC48B949480AF1700A504484
:104F180021461FF0CEFC002800F0F980444B4FF4E6
:104F2800E07A0AFB063A0AF1E00A504621461FF0E9
:104F3800C0FC002840F0EB80504621461FF0A3FC3F
:104F4800DFF80CA10FB9484600E008980CF07AFD8C
:104F58008AF800009AF80000DFF8F4B0002800F0A2
:104F6800D6800138C0B28BF800000BF075FE00281F
:104F780040F0CD809BF8000000F56A507C300CF0C2
:104F880061FD2C49C0B2087027B92B4B4B4413F86C
:104F98005EAC03E0069A131993F850A100EA0A0AD6
:104FA800BAF1000F00F0B380079821461FF081FC8A
:104FB800DFF890B000B31E4B4FF4E07000FB0630F2
:104FC800214670301FF075FCB0B91C49012F0B78D1
:104FD8004AEA030A8BF800A056D13823B8FBF3F24B
:104FE80003FB12834FF436614A43DBB2342101FBE1
:104FF8000323134AD31841E00D4B4FF4E07000FB34
:105008000630214670301FF054FC38B1079821460D
:105018001FF04FFC10B909490B7804E0074A1378D0
:105028001AEA030F16D023EA0A0A8BF800A02BE02D
:1050380018290020161E0020A090FF1F0C1A00201F
:10504800043E00207C1D0020DA3A00201F3C00208E
:10505800EB1A00204AEA030A012F8BF800A013D1AB
:105068003823B8FBF3F203FB12834FF436614A434B
:10507800DBB2342101FB03238D49CB1893F8302090
:1050880042F0200283F830208A488B498B4AFEF789
:105098004BFD894B1B781BB1FEF708F8002836D169
:1050A8008548874912F0FCFE68B10DF027F870BBFF
:1050B800834808F09DFD50BB0123814881497E4A01
:1050C8000093FEF707FD002300937F4A0133019305
:1050D8001378784802937849784A7A4B08F01CFD8F
:1050E800012F14D13823B8FBF3F203FB12884FF4D5
:1050F80036635A435FFA88F8342303FB08236C4964
:10510800CB1893F8312042F0010283F831200134A2
:10511800089A0999E3B205328B4209F1010908920C
:10512800FFF4E4AE069A013602F5E072022E06920A
:105138007FF4CDAE654E73786FF3C71373702B7819
:1051480003F08002D2B2002A00F0E48060490C78B3
:10515800002C40F0DF8003F02403042B0BD1FEF772
:1051680013FCFF230093402021460122234601948B
:1051780002940CF0E5FC2B8800246FF3C7136FF33F
:10518800820364F3451364F3410364F30003514A53
:1051980064F3492364F38A2314702B804E4B1A78E6
:1051A80042F0C0021A705A7864F3C3025A70FEF7CC
:1051B800CBFC4A481FF022FB49481FF01FFB494817
:1051C8001FF01CFB412248482146FBF7E3F8474BF8
:1051D8001A7802F0DF0264F304121A701A7E02F0E1
:1051E800DF0264F304121A7693F8302002F0DF022B
:1051F80064F3041283F8302093F8482002F0DF02A9
:1052080064F3041283F84820394B1A7802F0DF025D
:1052180064F386121A705A7C02F0DF0264F3861275
:105228005A74344B1A7864F345121A709A7F64F3EF
:1052380045129A7793F83C2064F3451283F83C2092
:1052480093F85A2064F3451283F85A202A4B1A78A7
:1052580002F0DF0264F386121A70284B5A7864F35E
:1052680045125A701A7802F0BF0264F345121A7098
:105278001A7D64F345121A75DA7C02F0BF0264F3F2
:105288004512DA7411E04FF436626243342101FBAF
:1052980003221B49013352189178382B6FF382018E
:1052A8009170F0D10134022C2CD00023EBE700BF21
:1052B800043E00207C1D0020651E0020581E002092
:1052C800161A0020411D0020161E00204B1A00202F
:1052D80060130020E81B0020043C0020661C00200E
:1052E8000E1A00203B1A0020591A00203C3B0020CF
:1052F800DF3A00201F3C0020BC3A0020833A0020FF
:105308000C3E0020042272480021FBF743F8714B41
:1053180000221A70704C2378002B48D129786F4AE4
:1053280001F00201C9B2D9B16D481188477863F319
:105338004D3163F3C30741F0800147701180CA20E3
:1053480020F0A4F8C62020F0A1F820F0EDF8654A76
:1053580013780BB90DF04AF8FEF79CF8FEF7A4FD98
:10536800614A2B8811786FF341036FF300016FF3E3
:10537800000311705D48002140222B80FBF70AF8DA
:105388005B481FF03BFA5B481FF038FA5A481FF099
:1053980035FA5A481FF036FA04224D480021FAF728
:1053A800F9FF4C4A00231370554A13706AE02F78AE
:1053B80007F00203DBB293B917F001070FD14C488D
:1053C8001FF01CFA2378F8B23B4113F0010F03D009
:1053D800FEF7F6F90CF088FE0137042FF2D12B788E
:1053E8003E4F13F0010F25D0FEF7F2FC3B8843F047
:1053F80002033B80FEF786FA364B93F80080B8F13B
:10540800000F14D1CA2020F041F8CD2020F03EF83A
:105418003B883C4868F300033B80334B1A7842F0E2
:1054280001021A701FF0EAF9FEF734F802E00120D1
:10543800FEF7CAFB2B7803F00202D2B212B3304A4D
:1054480012782AB113F0010F02D10220FEF7BCFB3B
:10545800FEF7F0FE2C4927481FF0EEF925492648AB
:105468001FF0D4F9FEF78AFB224928481FF0CEF92D
:10547800274926481FF0D5F9FEF71AFB1F481D4992
:105488001FF0E5F9204923481FF0C0F915490B78AA
:105498000BB9FEF79BFA737803F08003DBB2002B9D
:1054A80040D12B7803F02403042B06D143F6EC20DB
:1054B8000CF0C8FA08B1062032E0FEF7E3FC08B1A8
:1054C80005202DE00DF07CF830B3032028E000BF64
:1054D8002F1A00200A1A00200C1A0020041C002091
:1054E800043C0020601300200D1A0020261C002018
:1054F800E5310020DF1B00203B1A00201E1C002085
:105508006E1C0020EC1A00204E1A00200E1C0020F1
:105518009B1A0020331A002001F060F810B1042013
:10552800FEF752FB694B1B781BB173786FF3C713F7
:105538007370674A137813B1664B1B78CBB12B781D
:10554800654E03F04403402B13D10021BF33009371
:105558003F200B460222019102910CF0F1FA3388A8
:1055680043F6CE2043F0040333800CF06BFA5B4B18
:10557800187057495A4E0B789BB1564B197881B918
:105588002A78554B02F04002D2B252B11A8861F320
:1055980082021A80337823B943F6CE200CF052FAEF
:1055A80030702A78DFF8308102F00400C0B24D4B29
:1055B80000287AD002F02000C0B2484F90B11A7883
:1055C800002042F0C0021A70FDF784FE3B78002BE1
:1055D80071D1B8F8002063F3820263F34512A8F88A
:1055E800002068E0D20052B219789211D2B241F08C
:1055F800C00112F0010F197003D0C9B260F3C711CE
:10560800197012F0020F03D01A786FF386121A700D
:105618001B78344A03F04003DBB24BB9537843F0AC
:105628000803537023781BB12B8843F400532B8055
:105638000120FDF74FFE43F6CD200CF003FAC0B26F
:105648000128307002D1264B02221A703C78002CB7
:1056580031D1FEF799F9FF2301220093402021461A
:105668002346019402940CF06BFA2B8843F6CD2064
:1056780043F020032B800CF0E5F9184B1A4A1870F8
:10568800144B14701A780AB1013A1A70197891B942
:105698000F4A13787BB1FF230093412002220B4667
:1056A800019102910CF04CFA05E01A7842F0C00220
:1056B8001A70FDF70FFE0CF033FF0C481FF0CCF802
:1056C8000B4BB8B91A7860F3820216E042580020F2
:1056D800F11B00206F1C0020041C0020E81B002088
:1056E800581A0020043C002060130020A31A002050
:1056F8000D1A00201A7842F004021A706A7852488B
:1057080012F001011A780CBF61F3410242F0020263
:105718001A704E491FF09BF84D494B481FF081F80D
:1057280049484C491FF07DF83378012B40F08980B7
:105738002B8800246FF349236FF38A232B80464B71
:1057480041221C7021464548FAF724FE44481FF0C0
:1057580055F8FEF7F9F93E481FF050F83D481FF09C
:105768004DF8404B1A7802F0DF0264F304121A7005
:105778001A7E02F0DF0264F304121A7693F83020DE
:1057880002F0DF0264F3041283F8302093F8482013
:1057980002F0DF0264F3041283F84820324B1A78CF
:1057A80002F0DF0264F386121A705A7C02F0DF02FC
:1057B80064F386125A742D4B1A7864F345121A70E2
:1057C8009A7F64F345129A7793F83C2064F3451264
:1057D80083F83C2093F85A2064F3451283F85A2042
:1057E800234B1A7802F0DF0264F386121A70214BF9
:1057F8005A7864F345125A701A7802F0BF0264F3BB
:1058080045121A701A7D64F345121A75DA7C02F093
:10581800BF0264F34512DA7411E04FF43662624352
:10582800342101FB03221449013352189178382B93
:105838006FF382019170F0D10134022C01D0002362
:10584800EBE70BB0BDE8F08F6A3600200E1C002095
:105858000E1A0020661C0020581A0020591A002031
:105868003B1A00203C3B0020DF3A00201F3C002070
:10587800BC3A0020833A00200C3E00202DE9FF416D
:1058880004460D460CF076FEA04B1A1992F880706B
:105898009F4A98461278AA2A0AD1A7F14F03DAB28A
:1058A8000B2A00F2AD819B4A5BB29A4040F1A88175
:1058B800994B0C2202FB04335A7A0833AA42C0F0EF
:1058C8009F81FF2A00F09C81FF229A70934808EB81
:1058D800D403214693F888511EF0EBFF06460028B2
:1058E80040F08E8104F007031D41502F05F001059B
:1058F80000F0268114D8462F00F0F28009D8412FF5
:1059080000F09E80452F00F01B812D2F40F07681FE
:1059180034E0482F00F0C5804F2F40F06F810EE033
:10592800542F67D006D8522F00F08A80532F40F0AA
:1059380065811CE0A7F15903012B00F25F817848CB
:1059480021461EF0B6FF0646002840F059815A2F1E
:1059580001D1744802E0592F04D1734821461EF042
:1059680092FF54E121466F481EF08DFFF5E76F481E
:1059780021461EF09EFF002800F042816C48214617
:105988001EF097FF8046002840F03A81214668487B
:105998001EF079FF674821461EF080FF0227012686
:1059A80055B1A419142041463A464346009701963A
:1059B80002940CF0C5F82AE129463A46334604F128
:1059C80001080A2000970196CDF808800CF0B8F875
:1059D8002046FCF7CDFB414602462B461320009596
:1059E800FCF78CFE384629462A4633460095FCF7D4
:1059F80085FE0CE14E4821461EF05BFF0746002855
:105A080040F005810126022231463346A5193E2081
:105A18000092019602950CF093F82046FCF7A8FB3B
:105A2800294602463B4614200097FCF767FE2146AC
:105A38003F481EF028FF21463E481EF02FFFE6E0B3
:105A48003A4821461EF035FF0646002800F0DF8060
:105A5800374821461EF02DFF064628B92046FDF797
:105A680037FD002840F0D380002D40F08E8020467E
:105A7800FEF7E2F9002840F0C5802046FEF7CAFB91
:105A88002D4BDB7803F02003DBB20BB92B4B1855F9
:105A9800412F00F08880522F40F0B080204601212D
:105AA80083E0234821461EF004FF28B92046FDF76D
:105AB8000FFD002840F0A480002D66D12046FEF797
:105AC800BBF9002840F09E801B4BDB7803F02003D5
:105AD800DBB2002B67D1194B032283F8402062E028
:105AE800134821461EF0E5FE064628B92046FDF774
:105AF800EFFC002840F08B802046FEF79DF9002837
:105B08007ED1002D41D1204603214EE0A02C00205B
:105B1800E71B002000003080742E00204E1A002061
:105B2800F82900201829002088290020DF1B0020E0
:105B38000E1C0020161C0020783A0020591A00205C
:105B4800354821461EF0B5FE064600285FD020469F
:105B5800FDF790FE20B1214630481EF094FE4FE03C
:105B6800502F28D12E4B1B782BBB2046FDF76EFEFD
:105B780008BB2C4821461EF09CFE064620B920464C
:105B8800FDF7A6FC002842D115B1204602210CE001
:105B98002046FEF73FFB244BDB7803F02003DBB203
:105BA8000BB9224B185520460021FEF73BFA061E7A
:105BB80018BF01262BE02046FDF748FE0546F8B938
:105BC8001B4821461EF075FE0646D8B92046FDF74B
:105BD8007FFC0746D8B9164821461EF054FE154AE0
:105BE800135D8BB910494E7806F02006F6B26EB9EF
:105BF80008EB040393F80031135508E0012606E08A
:105C0800002604E02E4602E03E4600E01E463046EE
:105C180004B0BDE8F08100BFDF1B0020EC1A0020B3
:105C28006E1C00200E1C0020783A0020591A002013
:105C38003B1A0020261C0020032210B505490648FF
:105C4800FAF77EFE054806490222BDE81040FAF739
:105C580077BE00BF7626002004020020090200203B
:105C68007426002070B5844C237813F0010F0AD0F5
:105C78000CF04CFA38B10020804902F093FE804BBA
:105C88008048197849E0804D2B78002B4AD00CF0D9
:105C980043FA002846D07D4B1B7873B97C4B5B7860
:105CA80013F0010F09D00CF029FA30B9237803F06A
:105CB8002403042B01D10330BEE0764C207870B168
:105CC8000020754902F06EFE21780122734802F027
:105CD8008FFE00201021621C07F0D0FA02E0704904
:105CE80002F060FE6F4C684807F01CFB2378002B1D
:105CF80000F018810CF00AFA002800F013816A49B4
:105D08006A481022FAF71CFE68485B21FAF7C0FBC4
:105D1800002800F00781217801308322BDE8704017
:105D280002F066BE624C237803F00503012B5DD1B7
:105D38000020604902F036FE202110225E48FAF762
:105D480029FB601D5D490322FAF7A4FD40BBE01C56
:105D58005B490222FAF79EFD30B95A48FAF76AFD04
:105D68005849024654480BE0E01C57490222FAF70A
:105D780091FD40B95548FAF75DFD544902464E4831
:105D8800FAF7DEFD0EE0E01C51490222FAF782FD27
:105D980030B95048FAF74EFD4E4902464648EFE7FB
:105DA800FFF74AFF6278303AD3B2092B00F2BA8083
:105DB8003F4B9B78303BDBB2092B00F2B3800A21C2
:105DC80001FB0231C9B2002900F0AC80374BFF2239
:105DD8000C291A7740F2A68010295A7740F2A2803F
:105DE80013299A7740F29E80DA7770BD3A4C23786F
:105DF80003F00203DBB213B1002038498EE0234ED2
:105E08003378EBB9224B5B7813F0010F18D00CF004
:105E180075F9A8B932481EF01FFD60B12268314BF0
:105E280002EA03033BB918F005FE20B9E37803F052
:105E38004003DBB223B10020BDE870400AF0E4B9AA
:105E4800337863B90CF05AF948B1274B1B7803F043
:105E58000603042B03D02B780BB90120ECE7FEF7DF
:105E680011F810B10020214958E0214B1D78002D70
:105E780042D0204952E000BF041C002031F902083A
:105E88000A1A0020000200200C1A0020141E00200C
:105E9800D51E00205E1D002044CE02080502002009
:105EA80002CE02086E1C002023CE0208F401002056
:105EB800712600204BD30208040200209C550308D9
:105EC800A0550308AED30208A35503088DD30208D2
:105ED800A65503086CD30208783A0020A2E202080B
:105EE800A31A00203000000F0D1A0020D4E0020889
:105EF8006513002065CE02080B4802F002FD0A482F
:105F080002F0F6FC094802F0F3FC1DF051F9E378C1
:105F180003F02003DBB22BB105492846BDE87040E9
:105F280002F040BD70BD00BF681E0020881D002023
:105F38005DCD0208054B1B78D8019B015BB2DB11D4
:105F480040B243EAE070C0B2704700BF041C0020B2
:105F580070B50E4686B041000122054601F5E9718B
:105F680005A80BF080FD0021012E8DF815104FF0CB
:105F7800FF0205F1010305D1009201910293092066
:105F8800FB3A04E00092019102931E2004220B4682
:105F98000BF0D6FD05A83D49FAF700FB50B105A85E
:105FA8003B49FAF7FBFA28B105A83A49FAF7F6FA95
:105FB800002867D105A83749FAF7F0FA364B0446A6
:105FC800F8B95A78214642F010025A70FF2302228B
:105FD80000930190FE3B02903D200BF0B1FD4D2057
:105FE8000CF078F9691C0122234612200094FCF772
:105FF80085FB12202146224601230094FCF77EFBF4
:1060080003E05A786FF304125A700024E0B2552165
:1060180015F0E8FE38B12846214616F084F810B18C
:10602800204616F06FF80134082CEFD13EBB1B4810
:106038001B491C4AFDF778FD19481B4911F030FF30
:1060480068B10CF05BF850B9174807F0D1FD30B9CA
:10605800012315481549124A0093FDF73BFD144BDF
:106068000F491D700023009305330193114B0D4A0E
:106078001B780A4802930D4B07F04EFD02E00E4BC9
:1060880000221A7005A806B070BD00BF2D5603087F
:10609800A955030839580308043C00207C1D00203A
:1060A800651E0020581E0020161A0020411D0020E1
:1060B800973C0020161E00202E1A002007B541002C
:1060C800012201A801F5E9710BF0CDFC002301A81C
:1060D80004498DF80530FAF761FAD0F1010038BFAC
:1060E80000200EBD2D56030807B54100012201A866
:1060F80001F5E9710BF0B7FC002301A804498DF8FC
:106108000530FAF74BFAD0F1010038BF00200EBD78
:10611800F657030870B5154B04461B1893F88050C2
:10612800B1B1134821461EF0C4FB88B91148214675
:106138001EF0A9FBA5F15903DBB2012B0CD94F2D99
:106148000AD0542D08D021460B481EF09CFB07E0CE
:10615800084821461EF0A2FB074821461EF09EFB78
:1061680004480649BDE870401EF050BBA02C002032
:106178004E1A0020A31A0020431A00201E1C0020DB
:10618800024B1878C0F38000704700BF0D1A00203A
:10619800024B1A8860F308221A807047041C0020FA
:1061A800034B5878C00140B2C011C0B2704700BF5D
:1061B800041C0020014B1878704700BF0C1A0020FF
:1061C80030B5457800230021C218917055FA03F1C3
:1061D80011F0010F08D0064959188C7C017804EA9F
:1061E8000101A14208BF91700133042BEBD130BDEE
:1061F8005E1D002046F6A93104220BF034BC0000D5
:1062080070B5104C0546112220460021FAF7C2F855
:10621800002004F8010C2A78103414F8011FC3B2C6
:1062280091420BD152B10849013301F8013B1122C7
:1062380046F6F953BDE8704002F000BB013004286F
:10624800EBD170BD5F1D00205E1D00201FB520B181
:10625800134B1A8842F480521A80124B00245A7841
:10626800214642F010025A70FF23022200933D207B
:10627800FE3B019402940BF063FC4D200CF02AF8CD
:1062880020210122234612200094FCF737FA12201D
:106298002146224601230094FCF730FA1FBD00BFB7
:1062A800041C0020043C00202DE9F3412D4C07225A
:1062B800E37849F6B44702FB003349F6D540DBB230
:1062C80018180BF0BFFB257964795FFA80F800266F
:1062D80048FA06F313F0010F3AD03946042201A810
:1062E8000BF0C1FB9DF804009DF805309DF80610E1
:1062F8009DF8072000282BD0002929D0002B27D073
:10630800002A25D0934204D19C4221D185421FD333
:106318000FE09A4210D99C421AD3944218D89C4252
:1063280001D994421AD39C4201D1854216D2944293
:106338000ED18D420CD811E09C4201D185420DD27C
:10634800944201D18D4209D99C4207D8944205D381
:1063580001360437082EBBD1002000E00120BDE83B
:10636800FC8100BFB055002010B5044649F60D5019
:1063780000EBD4000BF066FB04F00704C0B2204128
:1063880000F0010010BD70B5C30849F60D555D1940
:10639800044628460E460BF055FB04F00704C0B22D
:1063A800012126B9A14040EA0101C9B202E0A14099
:1063B80020EA01012846BDE870400BF039BB000017
:1063C800F0B57E4B8DB0DD78042200EBC505EDB24B
:1063D800E90001F5084104A801F59E710BF043FBA3
:1063E800774B784E1A78002304A9C95C312905D166
:1063F8003039994041EA0202D2B205E0302903D18E
:106408002F39994022EA01020133042BECD1327072
:106418006C486D496D4AFDF787FB6B4B1B7813B9C8
:106428006A4B1B78F3B16848694911F039FD68B1C6
:106438000BF064FE50B9664807F0DAFB30B9012367
:1064480063486449604A0093FDF744FB00230093C6
:1064580002330193FD3302935A485B495B4A5D4B13
:1064680007F05AFB05EB0511002401F50A413470C9
:1064780004A8FC3108220BF0F6FA2646E0B25421B3
:1064880015F0B0FC002838D004AB1B5D312B03D1CC
:10649800204615F03DFD38B104AB1B5D302B2CD1E7
:1064A800204615F035FD40B34EB9FF230093342044
:1064B800314604223346019602960BF041FB04AEA6
:1064C800305D2146303815F031FD335D0126312B22
:1064D8004FF0030306D10093A3191BB20196029350
:1064E800352005E00093631C1BB201960293362009
:1064F800002104220B460BF023FB0134082CBDD1EC
:10650800A90101F50E4104A8B43120220BF0ABFA21
:10651800083C04AD274615F8013BE6B20134302BA0
:1065280003D13046FFF720FF38B115F8013C312B75
:106538002CD13046FFF718FF40B34FB9FF23009323
:106548003420394604223B46019702970BF0F8FAAB
:1065580015F8011C30463039C9B2FFF714FF15F899
:10656800013C0021302B4FF0FF0305D1009323B2EB
:1065780001910293372004E0009323B20191029322
:10658800382004220B460BF0DBFA0127202CC2D15D
:10659800114D6B7803F00403DBB263B1203C204655
:1065A800FFF7E2FE38B90134E4B2202CF7D16B785A
:1065B80060F382036B700DB0F0BD00BFB0550020D2
:1065C8000C1A00207C1D0020651E0020581E00208B
:1065D800161A0020411D0020043C0020014B1878A9
:1065E800704700BF651300202DE9F04F4E4B002285
:1065F8001A704E4A85B01678002E40F091804C4BA8
:106608004FF4B468DA78997808FB02F24FF03C0846
:1066180008FB01285A78474F90441FFA88F8BA4671
:106628006CE03AF815303C24DAB2544304EB1324F6
:106638004C44A4B2042CEEB207D842F25A739845DF
:1066480003D904F51C546034A4B2444511D949F661
:10665800D4400BF0F7F9C8EB0403834209DC364B4E
:106668001A787B1993F83830934302D02E490123C6
:106678000B702F4AD378B34232D142F26073B4FB25
:10668800F3F203FB12439BB2434523D12B4B9B7878
:1066980013F0090F44D12A4B5B7803F08003DBB277
:1066A800002B3DD1274B5B7803F00203DBB2002BB4
:1066B80036D1254B1A781BEA020F11D1019900989F
:1066C80041EA02021A70FFF7EFFD48B90098FFF798
:1066D80077FE05E01C4B02991A7801EA02021A704B
:1066E800013509F5B469072D1FFA89F999D1039E77
:1066F80007370136042E0AF10E0A11D04FF0010BAC
:106708000BFA06FB5FFA8BF301936FEA0B03F2B205
:10671800DBB24FF00009009202934D46039680E7E2
:1067280005B0BDE8F08F00BF65130020751C002080
:10673800B0550020761C00200C1A0020783A002062
:10674800133C002062340020741C002073B50C46F2
:1067580001EBC001C9B2C90001F508410546042290
:1067680001A801F59E710BF07EF9104B002003EB98
:10677800C402121B521982F8380001AA125C312A8D
:106788000AD10121814003EBC402121B521992F86D
:106798003860314382F8381001300428EDD101A95E
:1067A800312230231EF08DF8C0B27CBD761C00204B
:1067B80000B501EBC001C9B2890189B001F50E41EC
:1067C800B431202268460BF04EF920206946312268
:1067D80030231EF076F8C0B209B000BD07B501EB52
:1067E800C001C9B201EB011101F50A41FC310822CF
:1067F80068460BF038F908206946312230231EF02C
:1068080060F8C0B20EBD00002DE9F84300263446FA
:106818002BE021462846FFF799FF21468146284666
:10682800FFF7C6FF214640EA09092846FFF7D6FFC9
:106838005FFA89F949EA000010F0FF0F05D04046D9
:10684800394602220BF00FF903E04FF0FF33A8F8A6
:1068580000300135EDB20237072D08F10208D8D112
:106868000134E4B20E3E042C07D0054BC6F50847A8
:10687800C6EB0308CC370025CBE7BDE8F88300BF9B
:10688800761C002010B51FF083F84FF480301FF0FD
:106898009FF81FF0B7F90128044628D110201EF0F0
:1068A80099FF02201EF08AFF00201FF0D1F8002077
:1068B8001FF0E2F84FF480601FF0D4F84FF4404026
:1068C8001FF0E4F84FF480304FF4E0111FF09CF80B
:1068D80020461FF0A5F839201FF080F90028FAD0CB
:1068E80002201FF0A3F81FF0ABF80828FBD17C208A
:1068F80001211FF03DF946F6012001211FF038F96A
:106908000C4801211FF040F90B4801211FF03CF908
:10691800042001211FF038F97E201FF05FF938B1FB
:106928001FF086F9054B04211A7861F344021A70A6
:1069380010BD00BF03400600200808182558002095
:1069480010B50C46014620B110220C48F9F7F8FFA3
:1069580004E00A4820211022F9F71CFD34B1084848
:1069680021461022BDE81040F9F7EABF044820216B
:106978001022BDE81040F9F70DBD00BFF40100205A
:106988000402002010B5FF2B1446029A03D04218C7
:1069980002F8013C08E06FF07F439A4204D01314D8
:1069A800437013128370C2701BF0F4FA02E07F2068
:1069B8001FF05AFC1BF0DAFA0028F8D1ACB10B48EA
:1069C80090F82010163001F00F011BF0E3FA02E0F6
:1069D8007F201FF049FC1BF0C9FA0028F8D1044BAE
:1069E80093F8693013F0010FE9D110BD900C002025
:1069F8004057002010B50A4B002203EBC003013BAF
:106A08001046084951184C7813F8011F8C4205D1DB
:106A18000130C0B20C320828F3D1F73010BD00BFE6
:106A28003A630208742E002070B50D4C05460E46D8
:106A38004FF4007200212046F9F7ACFC2A46314693
:106A480004F50070F9F7FEFB642024F8035C1CF0E1
:106A580081FE0023A4F82D33024B64221A6070BD16
:106A6800A95800207C26002010B5054C002120469E
:106A78004FF40072F9F78EFC0023A4F82D3310BDF3
:106A8800A9580020164B2DE9F0415D8A0746284693
:106A9800FBF746F81349FBF74FF9134B134E1860F1
:106AA800D723B5FBF3F5EDB2822229460446F01947
:106AB80001F09EFF2846FBF737F801462046FAF713
:106AC8007DFF0B49FBF784F8FBF748FA0337BE193B
:106AD800C1B281223046BDE8F04101F089BF00BF54
:106AE800B031002000005743CC1C0020F4010020E6
:106AF800000020410000000070B54B4D2868FAF7EF
:106B08001BFC45A3D3E90023FAF7B6FAFAF702FF0C
:106B1800FAF712FC42A3D3E90023FAF761FC3EA37B
:106B2800D3E90023FAF786FDFAF7F4FEFAF704FC36
:106B3800FAF70EFAFAF7EEFE3C4906462860FBF72C
:106B4800EFF920B13046FBF709FAC4B25EE03046EF
:106B58003649FBF7F9F950B130463549FBF7E0F90A
:106B680028B13046FBF7FAF9C0B2441C4EE0304673
:106B78002F49FBF7E9F950B130462E49FBF7D0F918
:106B880028B13046FBF7EAF9C0B2841C3EE0304633
:106B98002849FBF7D9F950B130462749FBF7C0F926
:106BA80028B13046FBF7DAF9C0B2C41C2EE03046F3
:106BB8002149FBF7C9F950B130462049FBF7B0F934
:106BC80028B13046FBF7CAF9C0B2041D1EE03046B2
:106BD8001A49FBF7B9F950B130461949FBF7A0F942
:106BE80028B13046FBF7BAF9C0B2441D0EE0304672
:106BF8001349FBF7A9F948B130461249FBF790F958
:106C080020B13046FBF7AAF9C0B2841D0A202146FC
:106C1800BDE870400AF00CBF736891ED7CFF7F40BF
:106C28000000000080842E41D01C0020000010418C
:106C38000000F0410000484200008E420000B842C7
:106C48000000E0420000F2422DE9F04F9DB01BF039
:106C580037F909201CF01AFF1CF000FD4FF46140C1
:106C68001CF050FF09201CF0CDFF0022A3484FF470
:106C780080411EF014FEA24800211FF0DDF9A14951
:106C880004224B78DFF8A0E26FF300034B709E4BB1
:106C98009E4C1A705A715A709A70DA701A719A71F9
:106CA800DA719B4B033A1A709A4B00201F328EF808
:106CB800000020705A7105900546069006467F2010
:106CC8001FF0D2FA23780E2B01F2B681DFE813F019
:106CD8000F004F009500E0007902DE0330048504C0
:106CE800EA06DC07EF075808B108D00882098A4E7F
:106CF8008A48317801F00F01013149014118FFF745
:106D08001FFE337813F00F0308D1854A92F8012348
:106D1800012A41F09181834A138024E0012B03D199
:106D28007F4B93F819330BE0022B04D17C4B93F87B
:106D38000D33032B05E0032B06D1794B93F80D3364
:106D4800012B41F079810EE0774901220A707748DA
:106D58004FF400711EF0A3FD754BC8221A603378FA
:106D68006FF30303BFE333785A1C01F05FB8704B2D
:106D78001A6822B96D484FF400711EF090FDDFF8D3
:106D880098816C4898F8001001F00F010131490111
:106D98004118FFF7D5FD36B198F800305A1C62F358
:106DA800030388F800305F4B00221A8098F800101F
:106DB80001F00F02022A03D11A7842F010020AE009
:106DC800042A03D11A7842F0040204E0052A05D106
:106DD8001A7842F040021A7001F02EB9062A04D13E
:106DE8004D4B6FF3030119707EE301F00F0101228F
:106DF80012FA01F1198001F01FB9474E4E48317857
:106E080001F00F01013149014118FFF799FD96F88A
:106E1800008008F00F08B8F1070F27DC18F0010F01
:106E2800464B02D00020588002E04FF0FF315980D5
:106E38004FEA6809062209F1010902FB09394FF0F6
:106E4800FF32A9F802204046FFF7D4FDFF2806D0FC
:106E58003B4B03EB40005823437401F0EDB800238B
:106E6800A9F8023008F1010801F08AB800211022BF
:106E780013A8F9F78FFA0FA800211022F9F78AFA58
:106E880023780133237033786FF3030301F07BB861
:106E9800DFF884A09AF8008018F00F0840F03F81CE
:106EA800284E337803F04003DBB2F3B926486FF07D
:106EB8007F43817A0122009301F00F01FF23FFF73E
:106EC80061FD224B93F8692012F0400F08D093F827
:106ED8006C3013F0040F03D0337843F04003337061
:106EE8007378142262F3C7037370737813F0F80F82
:106EF80030D0174800F12001A7E300BF0018014077
:106F0800002C0140D2310020A02C0020D61C0020EB
:106F1800631300203C3B0020D51C00207A63020844
:106F2800742E0020043C0020AC260020000C0140F8
:106F38007C2600201A640208FA640208BE3B00207E
:106F4800F4010020633A0020900C002040570020F4
:106F58001A660208BC4B1B7803F04003DBB2002B17
:106F680000F0D980DFF80483DFF8049398F8003044
:106F780013F00C0B30D1B54E6FF07F4396F82B1001
:106F880006F12100009301F00F0101220523FFF70C
:106F9800F9FC96F84C104FF4860A06F1420001F00D
:106FA8000F010122FF23CDF800A0FFF7EBFC96F8B4
:106FB8004110FF2306F1370001F00F015A46CDF8C2
:106FC80000A0FFF7DFFC042389F8003098F80030B0
:106FD80043F0080301F02EB803F00803DBB2002BDE
:106FE80039D099F800A0BAF1000F03D0984800F101
:106FF800400138E0954E6FF07F4B717D06F10B0034
:1070080001F00F010122FF23CDF800B0FFF7BAFC11
:1070180096F82B1006F1210001F00F010122072339
:10702800CDF800B0FFF7AEFC96F836104FF48603A3
:10703800009306F12C00FF2301F00F015246FFF7E1
:10704800A1FC98F800306AF3C303DBB243F00403F1
:1070580088F800305AE099F800C0BCF1000F08D059
:107068007B4800F16001FFF76BFC99F80020303293
:1070780008E2764E6FF07F40717DFF23009001F0AB
:107088000F0106F10B000122CDF80CC0FFF77AFCC6
:107098009AF80030DFF8C4B103F0100A5FFA8AFAF0
:1070A800DDF80CC0BAF1000F0CD098F800206CF392
:1070B800820288F800205A1C62F303038BF8003020
:1070C80000F0BABF96F82B106FF07F42009206F1DD
:1070D800210001F00F0101220C23FFF753FC96F861
:1070E80036104FF4860300935246FF2306F12C0016
:1070F80001F00F01FFF746FC9BF8003083F0100207
:10710800C2F3001262F304138BF80030042389F8E9
:10711800003000F091BF4E4800F1800195E2B8F1CF
:10712800010F3CD14A4800F1A001FFF709FC002EED
:1071380000F082879AF80030444E5A1C62F3030329
:107148008AF8003096F82B106FF07F4906F121007D
:1071580042460F2301F00F01CDF80090FFF712FC13
:1071680096F82B1006F1210042460E2301F00F017C
:10717800CDF80090FFF706FC96F82B1006F12100D9
:10718800424601F00F010F23CDF80090FFF7FAFBFC
:107198003048802142461EF082FB00F04DBF2C484B
:1071A80000F1C001FFF7CCFB002E00F045872A4B09
:1071B80096221A609AF800306FF303038AF80030B9
:1071C80092E1264E317811F00F0A16D1244800F1C9
:1071D8002001FFF7B5FB204B1B68002B40F02C87E4
:1071E80013A8F9F727FB40221346014613A801F01C
:1071F80023FA3378012200F019BEBAF1010F39D110
:1072080012486FF07F4390F8201000220093163048
:1072180001F00F01FF23FFF7B5FB01F077FA002813
:1072280000F00A873378022262F3030333700D4BB0
:107238001A7842F080021A700B4B5A7842F0020218
:107248005A7000F0F9BE00BF633A0020900C00208D
:107258001A660208001001407C260020D51C002078
:10726800FA660208683A0020263D0020C45E002025
:107278004B60002001F00F0101F10E0303F00F0332
:10728800012B44D89B4849014118FFF759FB9A48FC
:107298006FF07F4390F8201000221630009301F021
:1072A8000F01FF23FFF76EFB1CF020F8337803F083
:1072B8000F03022B13D117F089FB002800F0BC86BE
:1072C8008E4B1A7842F040026FF304121A705A7803
:1072D8006FF345125A703378032200F0A7BD17F0F8
:1072E8005FFB78B117F0FEFB17F0B6FA844B00206D
:1072F8001A7858816FF3C7121A703378042262F330
:10730800030333707F4B1A786FF3000263E5BAF119
:10731800040F4DD1DFF8DC914901DFF810824944B0
:107328004846FFF70DFB98F80010774B01F0040270
:10733800D2B27AB941F004016F4883F800A088F806
:10734800001090F836104FF4860300932C3001F0AB
:107358000F01EEE293F800A0BAF1000F40F06C863E
:1073680065486FF07F45417D01220B3001F00F0128
:10737800FF230095FFF706FB64480122817AFF236B
:1073880001F00F010095FFF7FDFA98F8003005228B
:107398006AF3820388F800303378484662F30303BF
:1073A800337009F1A001FFF7CBFA554600F044BE4F
:1073B800DFF84481FF2398F8201000226FF07F49FE
:1073C80008F1160001F00F01CDF80090FFF7DAFA86
:1073D8002BB2072B18D1337808F121006FF3030380
:1073E8003370237801220133237098F82B100E2371
:1073F80001F00F01CDF80090FFF7C4FA444880214E
:1074080000221EF04CFA0025424E96F86B3013F01D
:10741800040F00F0118698F857106FF07F43002290
:1074280000933D48FF2301F00F01FFF7ABFA96F8F0
:107438006B303A4A03F00F03012B137003D1002D70
:1074480008BF01250CE0022B04D12BB2012B08BF89
:10745800032505E0032B03D12BB2032B08BF072517
:10746800ABB213F0010F02D02D4A3121517713F03E
:10747800020F02D02A4A3221917713F0040F00F04C
:10748800DB853322264BDA7700F0D6BD1948254E26
:1074980000F1C001FFF754FA96F80090DFF85C801D
:1074A80019F00F090CD117F0F1F898F8003069F3CA
:1074B800000388F8003033785A1C62F303033370F2
:1074C80017F076F998F8003013F0010F00F0B48542
:1074D8000022154880211EF0E2F90A4B00225A705A
:1074E800337862F30303337023780133237000F099
:1074F800A3BD00BFFA660208900C0020263D0020BC
:10750800683A00209E3C00204B60002001000020CB
:107518000010014040570020DD0C0020623A002096
:10752800F4010020D51C002000180140C45E002092
:107538008648874E00F1E001FFF702FA0FA8F9F735
:1075480079F90FA902468348F9F7FAF90021824828
:10755800B18090F8C5106FF07F4300220093BB30D4
:10756800FF2301F00F01FFF70DFA7C4A92F86B1028
:1075780092F86C30327843EA012312F0010FB3809D
:1075880010D0A3F1EB0292B20A2A04D9A3F5E6734C
:107598009BB2282B02D8F3880133F38033786FF33A
:1075A800000333707378002B40F04685684AD28810
:1075B8007AB16B4A1BA8117863F303011170227822
:1075C8008DF86F300132227028228DF86C201EF061
:1075D80085F90022F28000F02FBD624EDFF8ACA1E1
:1075E800337803F004085FFA88F8B8F1000F15D172
:1075F80009A841461522F8F7CDFE5B4BCAF8008072
:107608001B684546CDF827303368474643F00403E6
:107618003360564BA3F8368300F00EBD03F08003A9
:10762800DBB2002B67D1DAF80010002940F004859E
:107638004F48FFF785F94F484FF480511EF025F960
:10764800012806D04A4800F1A001FFF779F900F0B7
:10765800F3BC4649B1F83623002A43D009314648DD
:10766800013AF9F76DF9444B03F1100113F8012BB6
:107678000D2A01D00A2A02D1202203F8012C8B42BC
:10768800F4D13E4B4FF03C0808FB073808F11E08C0
:107698004046F9F7CFF8414602463948F9F7FAF873
:1076A800D8B9022F03D1336843F0100304E0032F45
:1076B80003D1336843F040033360327853005BB240
:1076C80003EAC263DB173268DBB263F3C7123260C6
:1076D8001BB1FFF7C9F900F0AFBC0137FFB2042FA7
:1076E80008BF0227254B3C2606FB07363046F9F72C
:1076F800A1F8314626E0DAF80080B8F1000F40F032
:107708009B84737803F02002D2B2002A40D11D4B2B
:1077180009A81A889B781C498DF82630ADF82420D2
:10772800F8F792FE114B5B7A302B07D1FFF79CF9E3
:10773800336843F40053336000F07EBC09A8F9F7BE
:1077480079F809A9FFF770F900F076BCFA66020823
:107758009E3C002008020020900C0020405700208A
:10776800D51C002080260020AB550308A058002017
:10777800FA67020800080140040200200C000020FB
:10778800A9580020B0550308B45503087C260020EA
:1077980003F04003DBB2002B40F08980B14800F1D0
:1077A8006001FFF7CDF8B048F9F744F88046AE49D4
:1077B800AE484246F9F76EF8002873D1AC4B434403
:1077C8005B7A302B6ED1FFF74FF93368DFF8D09230
:1077D80043F48043336099F82B106FF07F43009394
:1077E80009F12100082301F00F010122FFF7CAF86F
:1077F8006423CAF800307F201EF036FDDAF8003026
:10780800002BF8D1984699F88E10D633994E89F8FE
:1078180086304B3B6FF07F4A89F88730964801F0F5
:107828000F0142467433CDF800A0FFF7ABF896F885
:10783800B91106F5D670033001F00F014246FF2357
:10784800CDF800A0FFF79EF896F8C41106F5DD7094
:1078580001F00F014246FF23CDF800A0FFF792F890
:1078680096F8CF1106F5E270013001F00F0142469B
:10787800FF23CDF800A0FFF785F896F8DA1106F592
:10788800E87001F00F014246FF23CDF800A0FFF792
:1078980079F899F899107948CDF800A001F00F010E
:1078A800424646E07648F8F7C5FF75494AE796F834
:1078B80002B0DFF8EC910BF0020B5FFA8BFBBBF127
:1078C800000F3AD199F82010FF236FF07F4809F193
:1078D800160001F00F015A46CDF80080FFF752F864
:1078E800684B93F86B3003F00803DBB2002B00F011
:1078F800A38399F82B10012209F1210001F00F014F
:107908000323CDF80080FFF73DF83368554843F46A
:10791800003300F180013360FFF712F855485A46EA
:1079280090F8E51100F5EC70CDF80080033001F017
:107938000F01FF23FFF726F87EE3CAF8008099F8C5
:1079480020106FF07F4300934246FF2309F1160091
:1079580001F00F01FFF716F82AB241F211139A420B
:107968001DD1434B5B7A302B13D1FFF77DF8336879
:10797800454668F3514368F38E3368F34D333360FB
:10798800414B1A7868F303021A7023780133237085
:1079980052E33E48F8F74EFF3C49FFF745F8394EA9
:1079A80096F86B3013F0040F00F0468325B9384879
:1079B80020211022F8F7EEFC7F201EF055FC99F8E4
:1079C80057106FF07F43002200933248FF2301F0E5
:1079D8000F01FEF7D7FF96F86B202F4B02F00F022E
:1079E8000D2A1A7005D125B92C4A412191754FF4F9
:1079F80080551A78062A08D12AB2B2F5805F04D1D8
:107A0800264A3621D1754FF488551A78082A08D1A4
:107A18002AB2B2F5885F04D1204A3821117641F2A2
:107A280010151B780B2B09D12AB241F210139A4278
:107A380004D11A4B2A225A7641F211150D486FF0DB
:107A48007F4390F8F0110022009300F5F370FF23B4
:107A580001F00F01FEF796FF96F86B3013F0010F57
:107A6800AAD0E9E2FA6702081A010020A958002002
:107A7800A058002001000020140D00201F0D002038
:107A8800FC00002040570020D51C002038010020B1
:107A980004020020DD0C0020623A0020F4010020DE
:107AA800900C0020A34B1A7842B300221A700F20C2
:107AB800FAF7CAFA06460A20FAF7C6FA9E4B9F4911
:107AC80058824A7812F0010F18D06436301A588359
:107AD8009B4B1A78642A01D19B321A701B78984EF6
:107AE800FF2B0BD00A21B3FBF1F1964B193119800A
:107AF80095481EF0A1FA337801333370DFF86482B9
:107B080098F8003013F00F0612D18E4B19228B48CB
:107B18001A804378192143F0010343708A481EF004
:107B28008BFA8A4800F12001FEF70AFF04967CE2EE
:107B3800012E68D1804B5A8BA2F1690189B21129B3
:107B480008D8049911F0010F04D141F00101C9B21C
:107B580004910592049A12F0020F0DD15B8A7C4AB7
:107B68001380A3F5C263023B9BB2D72B04D80498B9
:107B780040F00203DBB204931B20FEF783FF059954
:107B8800744B0AB2632A05DD642192FBF1F23032AC
:107B98001A7401E0092A0CDD059A11B2642291FBDE
:107BA800F2F002FB10120A2012B292FBF0F230320D
:107BB8005A74059802B2642092FBF0F100FB11217F
:107BC8000A2209B291FBF2F002FB101230329A74C9
:107BD8005B4B1B78FF2B08D158495B484B786FF3F8
:107BE80000034B7000211EF027FA049A032A40F084
:107BF80023825248002143786FF3000343705248B0
:107C08001EF01AFA11E2022E03D1534BC8221A6051
:107C18000BE2032E16D1504B1B68002B40F00C8250
:107C28004A4800F14001FEF78BFE1B20FEF72AFFB1
:107C3800414B5B8AA3F51E630F3B9BB2542B00F2AA
:107C4800FB81F2E1042E0CD13B4B988A0FF0DAFC51
:107C5800002840F0F1813D4800F16001FEF770FE18
:107C6800E3E1052E07D1344B988A0FF0CBFC0328AB
:107C780040F0E281D9E1062E40F0D78122786FF3F7
:107C8800030301322270D5E1344800F12001FEF7E8
:107C980057FE334B1B78002B00F0CE81237801333D
:107CA8002370304B1A786FF30302FFF794B82D4E08
:107CB800DFF8A480337813F00F021AD12A4800F1B4
:107CC8002001FEF73DFE2948F8F7B4FD2749024692
:107CD8002748F8F7B7FA2548F8F7ACFD254BA3F87D
:107CE800160233785A1C62F3030333701BF0B4FF97
:107CF80091E0012A16D1D8F80030002B40F09C8181
:107D08001BF0D6FF012840F097811B48F8F792FD39
:107D1800194902461948F8F7BDFD002840F08C8142
:107D280011486FE0D8F80020002A40F085810B2127
:107D38007BE000BF66130020B0310020D231002064
:107D4800E41C00208C0C0020002C0140BA680208BA
:107D5800D81C0020F40100207C2600203A69020883
:107D6800D41C0020D51C00207A6902087401002068
:107D780050380020445C002092010020455C00201F
:107D8800874E337813F00F080CD186484146FEF72A
:107D9800D7FD33785A1C62F303033370824BA3F880
:107DA800028049E1B8F1010F18D1804804211DF083
:107DB8006CFD002800F040817A4800F12001FEF7B0
:107DC800BFFD33784FF0FF315A1C62F30303337061
:107DD800774B64221A60744B59802DE1B8F1020F79
:107DE800DFF8CC811BD1D8F80030002B40F024817B
:107DF8006E4804211DF049FD002840F01D816A4BA2
:107E08005880684800F14001FEF79AFD33785A1C03
:107E180062F3030333706423C8F800300CE1D8F828
:107E28000020002A40F008810C21217062F303032E
:107E3800A9E0604910234FF40052CB700D3B8B70C2
:107E48000A805D481DF0D2FC0A2200215B48F8F741
:107E5800A1FA80201DF02EFC237801332370504BAB
:107E68001A786FF303021A70514BC8221A60E3E0C4
:107E78005348DFF848A100F12001FEF761FD9AF8A8
:107E88000030002B00F0D8804E48DAF80020444E2D
:107E98000260BAF8042082809AF80620827131784C
:107EA80011F00F0159D1DFF80881D8F80010002926
:107EB80040F0C2809AF80410A2F5A6524FF0640B65
:107EC800103A0BFB01229AF805004FF00A0909FB4A
:107ED80000200393F9F724FE3B49F9F72DFF0246EA
:107EE8009AF80200039BA0F5A65010380BFB030B71
:107EF8009AF80100354B09FB00B018600392F9F7B6
:107F08000FFE039A01461046F9F75AFD304B1860E8
:107F1800F9F712FA1EA3D3E9002382468B46F9F734
:107F2800E5FC002800F08880504659461AA3D3E99A
:107F38000023F9F7D1FC00287ED0FEF7DDFD337869
:107F480048465A1C62F303033370C823C8F800304C
:107F580009F078FDC0B207906EE001296CD10D30B0
:107F68000799832200F044FD114BD3F80080B8F143
:107F7800000F61D140461DF09DFB2378013323702B
:107F8800337868F30303337056E000BFAFF3008023
:107F9800736891ED7CFF7F400AD7A3703D00804055
:107FA800D51C0020DA690208BE3B0020000C014005
:107FB8007C260020CE31002000100140EC1C00205F
:107FC8003A6A02080402002000007A44E81C0020F3
:107FD800D01C00208448854E00F12001FEF7B0FC3B
:107FE800F37913F0010F27D0DFF8488298F8009052
:107FF80019F00F0920D17E4B0A22597818781039C8
:1080080002FB0011B1701979D878103902FB001100
:108018007170D9799B79103902FB0312327018F00C
:1080280061FFF37969F30003F37198F800305A1C83
:1080380062F3030388F80030DFF8FC9199F80060D8
:1080480016F001063EF43BAE6A4B01221A701AF094
:1080580099FD2378092B01D00D2B28D101206649E1
:1080680012F0F8FA654B664A5B7803F01F03D35C9D
:10807800644A522B137002D1634B01221A70634B6E
:10808800634A03F1200153F8040B8B4242F8040BB6
:10809800F9D1002117A812F007FB17A80D211BF032
:1080A80077FD5C4B1A78013202F003021A7099F8D6
:1080B800006006F00206F6B2002E00F08B800FF08A
:1080C8004FFD13F0BDFE06980322431C93FBF2F20A
:1080D80002EB42029B1ADBB20693002B79D1DFF840
:1080E800488198F84960C246002E4DD0022E03D12F
:1080F80098F80130312B49D023780E2B13D14648FC
:1081080046490522F8F7C6FB8246002840D1B21F2F
:1081180037484349F8F714FC344B5646DA7942F0AD
:108128000102DA7135E00D2B03D13E483A490722A6
:1081380027E0032B22D13C4B002713F8012F2C2AD0
:1081480003D00137FFB2B742F7D113A832493A46F4
:10815800F8F7F6FB7B1C07E00AEB03025278303A8B
:10816800D2B2092A03D80133DBB2B342F4D30AEB03
:108178000701FA430FA80231D21802E0264909A8DC
:10818800721EF8F7DDFB03E0069E02E0012600E020
:1081980000261E4B204A03F1100153F8040B8B42B2
:1081A80042F8040BF9D1214B214A03F1100153F88D
:1081B800040B8B4242F8040BF9D1402388F81130A4
:1081C8001C3B88F82230023B88F84B301BF068FAD9
:1081D80000E0002699F8003003F0F5036FF3000380
:1081E80089F80030FEF76BBD7A6A0208B0550020A6
:1081F800DA1C002066130020E15B0020E05B002011
:1082080084A00208D03A0020D41C0020F4010020E9
:10821800163B00207E3A00204F580020B75503082F
:1082280054580020EC1C00204E5800200402002066
:1082380060580020D51C002028580020AFF300808B
:1082480010B5044640181146F8F796FA2046F8F794
:10825800F1FAC0B210BD42540131C8B270470000F3
:1082680010B50D4B0D4A1B780C460E2101FB03235C
:10827800997A39B101390523594301F56E514431D1
:1082880089B201E043F6C4310019042209F0EBFB7E
:10829800201DC0B210BD00BF655E0020A8170020D9
:1082A80010B5054B0C46197800190131042200F06D
:1082B8009FFB201DC0B210BD655E002000F5344054
:1082C80008B5CB3009F0BEFB10F0FF0F14BF00203B
:1082D800012008BD10B50A4600210446FFF7B0FF8B
:1082E80001462046FFF7DCFF114A01462046FFF70A
:1082F800A7FF232201462046FFF7ADFF014620468F
:10830800FFF7AEFF5B2201462046FFF7A4FF2322BA
:1083180001462046FFF79FFF01462046FFF7A0FFD2
:108328007C2201462046BDE81040FFF794BF00BFFD
:10833800BD55030810B55D220446FFF78CFF0D22DA
:1083480001462046FFF787FF0023235410BD38B5A8
:108358001D460C4640182C1911461A4600F048FBD9
:10836800E0B238BD2DE9F04118490446FFF7B2FFE5
:10837800174F0E263B78174D73430146EA5A20469D
:108388000423FFF7E4FF202201462046FFF763FF9E
:108398003B78014606FB035320469A7A0223FFF7EF
:1083A800D6FF202201462046FFF755FF3B780146BD
:1083B80006FB035520466A7A0323FFF7C8FF0146E8
:1083C8002046BDE8F041FFF7B5BF00BFC055030820
:1083D800655E0020A81700202DE9F047264E0E22E2
:1083E8003378264F534337F90380FA1824494FF45A
:1083F8007A73044698FBF3F8157AFFF76BFF4E2261
:1084080001462046FFF727FF1E4B1C2202FB0535BD
:108418005FFA88F8B8F1030F01460CBF05F11202A4
:1084280005F108022046FFF70BFFA146804600250C
:1084380019E019F8013BA32B07D133780E2202FB70
:108448000373204629465A7A08E0242B09D1337849
:108458000E2202FB03739A7A204629460223FFF76D
:1084680076FF0135EDB24545E3D120462946BDE802
:10847800F047FFF75FBF00BF655E0020A817002028
:10848800CA550308A4A00208074B187800F0040096
:10849800C0B240B11A686FF382021A60034B00221F
:1084A8001A70034B18787047783A0020101D002086
:1084B800F81C0020054B00211970054B05481A6867
:1084C80061F382021A601222F7F764BF101D0020C0
:1084D800783A0020F81C002038B5084C0849227862
:1084E8000546F7F7AFFE23780021E954054B1A68D3
:1084F80061F382021A60207838BD00BF101D002089
:10850800F81C0020783A0020064A07491378112BF6
:10851800C85401D801331370044A136843F00403A4
:1085280013607047101D0020F81C0020783A0020C6
:10853800054B1B7813F0010F05D1044B181810F8E0
:10854800010CFFF7E1BF7047111D0020BA6A02084D
:108558002DE9F041334C002314F8101094F82A2028
:1085680001F00F0161F3030284F82A2004EB4000B4
:1085780084F8293084F828304378DFF8B88063F32A
:108588000712638C4FF4D277E38498F800302A26D8
:108598007B4306FB0133244D2448E95A84F82A20FA
:1085A8001DF048FD98F8003094F82A207B4302F02B
:1085B8000F0206FB0233EB1859881C48013989B2AF
:1085C8001DF03CFD01210A4618481DF003FD01215C
:1085D80016481DF0F0FC98F8003094F82A207B43E8
:1085E800120906FB02331248E95A1DF023FD98F8D8
:1085F800002094F82A3057431B0906FB0376AD196F
:1086080069880B48013989B21DF016FD01210A4617
:1086180007481DF0DFFC06480121BDE8F0411DF0C8
:10862800CABC00BF121D0020C66A0208000800402C
:10863800003401403E1D002030B5164C94F82B50F4
:10864800A38445F00105002384F82B50628484F844
:10865800211084F8203019E0C55CA5F13002D2B2AF
:10866800092A08D9A5F14102D2B2052A9ABFA5F173
:108678003702D2B22A46084D013305EB420292F87E
:10868800495392F84823257062700234DAB28A425C
:10869800E2D330BD121D0020C66A0208124B10B585
:1086A8009A8C0024DA8483F8294083F828402246EB
:1086B80001210E481DF08EFC64210C481DF0BAFC07
:1086C80032210A481DF0BAFC0121224608481DF053
:1086D80081FC642106481DF0ADFC05483221BDE847
:1086E80010401DF0A9BC00BF121D0020000800406A
:1086F8000034014010B500212C220348F7F74AFE48
:10870800BDE81040FFF7CABF121D002070B5214C0C
:108718002378042B39D8DFE803F0030D152A30003D
:108728001D4B012093F82B3013F0010F30D020702F
:10873800013870BD184B93F82000FFF709FF02239A
:10874800237022E0144DEE8CFEB9FFF7A7FF95F8D1
:10875800203095F821200133DBB29A4285F8203089
:1087680001D8042300E003232370304670BD0A4B70
:10877800D88C50B90123237070BD074BDD8C35B9F7
:10878800FFF7B8FF2570012070BD002070BD0020E4
:1087980070BD00BF3F1D0020121D0020044B0022A9
:1087A8005A701A709A7842F001029A70704700BFA6
:1087B800681E0020202102480A46F7F7EBBD00BFDB
:1087C800F401002038B5044608460D46F8F732F89B
:1087D80098B10319202B094BC8BFC4F120001C19FC
:1087E800002308E014F8012BE02A14BFEA5C2022D9
:1087F80004F8012C01338342F4DB38BDF401002076
:108808000D4B46F669321B689B6893420FD043F6BE
:10881800FC2293420BD0122B09D0B3F5E97F08D084
:1088280046F60D401B1A584240EB030070470120E2
:1088380070470120704700BF781D0020F0B51F4623
:1088480087B006460C46084600211546F7F7A2FDF4
:10885800244B07B19F80B3F9041005A801EB8601EA
:10886800042209F000F9002605AB9B5D013BDBB251
:10887800B92B35D81D2B4FEA031209D8D31803F5A5
:108888002641684601F5BF71112209F0ECF80BE0AA
:108898001549D3185B186A4603F110071868596818
:1088A8000833BB4203C2F9D12046F7F7C3FFC7B26A
:1088B8006846F7F7BFFF3818A84203D8E019694699
:1088C800F7F75AFF6846F7F7B5FF7B1C1B18AB4252
:1088D80003D2E0190549F7F7B7FD0136042EC3D1D5
:1088E80007B0F0BD681E0020C8370308E25503082A
:1088F80010B500216C220446F7F74CFD0123A37044
:1089080010BD002343700370837843F00103837024
:10891800704700002DE9F0419378804613F0010F6D
:108928000D4614463AD06FF3000393701AF090FE88
:108938006378002B32D123780BB90A336370A3789C
:10894800174F6FF30003A3701AF082FE217807EB2C
:1089580008066118073130462A46F7F7F1FF304616
:10896800F7F768FFC6B2AE420DD80AD200232370CB
:1089780006EB08000A33637038182021AA1BF7F7A2
:1089880009FDAE420AD12278A3181B7A1BB1013225
:108998002270BDE8F08123700A236370BDE8F0817E
:1089A800F4010020054B1A780AB100221A701B78CE
:1089B80046F68A4202FB0311FFF704BF5B1D002045
:1089C800F8B505460C460818002109F031F8013CB5
:1089D800E4B26719384609F035F8C6B2202E03D834
:1089E8003846002109F024F80CB1202EEFD9F8BD43
:1089F80002F00F03032B22F07F0230B5D2B20CD95C
:108A08004FF47A7491FBF4F42025E4B2057002B1B6
:108A180014B13034047000220130B1F57A7F05DBDF
:108A28004FF47A7491FBF4F504FB1511022B0BD962
:108A3800642491FBF4F42025E4B2057002B114B16A
:108A48003034047000220130632904DD642491FB72
:108A5800F4F504FB1511012B0AD90A2391FBF3F352
:108A68002024DBB2047002B10BB130330370013043
:108A7800092904DD0A2391FBF3F203FB12113031BB
:108A8800017030BD13B5104B01461B689A899C7B59
:108A980012F0100214BF0220012034B10B4C9B7C51
:108AA8002478634303FB001109B23AB10DF10600C3
:108AB800022208F0D8FFBDF8060002E0084608F0D8
:108AC800C1FF00B21CBD00BF781D0020071E00209A
:108AD80010B50F4B1B689A899C7B12F0100214BFCB
:108AE8000221012134B10B4C9B7C2478634303FBA6
:108AF800010000B22AB108490222BDE8104008F07E
:108B0800ACBF054B1968BDE8104008F091BF00BF25
:108B1800781D0020071E0020201E00203038C0B21B
:108B2800092894BFFF20002070470000024B1A78E4
:108B38006FF300021A707047571E002070B5FFF7D8
:108B4800F5FF884B1A781E2A01D91E221A70864C06
:108B58002678254606F0F006202E72D109F0CEFAC6
:108B680000286ED1814B1B7833B92378C3F30312E5
:108B7800013262F307135EE07D4B1B7803F080033C
:108B8800DBB2002B59D07B48F7F754FEC5B27A4CBC
:108B9800BDB1204679493246F7F7D2FE0A2D0BD8E7
:108BA8002A4620467349F7F7CBFE60193146C5F1CE
:108BB8000A02F7F7EFFB04E020466E490A22F7F7AE
:108BC800BFFE6F4B1B7813F0010F01D0472300E065
:108BD8002023E372684C042204F10C00A521F7F766
:108BE800D9FB684B1A7852B1FF23012A237306D99F
:108BF800022A637303D0032AA37318BFE373624C7A
:108C0800257815F0600502D194F8A33013B95F48B0
:108C18005F4902E05D4804F1A3010622F7F790FEE0
:108C28005C4B1B78452B40F09A81002D40F09781D2
:108C3800237843F08003237070BD4F48564932466D
:108C480082E12C7804F0F004102C3FD109F056FA98
:108C580000283BD1202251494748F7F771FE464882
:108C68004E492246F7F76CFE4D4B1B7813F0010F67
:108C780006D04C48F7F7DEFD4A4902464A4805E067
:108C88004A48F7F7D7FD494902464748F7F758FEDB
:108C9800364B1B781BB946484649102254E14448D4
:108CA80045491022F7F74CFE314B1B7803F080033F
:108CB800DBB22BB13B48F7F7BDFD02463F484FE01A
:108CC8003A48F7F7B7FD02463C4842E02B7803F0F4
:108CD800F003302B7ED109F011FA00287AD1264C06
:108CE800202237492046F7F72BFEA521052204F15B
:108CF8000B00F7F74FFB334B1B78042B02D9FF23EC
:108D0800E37300E002D1FF23A37301E0032B02D138
:108D1800FF23637301E0022B02D1FF23237300E0DA
:108D28000BB1FF23E372284B5B7813F0600F05D07B
:108D38003F23E37223736373A373E373234B1B789B
:108D480003F02003DBB233B11848F7F773FD02468E
:108D58001F481649F8E01348F7F76CFD02461C480F
:108D68001049F1E0631E0020571E0020AC260020A9
:108D78008026002084260020F4010020B4FD02088B
:108D88005C5E002079270020B42600200E02002017
:108D9800CFD30208401D002072FD0208B733030834
:108DA800263D002001350308010200202235030872
:108DB8000402002084390308D83303081102002074
:108DC80074D402089F2C0020D8310020783A002063
:108DD8000F0200202B7813F0F0030CD120226049F9
:108DE8006048F7F7ADFD604B5E4819888322BDE8FF
:108DF8007040FFF7FDBD602B1ED109F07FF9D8B98F
:108E08005A4920225748F7F79BFD5948F7F712FDB2
:108E1800574902465748F7F793FD5748F7F70AFDB1
:108E2800554902465548F7F78BFD5548F7F702FDB7
:108E380053490246534887E02B7803F0F003102B80
:108E480006D109F05BF918B146484F4920227BE06A
:108E58002B7803F0F004402C02D0502C78D108E095
:108E680040484A492022F7F76BFD494B1B784BB91C
:108E78004CE03C4847492022F7F762FD464B1B78F7
:108E88003BB943E0454B5A7882B11B78022B14D189
:108E980005E0434B1B7813F0010F07D00DE0414864
:108EA800F7F7C8FC3F4902463F4835E03F48F7F727
:108EB800C1FC3E4902463C482EE03D48F7F7BAFC63
:108EC8003B4902463848F7F73BFD402C0BBF334B74
:108ED800384B5B78DB78022B0AD0042B0FD0012BA0
:108EE8001CD13548F7F7A6FC3349024633481BE046
:108EF8003348F7F79FFC32490246304814E03148BE
:108F0800F7F798FC2F4902462C480DE02E48F7F752
:108F180091FC2D4902462448F7F712FD2B48F7F734
:108F280089FC2A4902462548F7F70AFD284B1B7891
:108F3800ABB9202107222148F7F72CFA2248F7F786
:108F480079FC214902461D48BDE87040F7F7F8BC96
:108F5800204A6FF3071313701F4B00221A6070BD6D
:108F680011D40208F4010020561D0020F0D3020895
:108F7800F0CC0208F8010020FACC02080802002010
:108F8800F5CC02080F02002053D40208F933030875
:108F9800603A00201A340308AC26002072360020FC
:108FA8005C5E0020BF340308FD010020643503081F
:108FB80001350308542600203B3403080D02002025
:108FC8005C3403087D340308433503089E340308E2
:108FD80057340020571E0020781D0020204B70B504
:108FE800F022204D1A702B7813F0010F0BD01E4C75
:108FF800207810F0010006D11C49FFF7D3FC237834
:1090080043F0010323701A4E3378532B0ED1164CBC
:10901800237813F0010F07D000201649FFF7C2FC90
:1090280023786FF300032370FFF780FD3378232B39
:1090380014D10D4B1B7813F0010F0FD1FFF776FDFC
:109048002B780D4A43F006032B701378013BDBB2F3
:1090580013700A4A52F82320094B1A6070BD00BFEA
:10906800631E0020571E00207D1D0020882903084C
:10907800401D002067290308371E0020441E0020D9
:10908800781D00202DE9F0415C4BF0225C4D1A70F0
:109098002A7802F01003DBB2002B2DD1594963F373
:1090A80047120B601C462A70574A9A5C2D2A01D039
:1090B8000134E4B20133082BF6D1544E3A2130463C
:1090C800F7F7E6F938B1801BC0B2013030182146F5
:1090D8000222FFF78DFC4E4B1B78452B40F08B800E
:1090E80000242046013412F003FF082CF9D12B7814
:1090F80043F010032B7038E0464C237813F0010F2F
:1091080017D1404E4448FFF7F3FB404F31683846CB
:1091180001310222FFF76CFC2D23BB70307846F634
:1091280095533E496522FFF789FB237843F00103F5
:10913800237003200D21384AFFF7ECFB2D78304EC1
:1091480015F0E00541D110203549FFF72BFC304BD5
:109158001B78442B0DD12B4A136801332A4903F09D
:109168000703C95C2D29F8D01360BDE8F041FFF76B
:10917800DDBC532B0DD132784E3B63F3471232706E
:10918800204A28491268062000FB02125380BDE8D5
:10919800F081232B2FD11B4B1D60337803F0EF0395
:1091A80065F347133370FFF7C1FC23781E4A43F079
:1091B800060323701378013BDBB213701B4A52F885
:1091C80023201B4B1A60BDE8F081104C1020194970
:1091D800FFF7E8FB04F110002821F7F759F950B11F
:1091E800001B3178C0B20130201849098022BDE83F
:1091F800F041FFF7FDBBBDE8F08100BF631E002012
:109208007D1D0020201E0020A13B0020F40100202D
:10921800401D0020571E0020681E00206F1E0020E1
:1092280004290308BE3B0020371E0020441E0020EE
:10923800781D002025290308454B2DE9F041F0222F
:10924800444E1A703378444D43F0010333702B6851
:10925800424C9B7C022B06D1414B1B7803F0400308
:10926800DBB23BB10FE0012B0DD13E4B1B7813F065
:10927800010F08D109F0BAF8236800206FF355539D
:109288002360394944E0A378344F03F02003DBB26C
:10929800C3B909F0ABF8F87800F02000C0B288B97B
:1092A8002968324B897C1A7861F301021A703B688D
:1092B8002D4943F400133B60FFF774FB2C4B8022CD
:1092C80083F843200DF04EFD804678B12B689B7CD7
:1092D800012B08D1234B5B7803F01003DBB213B1E9
:1092E8000020244914E00020234911E00DF06AFD14
:1092F800074610B1404621490AE00DF0ABFD10B118
:1093080038461F4904E01A4B93F8433013B91D49F6
:10931800FFF748FB1C4B1B78232B16D1FFF706FCE5
:10932800337843F00603337009F060F823686FF36D
:10933800555323600CF00AFC144A1378013BDBB246
:109348001370134A52F823302B60BDE8F08100BF38
:10935800631E0020571E0020781D0020783A002048
:1093680080260020263D0020A92903082B3D002047
:1093780001220020EB290308CA2903082D2A030823
:109388000C2A03084E2A0308401D0020371E00201F
:10939800441E00202DE9F3416E4B6F4DF0221A70E8
:1093A8002B686E4C9B7C1BB9637843F0100302E07A
:1093B800637843F008036A4E6370337843F001031F
:1093C8003370238823F47E6323F01E03DB04DB0C55
:1093D800B3F5805F08D0634B1B7883B15F4B5B7834
:1093E80003F00803DBB253B1637800206FF3410345
:1093F8005D496370FFF7D6FAF8F762FE84E0637898
:10940800564F03F00203DBB2FBB9BB78EBB9574BFD
:1094180093F8008018F0010817D1F8F751FE7B780F
:1094280043F002037B702B68B3F91030022B7B7872
:109438000CBF43F0040368F3820300217B7008200B
:1094480001220B460091F9F759F9A378434A032BF7
:1094580028D003D8012B0BD00DD806E0052B2DD032
:10946800517825D3FF2B32D12BE000203E4949E02B
:1094780000203F4946E03F48F7F7DCF9DFF82C8148
:10948800C7B23C4908F110003A46F7F759FA0F2FCE
:109498003AD807F1100040442021C7F11002F6F72E
:1094A80079FF31E0344B187800282DD1334929E071
:1094B8006FF3410151700020314923E00020314908
:1094C80020E06FF34101517000202F491AE0053B5D
:1094D800DBB26FF34101022B517002D100202B49FE
:1094E80010E0012B02D1002029490BE0032B02D107
:1094F8000020284906E0052B02D10020264901E07A
:1095080026490020FFF74EFA637803F00203DBB226
:109518000BB9F8F7D5FD224B1B78232B18D1FFF791
:1095280005FB3378002243F0060333706378A2709A
:1095380003F0E50362F382036370F8F7C1FD194A8B
:109548001378013BDBB21370174A52F823302B60B3
:10955800BDE8FC81631E0020781D00205C5E0020B1
:10956800571E002072360020A9290308625E0020D9
:10957800EC2503086B5E0020605E00200D260308C2
:10958800B12A030891260308F42603082E260308A7
:109598004F26030870260308B2260308D3260308BB
:1095A800401D0020371E0020441E0020F40100202A
:1095B8007B4B2DE9F341F0227A4E1A7033787A4DBD
:1095C80043F0010333702B68784C9B7C022B11D13C
:1095D800774B1B7803F04003DBB293B1754B1B78D4
:1095E80003F02003DBB2BBB1A37803F04003DBB286
:1095F8003BB111E0012B0FD16F4B1B7813F0010F1A
:109608000AD1F8F75DFD2368002023F480036FF387
:10961800D753236069498FE0A778DFF8908107F076
:109628004003DFB2002F34D1F8F74AFD2968644BB4
:10963800897C1A78384661F301021A70D8F800302C
:109648005E4943F4800367F3D753C8F80030FFF747
:10965800A9F92B68198A21B90091082001220B4623
:1096680015E00BB2022B0CD101223B4608203946EB
:109678000097F9F743F8534B1A7842F008021A702A
:1096880007E0012B05D100970E2039463A46F9F735
:1096980035F80DF067FB074678B12B689B7C012BEA
:1096A80008D1454B5B7803F01003DBB213B10020FF
:1096B800454941E0002045493EE0414B394618788C
:1096C80000F00300F8F734FEFF280FD13D4B1B785C
:1096D80003F01803182B31D0A07800F08000C0B236
:1096E80010B138463A4927E03A4925E00DF06AFBBF
:1096F8008046E0B1334B187800F008085FFA88F824
:10970800B8F1000F0AD1F8F769FFC0B2022801D8F2
:1097180040460AE0062811D8404604E000F0100050
:10972800C0B210B138462C4906E02C4904E00DF0CF
:1097380091FB18B12A494046FFF734F9294B1B78A9
:10974800232B29D1FFF7F2F9337843F0060333705E
:10975800F8F7B6FC236823F480036FF3D75323602C
:10976800184B1A786FF3C3021A701F4A1378013B1B
:10977800DBB213701D4A52F823302B60104B1B7854
:1097880003F00303022B02D10DF0C2FA20B102B09C
:10979800BDE8F0410CF0DAB902B0BDE8F08100BFD5
:1097A800631E0020571E0020781D0020783A0020F4
:1097B80080260020B4260020263D0020A929030881
:1097C8002B3D0020901F0020EB290308CA2903081D
:1097D800B12A0308D22A0308902A03086F2A03082B
:1097E8000C2A0308401D0020371E0020441E0020BC
:1097F80010B5FFF79BF90A482523C377094B0A4A96
:109808001B6813219B7C1C3001FB03235B780939FF
:1098180003F00F0359438322BDE81040FFF7E8B86F
:10982800F4010020781D0020833A00202DE9F0473C
:10983800514D524F2B78F02243F001032B70504BBF
:10984800DFF878911A703B689C6847F2F373E21A64
:10985800544244EB0204132161434A4A565C5318AC
:10986800C6F300065FFA86F89246B8F1000F23D1D6
:1098780040464549FFF796F899F80030232B79D1EF
:10988800FFF754F92B78414A43F006032B701378FD
:10989800013BDBB213703E4A52F823303B603D4B2C
:1098A8001E703D4B1E703D4B1E703D4BC3F8008033
:1098B8003C4B1E70BDE8F08799F80020232A21D17F
:1098C8009A786FF300029A700EF0F6F9FFF72EF906
:1098D8002B782E4A43F006032B701378013BDBB23A
:1098E80013702B4A52F823302A4A3B600023137026
:1098F800294A1370294A1370294A1360294A137098
:10990800BDE8F087532A13D19A7812F001010FD1DC
:1099180072206043244D42F001022E5C61F3000680
:109928002E549A701E4B01221A60204616F022FD12
:10993800132303FB04A39B7813F0010F02D000202C
:109948001A4913E0164B1B6873B9382102221848CC
:10995800FFF74EF8204615F0A7FF014615480222EA
:10996800BDE8F047FFF744B813490020BDE8F047C9
:10997800FFF718B8BDE8F087571E0020781D0020B3
:10998800631E0020833A00203FE20208371E0020B1
:10999800441E00205D1D0020861D0020071E00209B
:1099A800201E0020121E0020C4540020E22C0308B0
:1099B800120200200D020020C12C0308401D0020C7
:1099C8002DE9F0412D4E2E4F307800F5E240F13070
:1099D80008F038F83B78C4B213F0010F26D0294DAF
:1099E8002B78552B0AD1EC2C01D0013CE4B230780D
:1099F800214600F5E240F13008F01AF82B78442BA4
:109A08000DD1A4F11403DBB2D72B01D90134E4B290
:109A18003078214600F5E240F13008F009F82B785B
:109A2800532B03D1FFF782F80EF046F9164B1B783B
:109A380003F08003DBB253B13B7813F0010F06D07B
:109A4800124820210422BDE8F041F6F7A3BC14F027
:109A5800800F0F4805D12B230A210374614311306D
:109A680006E02D230374373B5C43113004F5206175
:109A78000322BDE8F041FEF7BBBF00BF071E002070
:109A8800571E0020401D0020783A002004020020C4
:109A9800F40100201FB5204B20491A781AB1087824
:109AA80040F00100087009781C4C11F0010F31D00A
:109AB8001B490978532901D00AB103E082B9012270
:109AC8001A700DE023290BD1002018701549FEF7F4
:109AD80069FFFFF72BF8237843F00603237019E09A
:109AE8001B78012B16D120210A460F48F6F752FCA5
:109AF8000E4B68461B681022996807F0B4FF0024D3
:109B080009491DF8040001EB440101341AF0ECFE88
:109B1800102CF5D11FBD00BF071E0020571E0020C6
:109B2800401D0020FA2F0308F4010020781D0020B2
:109B3800034B1B78532B01D1FEF7F8BF704700BFCA
:109B4800401D0020084BFF281A68936807D1917BB5
:109B580041B10649927C097801FB023302E0927C0C
:109B680002FB003318467047781D0020071E0020AE
:109B78004328F8B504460D46174608D1114B0A2666
:109B88001A7891FBF6F66FF3C3021A7000E00E46DE
:109B98002046FEF7C3FF90B10A4B303C1A780A26DC
:109BA80002F00801C9B2002918BF002506FB0546C6
:109BB8006FF3C30236B21A70BE42A8BF3E4630B237
:109BC800F8BD00BF571E0020624B2DE9F3411A680B
:109BD8009846157C977C604C2DB16048217802220C
:109BE800FEF706FF00E02570FF01237807F51C4704
:109BF80007F5B47707EB4307594E0BB90DB10FE0E2
:109C080015B901A8394601E001A8B91E022207F0DA
:109C18002AFF9DF80430F3759DF80530337605E08A
:109C280006F117003F210222F6F7B4FB5B23B37558
:109C3800023373764B4B1B7813F0010F5DD04A4B00
:109C48001B78A3F13002D2B2092A31D822780AB996
:109C5800002D3CD1454A117896469942444A01D094
:109C68000021117043481178A3F1300490F800C026
:109C780004EB840404EB010802A801318444C9B24E
:109C88003D48641810F80880005D0CF8048C1170C9
:109C980008B1032901D9002111708EF800300DB9DF
:109CA800384600E0B81E01A9022207F0D6FE17E0E8
:109CB800232B04D12F4B1A7892B9013205E02A2BB5
:109CC80005D12C4B1A785AB1013A1A7008E0532B77
:109CD80006D12A4A533B1370264A1370FFF728FF10
:109CE800274B1B7803F08003DBB2002B2FD0214BCE
:109CF8001B78F6182023F37529E045B31A4B18781A
:109D0800A0F13003DBB2092B10D81C4A137803B931
:109D18002370013303F001031370D8F80030217861
:109D2800B3F91020FFF724FF207005E0432803D182
:109D3800124B1B7803B92370114B1B7803F0800377
:109D4800DBB223B1054820210222F6F723FBBDE848
:109D5800FC8100BF781D0020871D00200202002022
:109D6800F4010020571E0020401D00205A1D00202D
:109D7800861D0020581D0020346E0208121E002087
:109D8800783A0020F7B5384E384D3378384C6FF3B1
:109D98004103337019F04EFAFFF7CAFE02238DF81B
:109DA80007302B7883B1334AD17941F00101D17161
:109DB800314A207802EBC3035F6B93F83920397876
:109DC800FFF7D6FE38700DE0337813F0010F06D098
:109DD8002378303BDBB2062B9CBF264AD370032383
:109DE8008DF80730337813F0010F12D0234B1B780E
:109DF80003F08003DBB263B129781F4B204803EBE3
:109E0800C10393F838309DF80720C0182021F6F7D1
:109E1800C1FA2378232B09D11A4A2B781268927C2D
:109E2800013A934202DA114A0133137023782A2B3C
:109E380004D12B7813B10D4A013B13702378532BAF
:109E48000FD117F04FF80B4B00212970DA7961F325
:109E58000002DA71FFF76CFE0B4B9A7942F00402AC
:109E68009A7100232370FEBD571E0020121E002089
:109E7800401D0020B0550020346E0208783A0020BA
:109E8800F4010020781D0020841F00202DE9F74FE1
:109E9800924E934C3378934D232B934F25D12368BF
:109EA800986843F6F123984217D1DFF86082296851
:109EB80098F8000000F56A50713007F0B9FD98F87D
:109EC8000000013000F0010088F8000000F56A5039
:109ED800713007F0B7FD286007E000B2FEF7D2FD49
:109EE80028603B7843F008033B703378532B40F0ED
:109EF8006781236849F615529B68934202D12A6804
:109F08007A4B15E04BF2B642934202D12A68784B5D
:109F18000EE04BF23342934202D12A68754B07E0B8
:109F280049F66652934204D12A68734B02B1012262
:109F38001A7023689A6843F6DD239A420AD16F4B58
:109F480029681A7861F300021A7008F0D7F808B186
:109F580008F0F2F8236843F6E0229B68934206D1A2
:109F6800664B29681A7861F3C7121A7019E043F62C
:109F7800EA22934206D1614B29685A7861F30002BC
:109F88005A700EE043F6E72293420AD129685C4BE7
:109F980019B11A6842F0005202E01A6861F35D7262
:109FA8001A6023689A684BF24C539A420AD129687E
:109FB800544B19B11A7842F0200202E01A7861F382
:109FC80045121A7023689A684BF2D9539A4202D103
:109FD800287819F097FE236843F6DA229B689342A3
:109FE80003D12A68484B1A7008E049F61E5293427A
:109FF80004D12B6813B93B4B01221A6023689A6875
:10A008004BF2DA539A420BD1404A2B6812784049F6
:10A01800032B8B5404D13F4B5A7942F010025A71EA
:10A02800236849F65E529B68934202D129683A4AEE
:10A0380005E049F66152934203D12968374A117005
:10A0480016E049F66252934203D12968344A1170E6
:10A0580015E049F66452934203D12968314A1170D8
:10A068001CE049F66552934202D12A682E4B13E050
:10A0780043F60852934202D12A682C4B0CE04AF26C
:10A088006C72934202D12A68294B05E04BF2CA420E
:10A09800934203D12A68274B1A700AE049F61652F0
:10A0A800934206D12A68244B01201A7001460EF00B
:10A0B8000BFC2368986843F6F12398423ED1DFF8F9
:10A0C8004C80296898F8000000F56A50713007F054
:10A0D800AFFC002388F8003033E000BF401D0020AB
:10A0E800781D0020201E0020571E0020AC260020CE
:10A0F800603A0020573400203E1D0020D51E002065
:10A10800783A00205C5E00203E580020071E0020A0
:10A11800A017002054260020F83D0020F63D00201E
:10A12800293D00209D3C002004200020DE15002051
:10A13800751C0020F61C0020123C002000B2FEF71F
:10A14800C7FC23689A6843F698139A4236D129685F
:10A15800DFF8A8B2DFF8D0A20BEBC1031B79DFF858
:10A16800A082C3F34113012BDFF8C09221DD98F8D8
:10A17800000000F56650203007F05AFC98F80030CF
:10A18800DAF8001009EB030211720BEBC102127925
:10A19800C2F34112032A0CD1974A12689068103012
:10A1A800C01807F045FC98F80030DAF800204B4456
:10A1B8001A7498F800302A6809F80320FFF7B8FCE9
:10A1C8003B78DFF86C8213F0010F00F0DC80216827
:10A1D80043F698128B6893427FD1884A2B68914640
:10A1E80002EBC3010979C1F34111012906DD844A53
:10A1F8001278072A02D9FEF799FCD0E03278442A6F
:10A2080036D15FFA83F82DE008F101087B4B5FFA3D
:10A2180088F803EBC8031B79C3F34113012B06DD50
:10A22800784B1B7823BB764B1B78072B20D8DFF89D
:10A23800D0A19AF800301F2B08D807F05FFF70B143
:10A2480009EBC8031B7913F0100F08D19AF80030F6
:10A258001F2B07D909EBC8031B79DB0902D0C5F806
:10A26800008005E009EBC8031B7913F0080FCBD079
:10A278003378552B40F093802E782BE0013EF6B2D0
:10A2880009EBC6031B79C3F34113012B08DD5D4BB2
:10A298001B78002B40F08380594B1B78082B7ED805
:10A2A800DFF85C8198F800301F2B08D807F026FFEC
:10A2B80070B109EBC6031B7913F0100F08D198F899
:10A2C80000301F2B06D909EBC6031B79DB0901D027
:10A2D8002E6064E0002ED1D161E04BF2DA52934255
:10A2E8000AD005DCA3F53442CA3A012A0ED803E0A5
:10A2F8004BF23762934209D133782F2B4FD9B1F9FA
:10A308001020303293424ADC303B30E043F6F122F1
:10A31800934207D13A4B1B7823B13078B5F9001036
:10A328003B222CE007F0EAFE18B3236843F6C42169
:10A338009A688A4203D047F201118A4204D13078E0
:10A34800B5F900102D221AE0A2F56A5161390529E4
:10A3580003D943F6E9218A4201D1012307E043F6F4
:10A36800E0218A4202D00A318A4203D100232B60BD
:10A3780015E023683078B5F90010B3F91020FFF71D
:10A38800F7FB28600BE02368B3F90800FEF77AFBB7
:10A39800286098F8003043F0080388F80030FFF789
:10A3A800C7FB236843F6D222986890420BD12B68EA
:10A3B80013B91548154901E0134815490222F6F763
:10A3C800BFFA0226C8E14BF2376290420AD12B68E5
:10A3D80013B91048104931E0012B0E480CBF0F4942
:10A3E8000F492BE04BF2DA52904236D12B68012B01
:10A3F80020D108480B4921E0781D002014040020D2
:10A40800071E0020820D002012020020986E02080C
:10A418009A6E020804020020DE1B0308201C0308B1
:10A42800FF1B0308B51A0308201E0020A02C0020DB
:10A43800571E0020022B05D1A548A6491022F6F781
:10A448007FFA88E1032B02D1A148A349F6E7042B40
:10A458009F480CBFA149A249F0E74BF2CA4290427B
:10A468000AD12B6813B99A489E49E7E7022B984806
:10A478000CBF9D499D49E1E74BF2CB4290420AD17E
:10A488002B6813B992489A49D8E7012B40F06381A9
:10A498008F489849D2E749F66352904203D043F671
:10A4A800EE2290420ED128680A21B0FBF1F201FB9E
:10A4B8001201914B3031D97730322E2199775A7762
:10A4C800032649E143F6F12290423ED18B4B1B789B
:10A4D800E3B9022229688A48FEF78AFA43F6F2208D
:10A4E800FEF7D0FA022201468648FEF781FA3B7849
:10A4F80013F0010F00F08081834B1B7803F0800379
:10A50800DBB2002B00F078817D4819E0FEF7BAFA3B
:10A51800022201467A48FEF76BFA02227948296836
:10A52800FEF766FA3B7813F0010F00F06581764B71
:10A538001B7803F08003DBB2002B00F05D817148CB
:10A5480020210222F5F726FF56E143F698129042A1
:10A5580040F0B5802B686D4EDFF8A08156F83310B7
:10A5680010225B48F6F7ECF90DF1060298F80000A6
:10A578000DF1070110F0F2F94246334620B3167880
:10A588006349895D03291FD0296803EBC101097953
:10A59800C1F34111012917D1072E15D95D490B22A5
:10A5A8005D48F6F7CDF95D48711C0222FEF720FAE6
:10A5B8009DF807105A4801310222FEF719FA9DF852
:10A5C80006105848013118E02E68157803EBC601CB
:10A5D800097903EBC6063679C1F34111012906F062
:10A5E8000706C8BF05F00705012E0ADC4E494A4890
:10A5F8000B22F6F7A5F94948691C0222FEF7F8F97B
:10A60800A9E0022E0BD149490B224348F6F798F9E5
:10A6180032464248691CFEF7EBF90E369CE0032EE1
:10A628000BD143490B223C48F6F78AF93B48691C91
:10A638000222FEF7DDF90D368EE0042E11D13D49D8
:10A648000B223548F6F77CF93448691C0222FEF7DC
:10A65800CFF9334805F109010222FEF7C9F90C3692
:10A668007AE0052E11D134490B222B48F6F768F908
:10A678002A48691C0222FEF7BBF9294805F109019D
:10A688000222FEF7B5F90B3666E0062E63D12B4998
:10A698000B222148F6F754F92048691C0222FEF7DC
:10A6A800A7F91F4805F109010222FEF7A1F924487C
:10A6B80005F111010222FEF79BF90A364CE0B3F9C5
:10A6C8001060092E3EDD632ECCBF032602263AE039
:10A6D80004020020D61A0308F71A0308181B0308F7
:10A6E800941A0308831C0308C51C0308A41C030848
:10A6F800071D0308281D0308F4010020071E002079
:10A708000F02002012020020783A002014040020D2
:10A71800A02C00206C360308F9010020FA01002063
:10A72800FE010020010200202A36030885350308AF
:10A7380009360308C7350308A6350308E8350308B2
:10A748000202002001262D482968801B46F080025D
:10A75800FEF74EF900E010263B7813F0010F0BD0FE
:10A76800274B1B7803F08003DBB22BB12348202151
:10A77800801B3246F5F70EFE224EB37803F0020333
:10A78800DBB2002B38D0FEF73BF81F4D034628B943
:10A798002878F11D6522FEF751F808E0B27929788A
:10A7A800B388F01D01FB023109B207F05CF9236898
:10A7B80047F201129B68934213D006DC43F6C42289
:10A7C80093420ED043F69E5209E047F2811293421B
:10A7D80007D049F61E52934203D047F241129342E2
:10A7E8000AD105200B21074AFEF794F82978074873
:10A7F80001310222FEF7FCF8BDE8FE8F14020020AA
:10A80800783A0020681E0020071E0020F50100206D
:10A81800F0B5114B1F78114B303F1E680DE0D6F88C
:10A8280014C01CF803C00133644501D112E00023B1
:10A83800DAB28242F3D301350D70094B0622094979
:10A8480002FB07330D785B1993F86840002CEED1B2
:10A858000C70F9321046F0BD401D0020781D002014
:10A86800346E0208861D00202DE9F74F974C984E4C
:10A8780023689A6843F609539A4203D133780BB98F
:10A88800013333702368934F9968B3F910303A78DD
:10A89800B3F1010848BF03F106084FEAE808337826
:10A8A80008F1010812F0010F03FB08188A4D00F0A7
:10A8B800AD808A4B1A789946432A4DD128780FFAE9
:10A8C80088FA0AEBD00007F0BDF82268844B91683B
:10A8D80046F2C8629142186001D12A783AB12A78C2
:10A8E800012102F0070211FA02F25040186028789C
:10A8F80019780AEBD00007F09BF8236847F2E112B9
:10A908009B68934209D1744B1A78764B03EBD203B8
:10A91800734A126883F8A0211EE046F6A9329342D2
:10A9280005D13178002001310EF02AFB14E046F2FF
:10A93800BF7A4FF0000B23689B68534504D1012070
:10A948000BEB00010EF01CFB0AF1080A46F2DF735C
:10A958009A450BF1010BEED199F80030232B10D159
:10A9680022682B78927C013A93420ADA5A4A0133D8
:10A9780013705D4B9B7803F00203DBB20BB1FDF75C
:10A988000DFF99F800302A2B0CD12B7853B1524A7D
:10A99800013B1370544B9B7803F00203DBB20BB1FD
:10A9A800FDF7FCFE99F80030552B14D12368997CEB
:10A9B8000F2910D92A7808398A42474B01DA083218
:10A9C80000E000221A70484B9B7803F00203DBB2C8
:10A9D8000BB1FDF7E3FE99F80030442B42D1236810
:10A9E8009A7C0F2A3ED929783B4B072902D9083986
:10A9F800197001E0083A1A703B4B9B7803F0020388
:10AA0800DBB2002B2ED0FDF7C9FE2BE049F6D5436B
:10AA180099420ED1314B1B78A3F13101C9B20329F8
:10AA280007D842F006023A7007225343284A573B98
:10AA3800137023689A6843F609539A4212D13378FF
:10AA48001B2B08D9284B46F695429A809A7842F0F3
:10AA580002029A7006E05901C918244B0020C9184F
:10AA6800FDF7A0FFFFF764F8214A2B781178934689
:10AA7800994288BF137012780F32934202DD1C4A44
:10AA88000F3B137023684FF0000A93F81290B9F146
:10AA98000F0F9ABFC9F120095FFA89F94FF0100921
:10AAA8009BF800004FFA8AF318180FFA88F202EBA5
:10AAB800E000019306F0C6FF9BF80020019B5FFAB7
:10AAC80080FC9B1803F007032BE000BF781D0020D3
:10AAD800071E0020571E0020121E0020401D0020C7
:10AAE800201E0020A02C0020681E0020381F03080C
:10AAF800091E00204CFA03F06549013300F00100FB
:10AB080000280CBFA520DB20DBB201F809000AF100
:10AB1800010A09F10109082B5FFA8AFA5FFA89F933
:10AB280003D0B9F1200FE5D109E0B9F1200F06D023
:10AB380023684FFA8AF19B7C89189942B0DB3B78ED
:10AB480013F0010F15D0236852499B7C09780F2B0D
:10AB580001F0800198BFC3F11003C9B294BFDBB202
:10AB6800002331B1297810318A1A4949CB185F215D
:10AB78009954DFF8288198F80230474603F0020319
:10AB8800DBB2002B64D0FDF73BFE034600BB226816
:10AB980046F6A93192688A4206D024318A4203D007
:10ABA80043F6E5118A4204D130783B4965220023F7
:10ABB80009E043F609518A4208D130781C38C0B2FE
:10ABC80008F107016522FDF739FE18E02878F7E754
:10ABD800236846F669329B68934203D043F6FC2209
:10ABE800934202D1BA79317801E0BA792978BB88E1
:10ABF800294801FB0231BA7909B206F034FF23680B
:10AC08009A7C102A02D905200B211EE09B6846F683
:10AC1800693293420ED006DC43F6E512934209D01E
:10AC280043F6FC2204E046F6A932934202D02432CD
:10AC3800934201D1102007E043F60952934202D112
:10AC48000020102101E000200721144AFDF762FED0
:10AC5800226846F60D4193688B4216D046F6C72106
:10AC68008B4212D043F6ED218B4202D1084BDB21F7
:10AC78009977937C102B08D9297809480131022249
:10AC880003B0BDE8F04FFDF7B3BE03B0BDE8F08FE9
:10AC9800F4010020783A00206F1E0020681E002072
:10ACA800F5010020114B002270B50D461A7118B13C
:10ACB8001B7803B920234370BDB10D48F5F7BAFDE1
:10ACC8000446681C5CB10A492246F5F7BBFA022C17
:10ACD8000BDC601C28182021C4F1030201E02021AC
:10ACE8000322BDE87040F5F755BB70BDF41D002088
:10ACF800F51D002038B50546002408E0601906F067
:10AD0800A1FE3038C0B2092808D80134E4B2044B97
:10AD18001B78303B9C42F1DB012038BD002038BD58
:10AD28005C1D002008B506F08DFE0023C0B2064A5F
:10AD3800D25C824201D1202804D10133082BF6D1FC
:10AD4800002008BD012008BDD86E020870B506466F
:10AD58000D4600240DB12D232B55A01900210134D7
:10AD680006F066FE062CF5D170BD00002DE9F04F07
:10AD7800974C984F206839788368068A9AB201FB05
:10AD880006260D4648F63C118B4287B0B6B20BD169
:10AD9800914B1A785B7802F00702C3F3420303EB86
:10ADA800C20306EBC3062BE048F6FC218B4212D106
:10ADB800894B8A481A78597802F0070288235A433F
:10ADC800C1F34201773B03FB012320210822F61837
:10ADD800F5F7E0FA14E048F6B4618B420BD17E4BEC
:10ADE8001A785B7802F00702C3F3420303EBC2034D
:10ADF8009B01F61804E0B3F5E97F08BF02EB4506AE
:10AE0800774B784D1A78984612F0010F53D1236882
:10AE18009A6847F209039A4204D046F609639A42AF
:10AE280040F04481704B1B782A2B3BD16F4B93F831
:10AE3800009009F1010909F0010983F80090B9F1BE
:10AE4800000F1AD046F609639A4208D1684B46F6B5
:10AE580095429A809A7842F002029A7026E120215F
:10AE680010226448F5F796FA3B7800205901C91872
:10AE7800614BC918FDF796FD18E15D48FDF738FDEF
:10AE8800236848469A6846F609639A420CBF5B49AC
:10AE98005B49FDF787FD39785A4801310222FDF7F1
:10AEA800A7FD03E1552B02D0442B40F0FF804F4B08
:10AEB80000221A70FAE023685869F5F7BBFC4A4B80
:10AEC800834693F800A09946BAF1450F02D14E4B3C
:10AED80000221A705046FDF721FE00284DD04B4B3A
:10AEE8005FFA8BFB1A7852450ED15846FFF790FC53
:10AEF800FF2804D15846FFF78BFCFF283DD0444B70
:10AF08001A7801321A7015E0DFF804A100228AF8D5
:10AF1800002058460593FFF77BFCFF28059B04D0CB
:10AF28009AF8002001328AF8002099F80020FF28BA
:10AF38001A7022D02168374A4B6910601B5C8868F8
:10AF480047F209018842136092460FD1562B01D06F
:10AF5800542B0BD13B78123BDBB2022B06D82B7853
:10AF680030B2C01806F06EFDCAF800002B7830B277
:10AF7800C018DAF8001006F05BFD99F80030552B80
:10AF880017D12368997C0F2913D92A7808398A425E
:10AF9800144B01DA083200E000221A70144B9B7837
:10AFA80003F00203DBB20BB1FDF7F8FB184B0022EC
:10AFB8001A7099F80030442B3BD123689A7C0F2AE9
:10AFC80037D92978074B072926D90839197025E078
:10AFD800781D0020071E00200D1E002004020020FE
:10AFE800571E0020121E0020401D0020621E002057
:10AFF800681E0020F40100205B1703086C15030885
:10B00800AE150308F5010020581D00205A1D002028
:10B01800861D0020201E0020083A1A70964B9B7847
:10B0280003F00203DBB20BB1FDF7B8FB934B002230
:10B038001A7099F80030432B0CD1236830B25B6941
:10B0480019788F4B19602B78C01806F0F1FC8B4BE0
:10B0580000221A7099F80030232B13D122682B781C
:10B06800927C013A93420DDA864A01331370834B7E
:10B0780000221A70804B9B7803F00203DBB20BB1FD
:10B08800FDF78CFB99F800302A2B0FD12B786BB188
:10B098007C4A013B1370794B00221A70764B9B78DF
:10B0A80003F00203DBB20BB1FDF778FBFEF740FDBE
:10B0B800754A2B7811789246994288BF1370127896
:10B0C8000F32934202DD704A0F3B137023684FF032
:10B0D800000B93F81290B9F10F0F9ABFC9F120092C
:10B0E8005FFA89F94FF010099AF8000033B218187E
:10B0F8005844059306F0A6FC644A02F8090009F1D1
:10B1080001095FFA89F9B9F11F0F059B05D8216874
:10B118000BF1010B897C8B45E6DB98F8001011F0E8
:10B12800010F16D021685A48897C00780F2900F051
:10B13800800098BFC1F11001C0B294BFC9B200210C
:10B1480038B128789AF8006010305218801B5F21B7
:10B158001154226890684AF26A7290420AD14D4BA3
:10B168001B78532B2FD106F06DFC4B4B187006F053
:10B1780063FD28E0B0F5E97F25D1464A1278532AC5
:10B1880021D11846FFF7CEFD0646E0B93B78DA0034
:10B19800D31A03F11200FFF7ADFD60B1FF2300934E
:10B1A8003E4B01961B7879200133029331460422E5
:10B1B800334606F0C5FC3B780021DA00D31A03F1C8
:10B1C8001200FFF7C3FD2C4EB37803F00203DBB285
:10B1D800002B6ED0FDF714FB034680B9226848F6B1
:10B1E800B46192688A420AD046F609618A4214BF5D
:10B1F80028783878F11D6522FDF720FB0FE02368D9
:10B20800B2799B682648B3F5E97F0CBF397829786D
:10B21800B38801FB0231B27909B206F024FC236835
:10B228009A7C032A08D99A6848F63C118A4203D0C6
:10B2380046F609618A4214D19B6848F63C1293424B
:10B248000CD198F8003013F0010F01D010202CE039
:10B25800202107221348F5F79DF82AE0B3F5E97F86
:10B2680002D105200B2121E046F6096293421BD149
:10B27800002010211AE000BF681E0020861D002053
:10B28800201E0020121E0020091E0020F4010020AC
:10B29800783A0020401D00205C1D0020071E002079
:10B2A8006F1E00200402002000200721104AFDF72D
:10B2B80031FB23689A7C032A16D9B27802F002027D
:10B2C800D2B28AB19B6848F63C1293420CD046F63B
:10B2D8000962934208D0297806480131022207B052
:10B2E800BDE8F04FFDF784BB07B0BDE8F08F00BFA5
:10B2F800681E0020F50100202DE9F04F794E8BB033
:10B3080033689D6893F81290122D01D00B2D09D146
:10B31800754A122D92F80090A9F130095FFA89F95F
:10B3280015D01DE04BF2E7539D4203D028339D42D0
:10B3380040F053836D482821F5F7AAF88046002885
:10B3480000F04E8301302821F5F7A2F848E39F7BEF
:10B3580037B9674BB846D879FEF7F4FB044615E0D1
:10B368000027B846FF20FEF7EDFB4BF2D8339D428D
:10B3780004460BD14BF2B74006F064FBC0B209900B
:10B3880020B15B4B9B790BB1FDF7D0FB3368594D6E
:10B398009A68122A1AD19B7BC3B12B7813F0010F3C
:10B3A80008D12046FFF7A6FC534B10B101221A70B2
:10B3B80000E018704E4B9B7943B12046FFF79AFC8A
:10B3C80020B14D4B1B780BB1FDF7B0FB2978DFF8A6
:10B3D80044A111F0010100F087819AF80030DFF8EC
:10B3E80038B118460793FDF799FB079B002800F032
:10B3F800B5804249002008704148424A90F800C090
:10B4080013609C45404940F0898033689B8903F06C
:10B418000F03032B1ED13D4BACF1300C18784FF0C5
:10B428000A0E05903A480EFB0C00DDF814E000EB1C
:10B438000E0C0EF1010E5FFA8EFE70449CF8ADC042
:10B4480090F8AD00C2F800C083F800E0002872D17F
:10B45800187070E0082B2CD12C4BACF130001B7805
:10B4680000EB800C0CEB030E294BDFF8A0C013F89F
:10B478000E3008930BB98CF800309CF800E000EB14
:10B488008000059070440EF1010E5FFA8EFE8CF874
:10B4980000E01F4BDDF814C01B5C08900CEB0E009D
:10B4A800DFF86CE013601EF80030002B43D117481A
:10B4B80011E0072B11D1BCF1300F10D113480378DC
:10B4C80023B14FF02B0EC2F800E001E0C2F800C033
:10B4D800013303F0010303702DE0062B2BD10B7809
:10B4E800013327E0781D00205C1D002004020020A5
:10B4F800161E0020571E0020671300204358002006
:10B508005A1D0020201E0020121E0020861D00202B
:10B51800346E0208401D00205D1D0020DFF898E20F
:10B5280003709BF800304FF0010C8EF800C013B187
:10B538000B7863440B7040238BF800300B784B4535
:10B5480003D39B4B09F1FF30187008781168201855
:10B5580006F06EFA2B7843F004032B709AF800304B
:10B56800232B2FD1924B09F1FF311A788A4229DA1D
:10B5780072B932684BF2E75192688A4208D0283192
:10B588008A4205D02046079306F05CFA079BC8B1AB
:10B5980018780130C0B21870201806F053FA28B98C
:10B5A800834B20211878201806F042FA814B40225C
:10B5B8001A702B78804A43F004032B7000238BF811
:10B5C800003013709AF800302A2B10D1784B1A7873
:10B5D8006AB1013A1A70774B40221A702B78764A72
:10B5E80043F004032B7000238BF8003013709AF893
:10B5F8000030432B1FD16E4B1878484505D22018D0
:10B608002021079306F014FA079B9BF800203AB90B
:10B618001B7809F1FF32934202DA654A013313704D
:10B628002B78644A43F004032B7000231370624A9A
:10B638008BF8003013709BF8003013B15F4A013B60
:10B6480013709BF80030012B0ED1594B1A784A45DC
:10B6580001D201321A70584A002313702A7842F036
:10B6680004022A708BF800302B7803F00402D2B25F
:10B67800002A71D0524A6FF38203137000211122FD
:10B688005048F4F787FE504A494B11781B78994285
:10B6980088BF137011780F318B4202DD4A490F3B86
:10B6A8000B70117847481022611806F0DCF94548FC
:10B6B800F5F7C0F833684BF2E7519B68C2B28B428A
:10B6C80002D028318B4205D122B94048F5F7B2F8AB
:10B6D800421CD2B20F2A3FD83A4820218018C2F122
:10B6E8001002F4F757FE37E0DFF8D8B011225846B9
:10B6F800F4F750FE33684BF2E7529B68934202D04E
:10B708002832934209D1214604222E4806F0ABF98B
:10B7180040463946FFF7C6FA1EE021461022584631
:10B7280006F0A1F95846F5F785F802462021C2F13E
:10B7380010025844F4F72EFE21464A46244806F0E3
:10B7480092F9244A1020937882F8069043F0020375
:10B7580093700146FDF7DEF89AF80030532B75D147
:10B7680033689A684BF2D8339A4208D1204606F0DB
:10B7780069F920B14BF2B740012106F059F9336855
:10B78800DFF838A09B68122B40D12046FFF7B2FAA9
:10B798008346002830D0104BFF2219780F4BF9B997
:10B7A800009201911B78782001330293FB3A1FE045
:10B7B800121E002043580020861D00205D1D002019
:10B7C800571E0020F41D0020091E0020F51D002032
:10B7D8008F1D0020881D002067130020071E0020F1
:10B7E8000021009201911B787A20013302930422F0
:10B7F8000B4606F0A5F909E08AF800007D492046C5
:10B80800FFF7A4FA7C4B83F800B0EFE020464946E6
:10B81800FDF7D6F8794B0020187033688AF80000D5
:10B828009B684AF27E72934202D10090013005E093
:10B838004BF2FA32934206D10123009301460246A5
:10B8480003460DF0C9FB6E48FDF752F8FEF770F994
:10B858002B7813F0010F17D033684BF2E7529B682F
:10B86800934202D02832934204D140463946FFF72A
:10B8780019FA09E05F4B634A03F1100153F8040B0E
:10B888008B4242F8040BF9D133689A68122A1ED108
:10B898009B7BE3B12046FFF72DFAC0B12B7813F05C
:10B8A800010F14D1584B9A7922B9DA79574B1B7882
:10B8B8009A420CD0564B1A780023303A05E0554985
:10B8C8002A20C91801330874DBB29342F7DB3268C7
:10B8D80093680B2B01D0122B0AD14A4B991D13F8F0
:10B8E800010B202802D10D3003F8010C8B42F6D150
:10B8F80092684BF2D8339A4214D1434B9B798BB15F
:10B90800099878B14FF0000909EB040006F09AF89D
:10B9180018B1404B2A224B441A7409F10109B9F1B4
:10B92800100FF1D12B7813F0010F25D03A4B1B786B
:10B9380003F08003DBB2FBB133689A684BF2E7533C
:10B948009A422D4B03D04BF20F618A420CD11B78DF
:10B9580033B9B8F1000F0FD05F3388F801300BE02E
:10B9680057B15F22FA5407E0244A1B781278103343
:10B978009B1A284A5F21D154284CA37803F002036C
:10B98800DBB2002B32D0FCF73BFF2049034628B935
:10B9980008786522E11DFCF751FF12E03068B4F920
:10B9A8000430A27984680978122C01FB023105D190
:10B9B800807B18B91449C97902FB0131184806F08F
:10B9C80052F833689B68122B10D10820134A01469D
:10B9D8000BB0BDE8F04FFCF79DBF0027B84600E06C
:10B9E800074609F1FF395FFA89F9BBE40BB0BDE8F6
:10B9F800F08F00BFF41D0020121E0020091E002039
:10BA0800881D002004020020161E0020071E0020AA
:10BA18005C1D0020F4010020783A0020681E0020F8
:10BA28006F1E002024282DE9F041144626D16B4BC7
:10BA380043F63C321B686A4D9B686A4E934206D1B6
:10BA48002B7813F0010F0ED02438674909E04BF228
:10BA58000F6293420AD12B7813F0010F03D0634988
:10BA68000020FCF79FFF2978490800E02978301961
:10BA780001310222FCF7BCFF0234AAE0E72809D111
:10BA8800574B58481978801801310322FCF7B0FF4A
:10BA980003349EE0A3282AD1514D2B783F2B15D88B
:10BAA80010465349FCF77EFF5148F4F7C3FE2A219C
:10BAB80024184C48E4B2F4F7EBFC002800F08A8024
:10BAC800297802220131FCF793FF83E05901494D9F
:10BAD800C918691801F582411046DF31FCF762FF89
:10BAE80005F59240FE30F4F7A5FE241871E0F2281F
:10BAF80021D13B4F3B4D3978072605EB0208B1FBB6
:10BB0800F6F1404601310222FCF772FF39782D2305
:10BB1800B1FBF6F688F80230F3009E1B8B1B364FFC
:10BB2800DBB207EB83031988E21CA9529B78A8189B
:10BB3800837006344DE025280BD1304B46F69542EC
:10BB48009A8045229A719A78053842F002029A70D2
:10BB58003CE05E280BD1294B46F695529A80452247
:10BB68009A719A783E3842F002029A702EE07C2848
:10BB78000BD1224B46F248129A8011229A719A7878
:10BB88005C3842F002029A7020E0EC280BD11B4B83
:10BB980046F6D9529A8045229A719A78CC3842F062
:10BBA80002029A7012E0A7280BD1144B46F6F952FC
:10BBB8009A8045229A719A78873842F002029A70E0
:10BBC80004E0E02801D1541C03E018B1054B1855D6
:10BBD8000134E4B22046BDE8F08100BF781D0020A2
:10BBE800071E0020F4010020C00F03087E0F030881
:10BBF8003A1703083CCD0208B5F90208681E002070
:10BC080038B50A4B46F68A451B78002405FB030520
:10BC180007E0074B22461978FFF704FF041B2D198C
:10BC28000446287808B11F2CF3D938BD5B1D0020C5
:10BC3800071E002070B5002543F62064204605F055
:10BC480001FF064604F1080005F0FCFE16F0FF0FA0
:10BC580006D020F07F0010F0FF0F01D00135ADB203
:10BC680046F23F139C4201D00934E7E7284670BDED
:10BC780038B5B0F900500B4C05EBC50505F57855FE
:10BC88002835284605F0DEFEC1B211F0800F07D036
:10BC980023882846013B01F07F01238005F0C8FE78
:10BCA800208838BD561D0020454B2DE9F74F1B88CD
:10BCB800444A044689461788DFF80C8123B14FF0BF
:10BCC800000A0AE09A4608E00529FBD198F80030F6
:10BCD80043F0040388F8003070E098F8003013F05F
:10BCE800030F0BD013F0010F02D0B4F1FF3F05D1C1
:10BCF80003F00203DBB21BB1012C01D03F19BFB224
:10BD08003BB2B3F1FF3F04D0B3F57A7F08BF0027F9
:10BD180001E040F2E7370FFA87FB0BEBCB0303F5A3
:10BD2800785303F12000019305F08CFE10F0FF0F0B
:10BD3800019B16D0B9F1050F09D103F1280005F0D0
:10BD480081FE20F07F0010F0FF0FC6D022E0B9F18D
:10BD5800000F1FD003F1280005F074FE00F07F06E5
:10BD680018E00AF1010AB4F1FF3F1FFA8AFA04D178
:10BD780098F8003043F0010305E0012C05D198F84C
:10BD8800003043F0020388F80030BAF57A7F0DD00E
:10BD98003D46A2E74E4505D0B9F1000F02D0B9F1F2
:10BDA800050F9AD1BAF1000F05D000E03D46054ACB
:10BDB8002DB2156002E0034BC3F800B0BDE8FE8F5A
:10BDC800561D0020201E0020241E0020F0B50378F8
:10BDD8009BB05A1ED2B2792A0F4600F2C8805E0183
:10BDE800644AF3189B18644A46F68A4612784578DE
:10BDF80006FB0236E7213046F4F74AFB0446F0B961
:10BE080030467C21F4F744FB0446C0B9304625216E
:10BE1800F4F73EFB044690B930462421F4F738FB8A
:10BE2800044660B930464021F4F732FB044630B985
:10BE38003046F921F4F72CFB0446002876D0A41BE1
:10BE48000FB14E4800E04E4831462246A619F4F795
:10BE580077FD3046E721F4F71BFB30B128466946E9
:10BE6800652246F6D953FCF7E9FC30467C21F4F705
:10BE78000FFB50B1691EC9B201EB011101F5C241B6
:10BE880068464831112205F0EEFD30462521F4F7C9
:10BE9800FFFA38B1681EC0B26946652246F6954376
:10BEA800FCF7CCFC3046F921F4F7F2FA38B1681EF9
:10BEB800C0B26946652246F69553FCF7BFFC30468A
:10BEC8004021F4F7E5FA50B1691EC9B201EB01113E
:10BED80001F5E84168463B31112205F0C4FD3046C2
:10BEE8002421F4F7D5FA50B10FB1244800E02448D2
:10BEF800001929460222FCF77BFD02340BE00FB142
:10BF08001E4800E01E4800196946F4F735FC6846EB
:10BF1800F4F790FC0419002F29D01A4A93781419C1
:10BF280043F0020393700023E37116E03046F4F700
:10BF380081FC05461FB9124831462A4615E01028EB
:10BF480010DD2A460D483146F4F7FAFC0D4A93787D
:10BF5800551943F002039370EC7110200146FCF769
:10BF6800D9FC04E0084831461022F4F7E9FC1BB07C
:10BF7800F0BD00BF1FFF02085B1D00206F1E0020E0
:10BF8800EE320020681E0020040200200C4B1B78B3
:10BF980013F0010202D000200A4905E003F0020074
:10BFA800C0B218B108491046FCF7FCBC03F0040302
:10BFB800DBB20BB10549F7E705480121FFF706BFDA
:10BFC800241E0020F8D40208D7D4020819D5020884
:10BFD800591E002070B5124D124C00201249FCF772
:10BFE800F1FB2846A1780222FCF702FDE81CE17863
:10BFF8000222FCF7FDFC05F1080021790222FCF77A
:10C00800F7FC05F10B0061790222FCF7F1FCA1793C
:10C0180005F10E000222BDE87040FCF7E9BC00BF44
:10C02800F4010020591E0020456F02082DE9F34154
:10C03800504F514C3B689D7C237813F0010F2FD152
:10C04800022243F61E610DF1060005F00CFD4B4E71
:10C05800BDF806304FF0FF3033602946FFF724FE65
:10C06800237843F001032370454B1B7813F0030F2B
:10C0780014D1B6F90010434801EBC10101F578511C
:10C088002031092205F0EFFC3F4B1B881BB13046DD
:10C09800FFF7EEFD10B90020FAF77AF8FFF79AFFDC
:10C0A8003A4E3378552B0DD1DFF8D4803848FCF759
:10C0B8001FFC98F800304FF0FF306FF3410388F809
:10C0C80000300DE0442B2BD1DFF8B4803048FCF76A
:10C0D8000FFC98F8003001206FF3000388F8003057
:10C0E8002946FFF7E1FD98F8003013F0030F15D14A
:10C0F800224D2448B5F90010092201EBC10101F5D0
:10C108007851203105F0AFFC1F4B1B881BB1284626
:10C11800FFF7AEFD10B90020FAF73AF8FFF75AFF1B
:10C12800FFF734FF3378232B22D1154B184E1A789A
:10C1380002F0FC026FF382021A70FCF7F7FCB37886
:10C148006FF34103B370134B1D7835B9FCF726FB29
:10C158003046FCF7CDFB3D600AE02278013DEDB2A8
:10C1680042F0060222701D700B4B53F825303B60DD
:10C17800BDE8FC81781D0020571E0020201E0020ED
:10C18800241E0020591E0020561D0020401D00209E
:10C19800681E0020371E0020441E00202DE9F041B3
:10C1A8001646104A0F4653780E21C3F342034B43F9
:10C1B800117803F50843CC330B4D01F00701044611
:10C1C80003EB4101022205F04EFCE8192178022216
:10C1D800FCF70EFC6178A8190222BDE8F041FCF7D3
:10C1E80007BC00BF0D1E0020F4010020044B0222F2
:10C1F8005978044BC1F3420118180131FCF7F8BB18
:10C208000D1E0020F401002010B5074B074C1B78C9
:10C21800074A03F0070304EB83031C881118145220
:10C228009B788B7010BD00BF0D1E0020B5F9020869
:10C23800F4010020084B1B789B0902D0012B06D182
:10C2480002E01020054904E01020054901E00549F5
:10C258001020FCF7A7BB00BF0D1E00209AE10208C2
:10C26800BBE10208DCE102082DE9F041DFF8688053
:10C278000F4698F80010174DC1F382010446164680
:10C2880005F1080001310222FCF7B2FB98F8001012
:10C29800042201F01C0101F51C41B431204605F0CF
:10C2A800E2FBE81921780222FCF7A2FBF81C281807
:10C2B80061780222FCF79CFBA819A1780222FCF7FE
:10C2C80097FBF01CE17828180222BDE8F041FCF742
:10C2D8008FBB00BFF4010020591D0020064B1B78BE
:10C2E80003F08003DBB233B1435C04482021C0185B
:10C2F8000222F4F74FB87047783A0020F401002082
:10C308002DE9F743654D664C2B6821789B6802221E
:10C3180003EB41010DF1060005F0A5FB2B68A946CA
:10C328009A6843F6F4239A4208D100205D49FCF745
:10C3380039FBBDF806804FF4B46303E0BDF806800E
:10C348004FF46163B8FBF3F103FB11883C221FFA39
:10C3580088F8B8FBF2F302FB1388CFB2DEB20222F0
:10C3680051483946FCF744FB5FFA88F802224F48E7
:10C378003146FCF73DFB02224D484146FCF738FBAD
:10C388004C4B1B7813F0010F6ED04B4B4B4D18786C
:10C39800232804D12B78012B62D8013305E02A2801
:10C3A80005D12B78002B5BD0013B2B7058E0A0F116
:10C3B8003003DBB2092B01D943284BD12B7873B951
:10C3C800D9F8003039B29A6843F6F4239A4201D179
:10C3D8000A2200E01122FDF7CBFBC7B216E0012BC1
:10C3E8000ED1D9F8003031B29A6843F6F4239A4254
:10C3F80001D1172200E03B22FDF7BAFBC6B205E0E7
:10C4080041463B22FDF7B4FB5FFA80F8D9F80030CB
:10C418009A6843F6F4239A4209D13C235E434FF4C9
:10C42800B46303FB0767B844ADF8068006E03846F6
:10C43800314642460FF0B3FEADF80600D9F8003099
:10C4480020789B680DF1060103EB4000022205F0FD
:10C4580004FB05E0532803D100232B70FDF768FB8C
:10C4680017482978FFF73AFFD9F800309A6843F659
:10C47800F4239A4210D02078124965220023FCF751
:10C48800DDF905200B21104AFCF744FA21780F4802
:10C4980001310222FCF7ACFABDE8FE83781D0020CA
:10C4A800071E0020BF130308040200200A02002010
:10C4B80012020020571E0020401D0020121E0020DE
:10C4C800566F02086F1E0020681E0020F50100202C
:10C4D80073B59A4B9A4D1A7812F0010F05D12A7844
:10C4E80012F0380204BF2A706A701A78934E42F02C
:10C4F80001021A702B78924C13F038023ED1914900
:10C508000978552904D113F0070F2FD0DA1D0AE056
:10C5180044290CD103F0070201323D3992FBF1F1B5
:10C52800C800411A521A62F3020323701EE053290D
:10C538000AD1C3F3C201013161F3C50323706378E3
:10C5480062F34303637011E023290FD1FCF7EEFA7D
:10C5580033787D4A43F0060333701378013BDBB22E
:10C5680013707A4A52F82320794B1A6000207949CF
:10C57800FCF718FA1C20FFF747FEDDE0082A2ED149
:10C5880075490020FCF70EFA0620FFF72FFE0C2055
:10C59800FFF73AFE1521182201A8FFF7FFFD694BA6
:10C5A8001B78552B06D1637803F0FE03C3F34202D0
:10C5B800013A07E0442B0BD1637803F0FE03C3F381
:10C5C8004202013202F0030262F343036370B3E0F4
:10C5D800532B28D0232B40F0AF802378A6E0102AD5
:10C5E80051D15D490020FCF7DDF90620FFF7FEFD7B
:10C5F8000C20FFF709FE1521182201A8FFF7CEFD30
:10C608006178564801F00101FFF768FE4D4B187834
:10C61800232801D02A2804D16378DA4362F300037F
:10C62800D4E7532804D12378C3F3C202013280E04F
:10C63800A0F13003DBB2092B01D943287CD16B78F8
:10C6480002AA03F001033B21D41883F001024B43F3
:10C65800172606FB023214F8041CFDF789FA04F8C1
:10C66800040C6B780E22C3F342035343287803F576
:10C678000843CC3300F0070003EB400001A90C3A53
:10C6880005F0EBF958E0182A4DD133490020FCF7A2
:10C6980089F90620FFF7AAFD0C20FFF7B5FDFFF783
:10C6A800C9FD284B1B78552B07D1237813F0C00FF1
:10C6B80042D0C3F38112013A06E0442B07D1237814
:10C6C8009A09012A38DC013262F3871333E0232BFD
:10C6D80004D12378C3F3C202023A2AE0532B2BD1A8
:10C6E800FCF724FA33781E4A43F006033370164BDE
:10C6F8001648197840F82120013119702378C3F3BE
:10C70800C201013161F3C503C3F381112370104BDA
:10C7180011B1012904D101E01C3202E0114A00E004
:10C72800114A1A6008E0114A00211170C3F3C202CD
:10C73800013A62F3C50323707CBD00BF571E002079
:10C748000D1E0020401D0020371E0020441E002022
:10C75800781D002058E1020879E10208596F0208A3
:10C768005C6F0208946F0208B06F0208121E002066
:10C7780073B5494B494D1A7812F0010F04D12A7844
:10C7880012F0030208BF2A701A78434E42F00102E1
:10C798001A702B78414C13F003022ED1404A1278BC
:10C7A800552A03D1C3F38202013A04E0442A06D190
:10C7B800C3F38202013262F38403237017E0532A21
:10C7C80003D15A1C62F30103F7E7232A0FD1FCF7C0
:10C7D800ADF93378334A43F0060333701378013BDD
:10C7E800DBB21370304A52F82320304B1A6001A88C
:10C7F80010211B22FFF738FD4CE0012A4AD101A87D
:10C8080010211A32FFF730FD254B1878232804D160
:10C818002378C3F34112013205E02A2807D123788F
:10C82800C3F34112013A62F3461323702CE05328F4
:10C8380004D12378DA1C62F30103F6E7A0F1300390
:10C84800DBB2092B01D943281ED12B7802AAC3F3E6
:10C858004113D4180C215A1C03F001034B4302F076
:10C8680001021F2614F8041C06FB0232FDF780F9AA
:10C8780004F8040C287801A900F01C0000F51C40FD
:10C88800B430042205F0E9F829780948C1F34111C8
:10C89800FFF724FD7CBD00BF571E0020591D002056
:10C8A800401D0020371E0020441E0020781D002057
:10C8B800CC6F0208064B1B7803F08003DBB233B160
:10C8C800435C04482021C0180322F3F763BD704776
:10C8D800783A0020F40100204328F8B504460D46B4
:10C8E800174606D1104B00261A786FF3C3021A7048
:10C8F80000E00E462046FCF711F990B10A4B303C97
:10C908001A780A2602F00801C9B2002918BF0025C2
:10C9180006FB05466FF3C30236B21A70BE42A8BFC3
:10C928003E4630B2F8BD00BF571E00202DE9F34146
:10C938006E4F6F4E3B7843F001033B70347844B937
:10C948004BF22F4005F07EF86A4B6B491860204681
:10C9580017E0012C02D10020684912E0022C02D114
:10C96800002067490DE0032C02D10020654908E04A
:10C97800042C02D10020644903E0052C03D163494B
:10C988000020FCF70FF83178D9B9614B1B78312BAF
:10C9980001D1013101E0302B05D1564B4BF22F402C
:10C9A800196005F045F85B4B1A785B4B02F0800282
:10C9B800D2B20AB1202202E04E4A12683032DA7747
:10C9C8006EE001290BD002290CD003290DD00429CF
:10C9D8000ED04BF22B45052918BF00250AE04BF273
:10C9E8001B4507E04BF21F4504E04BF2234501E0ED
:10C9F8004BF227452946042201A805F034F8474B95
:10CA0800474A03F1100153F8040B8B4242F8040B18
:10CA1800F9D1032243489DF80410FBF7E9FF0322EC
:10CA280041489DF80510FBF7E3FF03223F489DF8B6
:10CA38000610FBF7DDFF3E4803229DF80710FBF7C1
:10CA4800D7FF334B3B4C1878232804D12378022B8B
:10CA580022D8013304E02A2804D12378E3B1013B2A
:10CA6800237019E0A0F13003DBB2092B01D9432868
:10CA780012D194F8008002AA904418F8041CFF22EE
:10CA8800FFF72AFF08F8040C207802AA131813F8F5
:10CA9800041C281804F0CCFF27482178FFF70AFF68
:10CAA8001B4B1B78532B1FD1224B00221A70337853
:10CAB8000133DBB2062B337004D0012B14D10D4B9C
:10CAC8001B688BB1FDF734F8002333703B781B4AA1
:10CAD80043F006033B701378013BDBB21370184A2E
:10CAE80052F82320174B1A60BDE8FC81571E00201E
:10CAF800071E0020201E0020452D03086E2E030867
:10CB08008F2E0308B02E0308D12E0308F22E030837
:10CB1800401D0020783A0020F4010020D455030875
:10CB28000402002005020020090200200D02002056
:10CB380011020020121E0020D06F0208371E0020AC
:10CB4800441E0020781D002070B5174C0D4606467F
:10CB5800002120464FF4C172F3F71CFCFF2D0AD1C7
:10CB6800B10001F5D84120469531042204F07BFF3D
:10CB780023789BB970BDFE2D01D1173E02E0FD2D33
:10CB880002D10136267009E0B60006F5D840953086
:10CB9800401904F057FFC0B2207020B10248BDE828
:10CBA800704018F0FDBB70BD7C2000202DE9F041DD
:10CBB80018F028FC60B110208F49FBF7F3FE8F4B6B
:10CBC8001B78432B40F0EF81BDE8F04118F03CBCE6
:10CBD80018F02AFC002826D0894C23786BB1102045
:10CBE8008849FBF7DFFE88482D211030F3F750FC09
:10CBF800002800F0D881217810E010208349FBF745
:10CC0800D1FE81482D211030F3F742FC044600285C
:10CC180000F0C98118F020FC014620468222BDE8B8
:10CC2800F041FBF7E5BE7A4C43F6CC2223689B68BB
:10CC3800934250D0774E744D307803EB800004F067
:10CC480001FF032201467448FBF7D2FE2368986867
:10CC580046F6F95398422BD0203B984228D0337897
:10CC6800013000EB830004F0EDFE0322014605F1DC
:10CC78001500FBF7BDFE236830789B68023303EB91
:10CC8800800004F0DFFE0322014605F11900FBF7DE
:10CC9800AFFE236830789B68033303EB800004F011
:10CCA800D1FE0322014605F11D00FBF7A1FE0EE0AF
:10CCB8002D2103225948F3F76DFB2D2103225848F3
:10CCC800F3F768FB57482D210322F3F763FB202372
:10CCD8002B772B762B75544B1B7813F0010F00F034
:10CCE800BD80236843F6CC229B68444D934261D0B3
:10CCF8004E4E484F32783878D31803EB800004F052
:10CD0800A1FE4B4B0146186028789846A0F13002E6
:10CD1800D2B2092A01D943280FD109B2BA22FCF7A5
:10CD280027FF236832789B680146C8F800003878E6
:10CD3800D31803EB800004F07BFE2B782A2B04D158
:10CD4800337813B1394A013B13702B78232B0ED15A
:10CD58003378022B0BD8226846F6D95192688A425A
:10CD680005D020318A4202D0304A013313702B7823
:10CD7800552B01D0442B0FD1236831789B68A3F53C
:10CD8800D843B3F1950248BFA3F192023B7803EB75
:10CD9800A202D0B2FFF7D8FE264B1B7803F080031F
:10CDA800DBB23BB13278184B03EB820320225A7472
:10CDB8009A74DA742B78532B06D023689A6843F652
:10CDC800CC239A4240F0EF80FBF7B0FE236846F68A
:10CDD80095429B68934203D10E4B0220197806E0D6
:10CDE80046F6F952934227D10A4B002019780131AF
:10CDF800BDE8F0410CF0C4B874160308401D0020CB
:10CE0800D81500204B150308F401002095160308D7
:10CE1800781D0020071E00200502002009020020BE
:10CE28000D02002011020020571E0020121E0020B3
:10CE3800201E0020783A002046F6D952934204D1A9
:10CE48005A4B012019780918D2E746F695529342B1
:10CE580040F0A980554B03201978C8E723684AF2A7
:10CE68007E729B6893423FD1504E10205049FBF789
:10CE780099FD31784F4D01EB011101F5264101F57E
:10CE8800BF711022284604F0EEFD2B4605F1100173
:10CE98002A461078474F78B94749FBF783FD38464B
:10CEA800E721F3F7F5FA78B13178401B38180131EA
:10CEB8000322FBF79DFD07E013F8010B10B92030A2
:10CEC80003F8010C8B42E4D13C4D2B782A2B03D17B
:10CED8003078FD21FFF738FE2B78432B63D130786B
:10CEE80023680130C0B259E043F6CC229342334E56
:10CEF8001AD010203249FBF755FD33782A2B52D12E
:10CF0800304B1B689B68A3F5D843B3F1950248BF23
:10CF1800A3F19202254BFF211B7803EBA202D0B2AA
:10CF2800BDE8F041FFF710BE3378204D552B04D1F2
:10CF38002B78142B01D1033B2B703378442B05D16C
:10CF48002B78122B02D1194B15221A702B78DFF887
:10CF580078805901C918414401F5944100201F31D6
:10CF6800FBF720FD08F59241102017312F78FBF7C9
:10CF780019FD3378112F8CBF032700272A2B05D1E1
:10CF88002878FE21C01BC0B2FFF7DEFD3378432BA3
:10CF980009D12B78173BDF1B2368F8B2997CBDE8D1
:10CFA800F04118F017BABDE8F08100BF071E002055
:10CFB80053160308F401002063F70208401D0020FF
:10CFC80011160308781D00203CCD020810B50E4B41
:10CFD8001B78452B17D10D4B1A7842F006021A70B0
:10CFE8000B4A1378032B0ED80A490B4C086844F8EF
:10CFF80023000133137083680B60FBF7DBFBBDE88C
:10D008001040FBF793BD10BD401D0020571E0020A7
:10D01800371E0020781D0020441E002010B50C4B40
:10D0280004462146D8790FF07EF860B12046552194
:10D038000EF0D8FE48B120460EF06AFFD0F101008C
:10D0480038BF002010BD022010BD022010BD00BF57
:10D05800161E002008B50FF055F8C0B208BD000034
:10D068002DE9F047634B644C1A78994612F0010F8A
:10D07800624D65D02078FFF7D1FF614A2B181178EF
:10D08800604F93F8A031604E442938703360904661
:10D098000AD12D2B08D038B995F8A11101233B707E
:10D0A80031602078FFF7D6FF98F80030552B10D163
:10D0B80033682D2B0DD03B785BB1013B514ADBB275
:10D0C8001370EB1893F8A0114F4B20781960FFF7F5
:10D0D800C1FF98F80030232B19D14C4B20781B68DE
:10D0E8009B7C013B984212DA434B0130C0B2187066
:10D0F800FFF794FF3870281890F8A0313360444B3C
:10D108009B7803F00203DBB20BB1FBF747FB98F8FF
:10D1180000302A2B14D1207890B1374B0138C0B297
:10D128001870FFF77BFF3870281890F8A03133602B
:10D13800374B9B7803F00203DBB20BB1FBF72EFBF6
:10D14800344EFCF7F5FC237832789A4288BF337066
:10D1580032780F32934202DD2E4A0F3B1370DFF80C
:10D16800C480002730783818C0B2FFF757FF281856
:10D1780090F8A0310137102F08F8013F07D0254B50
:10D188001A78224BBA181B689B7C9A42EADB99F8FA
:10D19800003013F0010F13D01F4B1A781F4B02F009
:10D1A8008002D2B22AB1227831781032521A5F2125
:10D1B80005E0227831781032521A134909689954D7
:10D1C800134DAB7803F00203DBB25BB12078E91DA5
:10D1D800652246F69553FBF731FB05200B212A46BD
:10D1E800FBF798FB21780E4801310222BDE8F04791
:10D1F800FBF7FEBB571E0020121E0020346E0208EB
:10D20800401D0020581D0020201E0020781D0020F1
:10D21800681E0020091E0020783A0020F401002032
:10D22800F50100200302002038B50546002401233B
:10D23800A3402A78E0B29A4205D10E49102246F658
:10D24800D953FBF7FBFA0134042CF0D1043C0A4B08
:10D25800E0B2E3189A782B78934206D12BB10549AE
:10D26800102246F6F953FBF7E9FA0134042CEED103
:10D2780038BD00BF421D0020161E00202DE9F041D8
:10D28800074610460D461446F3F7D4FAC3B2804653
:10D29800B3B1AB4214D80B4E20212A46F019F3F74C
:10D2A80079F82046F3F7C6FAC8EB05056D08EDB224
:10D2B800EF1902462146F019BDE8F041F2F7C2BF66
:10D2C800BDE8F081F4010020F0B5154B0C781A1870
:10D2D80095781F46FDB100233A1892781A4112F04A
:10D2E800010F4FF001020DD0AC420E7803D09A40E6
:10D2F80042EA060604E09A40C2F10F0202EA060674
:10D308000E7005E09A400E78C2F10F0232400A70A2
:10D318000133042BE0D10B7803B90C70F0BD00BFCA
:10D32800161E0020312200230178194111F0010F47
:10D3380002D00449C9188A7501330132042BD2B2CC
:10D34800F2D17047F401002070B57D4B044631B12D
:10D358001B78532B40F0F280533B037070BD1A7852
:10D36800302A35D1774A53785BB1774B77491B78A8
:10D37800182000FB03135B7913F0100F01D0012371
:10D388005370734B20781978014013D09278002A93
:10D3980040F0D4801978114111F0010F06D0012115
:10D3A80091402078C1F10F01014021700132042A17
:10D3B800F0D143E01A780A4112F0010F04D001229B
:10D3C8008A4020780243227001310429F2D135E0E5
:10D3D800A2F13101C9B203293AD85A494A785AB157
:10D3E800594A5A481278182505FB0202527912F058
:10D3F800100F01D001224A701B78554A313B127830
:10D40800DBB21A4112F0010F00F09880227852FA2C
:10D4180003F010F0010F0BD08978002940F08E80BE
:10D42800013111FA03F3C3F10F0303EA020204E026
:10D43800012111FA03F343EA0202227000211222A9
:10D448004448F2F7A7FF2046BDE87040FFF7ECBE5E
:10D45800132A0CD0552A17D13B4B3C4A1B7818216C
:10D4680001FB03235B7913F0200F03D170BD354B0B
:10D4780001225A7000202146FFF726FF344B9B7883
:10D48800002B5BD0002051E0142A0CD02A2A17D197
:10D498002D4B2E4A1B78182101FB03235B7913F0CF
:10D4A800200F03D170BD274B01225A70012021465D
:10D4B800FFF70AFF264BDB78002B3FD0012035E031
:10D4C800152A0CD0232A17D11F4B204A1B78182164
:10D4D80001FB03235B7913F0200F03D170BD194BB7
:10D4E80001225A7002202146FFF7EEFE184B1B79E5
:10D4F800002B23D0022019E0162A0CD0442A1DD173
:10D50800114B124A1B78182101FB03235B7913F096
:10D51800200F03D170BD0B4B01225A700320214606
:10D52800FFF7D2FE0A4B5B7943B103200949102269
:10D5380046F6F953BDE87040FBF780B970BD00BFEF
:10D54800401D0020671300200A1E00203C3B0020DD
:10D55800161E0020421D00202DE9F04F87B09DF8CF
:10D5680040408146072C0D4605929A4637D1073C24
:10D5780027462B78234113F0010F2CD0012623B224
:10D588004FF0000802935120314632463346009648
:10D59800CDF8048004F0D4FA1B204146A219434672
:10D5A800CDF80080F5F7AAF837B9112039463A4680
:10D5B80033460097F5F7A2F8534B204613F824207A
:10D5C80001276FF3000203F824201199F5F720FFD3
:10D5D8002046F6F721F90134042CCAD10DE2012CBA
:10D5E80003780CD10BB90B7823B3FF2300930021E8
:10D5F800464B01911B780C200133029316E0022C54
:10D6080009D10BB90B78ABB10021FF23009301912D
:10D61800029134200AE0062C0CD10BB90B784BB1DF
:10D628000021FF23009301910291652004220B46FB
:10D6380004F086FABAF1010F99F800302BD13BB10A
:10D64800334B0020D979024653460090F5F756F837
:10D658002B783BB12E4B0120D9790022034600924A
:10D66800F5F74CF80020F5F7C5FE99F80030002BC7
:10D678005BD0284B1978002957D1274BDB78002B32
:10D6880053D0FF2300933A2001220B4601910291C7
:10D6980004F056FA49E063B1052C4FF0000102D1BD
:10D6A80000910F2001E000910B200A460123F5F7B5
:10D6B80025F82B7883B1052C4FF0000106D11020F6
:10D6C8000A4601230091F5F719F812E00C200A46E2
:10D6D80001230091F5F712F8022C25D0032C01D173
:10D6E8000E4B02E0042C02D10D4B1F781DE0052CD7
:10D6F80001D10C4BF9E7012C01D1044BF5E7062CBD
:10D708000CBFFF27002710E01E1A0020EB1A00208C
:10D71800161E00200C1A002067130020302000205D
:10D728001B570020973C0020FF2799F80030002B5A
:10D7380000F0B580934B944E1A78984602F0200278
:10D74800D2B262B1317811F0010108D1FF23009300
:10D75800282001220B460191029104F0F1F998F872
:10D76800003003F01003DBB26BB1317801F0020135
:10D77800C9B241B9FF230093292001220B46019128
:10D78800029104F0DDF998F8033013F0010F0DD081
:10D79800317801F00401C9B241B9FF2300932A206E
:10D7A80001220B460191029104F0CAF998F803305E
:10D7B80003F00203DBB26BB1317801F00801C9B2A2
:10D7C80041B9FF2300932B2001220B4601910291BE
:10D7D80004F0B6F998F8033003F00403DBB26BB138
:10D7E800317801F01001C9B241B9FF2300932C2010
:10D7F80001220B460191029104F0A2F998F8033036
:10D8080003F00803DBB26BB1317801F02001C9B233
:10D8180041B9FF2300932D2001220B46019102916B
:10D8280004F08EF911F006F968B1317801F0400181
:10D83800C9B241B9FF230093492001220B46019147
:10D84800029104F07DF998F8033003F04003DBB24D
:10D858006BB1317801F08001C9B241B9FF2300935F
:10D868004E2001220B460191029104F069F9767865
:10D8780016F0010613D14548314617F01AF858B189
:10D88800FF230093731C00211BB202937520012211
:10D898000B46019104F054F90136702EEBD1119B1F
:10D8A8003B4A19783B4B51B199F8001011702A780E
:10D8B8001A702B780BB1542005E0522003E0117048
:10D8C8002A7853201A7004F005FD119B00261A7857
:10D8D800314B1A7099F80030334113F0010F2DD0F5
:10D8E8003146059816F0E5FF0122014628B933B202
:10D8F800019000920293104605E0002133B2009295
:10D908000191029324200B4604F01AF9BAF1010F91
:10D9180005D1224B8020DA790521013208E0022C5A
:10D9280007F1010202D18020072101E080200621B1
:10D938003346F6F7AFFA3046F5F742FF2B78334116
:10D9480013F0010F55D000214FF0010B33B20293B1
:10D9580002205A460B46CDF800B0019104F0F0F8C9
:10D96800DA45DFF83C801DD118F8263013EA0B039E
:10D9780032D10A4A0520D1790093594406EB0B02AB
:10D9880028E000BF783A0020DD1B0020FC190020A9
:10D99800561A0020571A0020FB1B0020161E0020D4
:10D9A8001E1A002018F8263013F0010314D1022C97
:10D9B8000CD1134B1B7803F02403042B04BF114B29
:10D9C80083F800B000230093072001E000930620AD
:10D9D800791C721CF4F792FE11993046F5F718FD80
:10D9E8003046F5F719FF18F826306FF3000308F8EA
:10D9F80026300136042E7FF46DAF07B0BDE8F08FF6
:10DA0800041C0020601300202DE9F04180460E46DA
:10DA1800174646F2BF7500243846214616F049FFDE
:10DA280088B1294608220B4804F01DF809484146E8
:10DA380016F0ECFE074816F00FFF20B90123A340AB
:10DA480032781343337001340835042CE4D1BDE82F
:10DA5800F08100BFF31B00202DE9F04387B080461A
:10DA6800894604A847F2E911082203F0FCFF0024C4
:10DA780040462146E7B216F01CFF002843D038463E
:10DA8800F4F776FB0025661C0246314611202B462A
:10DA98000095F4F733FE012321462A460420FF08A7
:10DAA8000095F4F72BFE4BF2DF50381803F0CAFF4D
:10DAB80004F00703C1B2194111F001014FF002024D
:10DAC8004FF001030AD00092019336B2772029461D
:10DAD80092182B46029604F033F814E00092019352
:10DAE80036B2232004220B46029604F029F8B9F135
:10DAF800000F08D004A8214616F0DBFE18B105482F
:10DB0800214616F0C0FE0134402CB1D107B0BDE863
:10DB1800F08300BF331A00202DE9F74F17469846C7
:10DB28003B7805460C469DF830909DF834B09DF83A
:10DB38003820DFF8B8A043B102EA03033B70097844
:10DB48009AF800208A18D31A0370237883B12248E0
:10DB58002146F5F70DFE21491F4816F057FE1E48CD
:10DB68000121FFF779FF1C4841462246FFF74CFF89
:10DB78001B4B00261E70297843F6FB2003F058FF44
:10DB8800494646F2CD6003F053FF204639464A46DF
:10DB9800F5F7E6FB134B42461E7139464B462046C5
:10DBA800CDF800B00195FFF7D7FC2846F8F728FB19
:10DBB8002B780D480D498AF80030F5F7D9FD11F09A
:10DBC80079FF88F800603E7026702E7003B0BDE8BB
:10DBD800F04F04F089BA00BFFC1B00204E1A002049
:10DBE800541E002067130020DF1B00200C1A0020A1
:10DBF80010B50B4B0B4C024603CB206061600A4802
:10DC0800114616F024FE2146074816F0FFFD064887
:10DC180016F022FED0F1010038BF002010BD00BF71
:10DC2800302E0020E91B0020F31B002010B50A4C01
:10DC3800637C4BB100200949FAF7B4FE084B1B7806
:10DC4800432B01D1433B6374607C20B90549BDE88F
:10DC58001040FAF7A7BE10BD421D0020A5F7020824
:10DC6800401D002084F70208034B1A7801321A700D
:10DC780001230370704700BF541E002010B50C48E4
:10DC8800FAF736FE0B4A002414700B4A0B4B14703B
:10DC98000B4A5C7114700B4A1C7114700A4A5C7050
:10DCA80014700A4A1470FAF741FF094B1C6010BD42
:10DCB800681E0020161E0020411D0020671300204A
:10DCC800581E0020651E00207C1D0020541E0020C8
:10DCD800781D00202DE9F04F974B984E93F800904F
:10DCE8003368DFF8A8829C7C954BF0221A7098F86C
:10DCF80000308BB00D2B354647463DD1914B93F8FC
:10DD080005C0BCF1010F02D900208F492FE01AD1BC
:10DD180000245C718D4A8E4B8E498F488F4D04705C
:10DD28001C7014700C70CDF800C001942D78029509
:10DD3800FFF7F2FEFAF7FAFE894834600BB0BDE847
:10DD4800F04FFAF7D5BD87488249F5F711FD864BA4
:10DD5800864A03CB864B10601B785160532B5FD1EA
:10DD680098F800308349013388F8003000200BB060
:10DD7800BDE8F04FFAF716BE092B0FD17C4B1B7884
:10DD8800532B3DD17C4B00221A700D2388F80030AC
:10DD98007A4B1A7842F006021A7089E20E2B37D1B4
:10DDA800734B1B78532B2BD175496E4816F02EFDFB
:10DDB8006C48FFF71DFF044640B198F80030052273
:10DDC800013B88F800305F4B5A7171E2082246F235
:10DDD800CE61664803F047FE64496A4816F037FD8D
:10DDE800012300935D4B01941B785B4802935949CA
:10DDF800564A574BFFF790FEFAF798FE346057E201
:10DE0800232B40F055820BB0BDE8F04FFFF736BF2B
:10DE180033B95D4B1A781AB901321A7011F04AFEFB
:10DE2800631E48BFA31DDB10013303FB09F91FFA6A
:10DE380089F909F5CC46A9F59449A9F121094F4B6F
:10DE4800CDF81C901A78CE3612F0010F4A4C00F02B
:10DE58002081474B1A789946432A40F0C9803B787D
:10DE68000D2B40F0C5803F48217816F022FD002890
:10DE780000F0BE803D48217816F01BFD002840F0D8
:10DE8800B780079920780FFA81FB0BEBD00003F0DD
:10DE9800D9FD23784FF0010A03F007020AFA02FAC3
:10DEA800DFF8EC805FFA8AFA10EA0A0FC8F8000077
:10DEB80027D0244BDB78002B40F09A80274BD87969
:10DEC800F8F7FCF8002800F09380D8F80010CAF1A1
:10DED800FF0A20780AEA0101C8F800100BEBD0000D
:10DEE80003F0A6FD20780FFA86FB0BEBD00003F0B9
:10DEF800A9FD00EA0A012078C8F800100BEBD00051
:10DF080061E032B202EBD300059203F09BFD10EA08
:10DF18000A0FC8F800003DD140EA0A01059B2078A5
:10DF2800C8F8001003EBD00003F082FD21781548F3
:10DF380016F0A9FC5CE000BF071E0020781D002039
:10DF4800631E0020671300204AF80208581E0020AC
:10DF5800411D0020651E00207C1D0020161E00208B
:10DF6800681E0020FC1B0020302E0020F419002021
:10DF7800401D002010F90208121E0020571E002024
:10DF8800431A00204E1A0020A8140020541E002016
:10DF9800201E0020924BDB7823B9924BD879F8F7F2
:10DFA8008DF8B8B92078DDF814C0CAF1FF0A0CEB77
:10DFB800D00003F047FD8C4A00EA0A01059B20784F
:10DFC800116003EBD00003F033FD2178874816F089
:10DFD80065FC0DE020780BEBD00003F033FD40EA40
:10DFE8000A012078C8F800100BEBD00003F020FDE0
:10DFF80099F80030232B10D12A682378927C013AB3
:10E0080093420ADA7A4A013313707A4B9B7803F009
:10E018000203DBB20BB1FAF7C1FB99F800302A2BE7
:10E028000CD1237853B1724A013B1370714B9B7822
:10E0380003F00203DBB20BB1FAF7B0FB99F800303A
:10E04800552B12D129682278897C694B08398A4274
:10E0580001DA083200E000221A70664B9B7803F060
:10E068000203DBB20BB1FAF799FB99F80030442BA5
:10E078000FD122785E4B072A9CBF2A68927C083A07
:10E088001A705C4B9B7803F00203DBB20BB1FAF712
:10E0980085FBFBF74DFD584A237811789246994243
:10E0A80088BF137012780F32934202DD524A0F3B39
:10E0B80013702B684FF0000B93F81280CDF818B04E
:10E0C800B8F10F0F9ABFC8F120085FFA88F84FF02F
:10E0D800100839784FFA8BF30D2905D19AF80020EA
:10E0E8009B18DB10454A04E09AF800209B18444A24
:10E0F800DB10D35C9AF8002005934FFA8BF39A183B
:10E108000D2902F007094FEAE20202D13D49895C74
:10E118000691DDF81CC004930FFA8CF0101803F078
:10E1280091FCC0B2049B08909AF8000032B218180B
:10E1380002EBE00003F086FC39789AF80020049B93
:10E14800C0B209919A1846E0059BDDF824C043FA4D
:10E1580009F12D4B01F0010100290CBFA521DB219C
:10E16800BCF10D0F03F8081014D128494FEAE20C4E
:10E1780011F80C1041FA09F111F0010F08D0DDF87F
:10E1880018C04CFA09F111F0010F03D0582110E022
:10E198002D210EE0DDF820C04CFA09F111F0010F35
:10E1A80001D0502105E040FA09F111F0010F02D029
:10E1B800542103F8081009F101095FFA89F90BF1F4
:10E1C800010B08F101080132B9F1080F5FFA8BFB66
:10E1D8005FFA88F81CD0B8F1200FB5D125E000BF50
:10E1E80067130020161E0020201E00204E1A002053
:10E1F800121E0020681E0020091E0020431A00205D
:10E20800A31A0020F4190020F4010020FC1B0020B0
:10E21800B8F1200F09D09AF800304FFA8BF2D218D3
:10E228002B689B7C9A42FFF654AF23490B7813F076
:10E23800010F17D02B68214A9B7C12780F2B02F014
:10E24800800298BFC3F11003D2B294BFDBB200239F
:10E2580042B122789AF800101032521A1849CB1895
:10E268005F219954174EB37803F00203DBB293B1E0
:10E27800F11D652246F695432078FAF7DFFA2B68F8
:10E288009B7C102B02D905200B2101E000200721DF
:10E298003246FAF73FFB2B689B7C102B08D9217874
:10E2A8000948013102220BB0BDE8F04FFAF7A0BBD4
:10E2B8000BB0BDE8F08F00BF571E0020783A002051
:10E2C800F4010020681E0020F50100202DE9F0432C
:10E2D800002387B08DF817307C4B1B78012B00F09A
:10E2E80070827B4B1A78984672B17A4BDB78002B98
:10E2F80040F06782784C2378002B40F0B580FAF71D
:10E3080015FC09232370AFE0734B19781C460829C4
:10E3180000F2AA8071490978232913D11A70FAF7F3
:10E3280005FC6F496F4A0B7853B16F48013B04787D
:10E33800DBB244F0060404700B706C4951F82330CA
:10E348001360AFE2684B1A7812F0010F04D1012173
:10E358000A438DF817101A70F4F704FE28B92378C9
:10E368001BB90DF11700FFF77FFCF4F709FE30B970
:10E378002378012B03D10DF11700FFF775FCF4F793
:10E388000DFE30B92378022B03D10DF11700FFF7EA
:10E398006BFCF4F70FFE30B92378032B03D10DF192
:10E3A8001700FFF761FCF4F713FE48B9F4F73CFED9
:10E3B80030B92378042B03D10DF11700FFF754FC73
:10E3C800F4F766FE30B92378052B03D10DF1170059
:10E3D800FFF74AFCF4F750FE30B92378062B03D137
:10E3E8000DF11700FFF740FCF4F700FE30B9237871
:10E3F800072B03D10DF11700FFF736FCF4F704FEE5
:10E4080030B92378082B03D10DF11700FFF72CFC46
:10E418009DF8173043B32378082B23D8DFE803F09F
:10E4280005080D101316191C1F000020304901E0C3
:10E4380030490020FAF7B6FA16E000202E49F9E72D
:10E4480000202E49F6E700202D49F3E700202D494A
:10E45800F0E700202C49EDE700202C49EAE70020EE
:10E468002B49E7E7FAF762FB1B4F3B783D46092B40
:10E4780040F0B2801C4E194F317811F0010153D190
:10E48800244C12222046F1F785FF01236374224AA7
:10E4980098F80030137003B96374637C13B11F4B91
:10E4A80000221A70FFF7C2FB1B48617CFEF74CFF85
:10E4B800337803F0FD0343F001033370184B1A78E7
:10E4C80082B33A7000221A702EE000BF631E00204B
:10E4D8000C1A002067130020541E0020401D002045
:10E4E800371E0020781D0020571E0020441E0020E3
:10E4F800F6FD0208D5FD020817FE020838FE0208DC
:10E5080059FE02087AFE02089BFE0208BCFE0208B9
:10E51800DDFE0208421D00207C1D00206013002043
:10E528000C1E002030233B703B78884E13B973785B
:10E53800102B4DD1DFF86492854CFFF777FB8448A8
:10E5480099F81110FEF700FF237823B1002010215D
:10E558004A46FEF793FE98F8003024787D4A24EA6C
:10E56800030111707C4A23EA040111703A78A2F180
:10E578005200C0B2012803D97078744F10280CD10A
:10E58800002373701CB911B10133009311E1042306
:10E5980073712B7801332B701AE0432A18D1BBB959
:10E5A800FC78ACB96D4BD879F7F788FD38B96C4968
:10E5B800FAF7F8F905237B7108332B7004E020463D
:10E5C8006849FAF7EFF97C71674A684B1A6069E1A4
:10E5D8005F48FEF7A7FE65E10A2B31D15D4809F0D7
:10E5E800BDFCC6B2594C36B36379042B02D1002066
:10E5F8005F4903E0022B04D15E490020FAF7D2F903
:10E6080002E00BB904336371314602225A48FAF723
:10E61800EFF95A4B1E78232E00F0D3803046FAF7D4
:10E628007DFA002800F03E81312E40F03B812B78A6
:10E6380001332B7002E03B7801333B70042332E056
:10E648000B2B32D1434809F06FFCC6B23F4C36B3AE
:10E658006379042B02D10020494903E0022B04D13D
:10E6680048490020FAF79EF902E00BB904336371B8
:10E67800314602224048FAF7BBF9404B1E78232E58
:10E6880000F09F803046FAF749FA002800F00A8126
:10E69800312E40F007812B7801332B7002E03B7854
:10E6A80001333B7008236371FCE00C2B40F0FA80C7
:10E6B800284809F01FFC0021C4B2264809F0F0FBE5
:10E6C800002C6DD0214E33792BB9BE2016F0DEFE1A
:10E6D80033790133337173791C4A092B02D900202D
:10E6E8001F4915E010D11D4B00241C705471264B96
:10E6F800194A1849164801251C7014700C700470CA
:10E708000095019402949EE0082B04D11F49002033
:10E71800FAF748F911E0062B02D100201C49F7E767
:10E72800042B02D100201B49F2E7022B02D1002062
:10E738001949EDE70BB9083353717379082B3CD8A5
:10E748000D4821460222FAF753F936E067130020F4
:10E758007C1D0020651E0020581E0020161E00206B
:10E768004AF80208C6F70208D86F0208781D002088
:10E77800CEF80208EFF80208F4010020401D00203E
:10E788008CF80208ADF80208411D0020E7F70208DE
:10E7980008F8020829F802086BF80208421D002050
:10E7A800012542484249434A2B460095F5F792F91C
:10E7B8000095414B01941B7840E0404F3C78232C56
:10E7C80002D1FFF75BFA6DE02046FAF7A7F90028B7
:10E7D80068D0303CE4B2631EDBB2012B3C7039D800
:10E7E800022C354D1ED1E879F7F768FC002838D09F
:10E7F8002E48FFF7FDF9002833D1082246F2CE61F2
:10E808002F4803F030F929492D4816F00AF82C4909
:10E81800082246F2CE6003F020F92949294816F06B
:10E8280016F806E0012321482149224A0093F5F70A
:10E8380051F901230024009301942B780293224874
:10E848001C49224A1A4BFFF767F9FAF76FF9204B70
:10E858001C6027E0032C25D1174BD879F7F72EFC3D
:10E8680010B90C2373711DE000241048214616F0DE
:10E8780020F828B1E02016F009FE204616F042FEE6
:10E888000134402CF1D1134A0023137073712B7893
:10E89800114A01332B700E4B1A60104B1A7842F054
:10E8A80006021A7007B0BDE8F08300BFFC1B002009
:10E8B800411D0020651E0020161E0020401D00205E
:10E8C800F41900204E1A00207C1D0020581E00203C
:10E8D800781D0020121E0020D86F0208571E002045
:10E8E80088234B43054A03EBD003D35C00F00700B1
:10E8F80053FA00F000F00100704700BF840D0020BB
:10E9080070B504461646157839B912E00135EDB2EE
:10E9180028462146FFF7E4FF48B9202DF6D970BDF7
:10E92800013DEDB228462146FFF7DAFF08B1356010
:10E9380070BD002DF4D170BD064B38211B78032221
:10E9480001FB0031044844230370C9B2173BC3706C
:10E95800FAF74EB8121E0020F4010020012802D058
:10E96800022806D102E01D20044904E01D200449C4
:10E9780001E004491D20FAF715B800BFF1F00208BC
:10E98800D0F0020812F10208037809680F4A03EB75
:10E998000310401802EBC00050F8240C0C498842C0
:10E9A8000FD1882101FB03239A68A0F59C63063BDD
:10E9B8009A4208D0A0F598600538101A18BF0120AF
:10E9C8007047002070470020704700BF840D00206A
:10E9D800AFF0020803780A6803EB0313D318084A58
:10E9E800053B02EBC3035968064A914205D1187AE0
:10E9F80009288CBF0020012070470020704700BF05
:10EA0800840D0020AFF002082DE9F04F984B994F84
:10EA1800F0221A703B6889B09C6847F2F373E11AD8
:10EA28004C4244EB0104DD3A6243934B9D5C03EB9B
:10EA38000208C5F30005EEB23A46002E2CD1304646
:10EA48008E49F9F7AFFF8E4B1B78232B41F02A82B2
:10EA580098F8013066F3041388F80130FAF766F87D
:10EA6800884B1A7842F006021A70874A1378013BDD
:10EA7800DBB21370854A52F823303B60844B1D701B
:10EA8800844B1D70844B1D70844B1E60844B1D701D
:10EA9800844B1D7001F006BA814D95F80090B9F1CC
:10EAA800000F0CD04FF43661614309F1FF30342375
:10EAB80003FB00137C49CB181B798DF81F307B4B67
:10EAC8001E787EB17A4E2046317810F097FE0028E5
:10EAD80040F05C84754930700870074606468046E9
:10EAE80000F05BBC6D490B688B46A3F1120003284C
:10EAF80009D9A3F11601032909D9A3F11A01032998
:10EB080009D9374605E037464FF0010805E0374692
:10EB18000126B84601E00127B0465949097853292A
:10EB280040F0D581B9F1000F3AD1722262436149B0
:10EB3800885C10F0020F0AD0002B41F0B38101333A
:10EB480063F383008854CBF8003001F0ABB95A4B1B
:10EB5800997989B120464A4610F038FEFF2801F01D
:10EB6800A18101302870CBF80090F9F7DFFF20462B
:10EB7800FFF7E2FE01F096B9DFF8FCC0132202FBB2
:10EB880004C25178204669F3041151704B4A02219E
:10EB980082F80090039310F0BFFD0122039BCDE2A1
:10EBA80009F1FF312046C9B210F028FE002840F0D4
:10EBB8008B80DFF810B1DFF8EC909BF80020012380
:10EBC80032B98BF80030324B89F800201A70E4E330
:10EBD80005900393F9F7AAFF05988BF80000039BAB
:10EBE80089F80030364A835C9246A3F13001C9B2F5
:10EBF800092904D9413BDBB2052B01F253810130CD
:10EC08000A28EFD14FF0000847460AEB480015F0F4
:10EC180085FE7B080237FFB20A2F294E0AF8030047
:10EC280008F10108F1D1304611F0D4FA002801F0BA
:10EC38003981304611F03CF80746002841F032810E
:10EC48001D4B3046997911F0D4FA002801F02A8139
:10EC58002978337901392046C9B2022200970196F2
:10EC680011F01AFB022389F8003001F01BB900BF2C
:10EC7800631E0020781D0020833A00203FE202082E
:10EC8800401D0020571E0020371E0020441E002073
:10EC98005D1D0020861D0020071E0020201E00206C
:10ECA800121E0020091E0020043E0020541D0020D2
:10ECB800081E0020C454002067130020561E0020A0
:10ECC800381E0020131E0020DBF80030DFF8089300
:10ECD800202B27D0212B23D14FF436626243297889
:10ECE8003420013900FB0122AC489DF81F3012186E
:10ECF8004FF0000B20460192C9B20322CDF800B0B4
:10ED080011F0CAFAF9F712FF2A78A54B013AA5487B
:10ED18001A701423C9F800B085F800B003703CE3FA
:10ED28001E2B03D10133C9F8003019E31F2B18D16A
:10ED38004FF43662624329783420013900FB0122FE
:10ED480096484FF0000B121801929DF81F3020468C
:10ED5800C9B20622CDF800B011F09EFAC9F800B089
:10ED6800FEE29A1F062A0ED88F4B1A7819462AB93E
:10ED780001321A708D4B1A788D4B00E3012A40F04E
:10ED88000C830223A1E1A3F10D02042A3AD8894990
:10ED9800D3B291F800C095F800E08048864ABCF1EB
:10EDA800000F1ED04FF0000C81F800C011784FF40E
:10EDB800366262430EF1FF3E0CF1340C0CFB0E225E
:10EDC8008018C0184174382000FB04EE5FFA8EF0FA
:10EDD80000EB800000F5F8401B30C01802F028FE58
:10EDE800DBE24FF0010C81F800C04FF4366161435B
:10EDF8000EF1FF3E0CF1330C0CFB0E1E7044C318D1
:10EE08005B7C59E0A3F112020B2A4CD86B4A297893
:10EE18001078002845D000201070A3F1120938227C
:10EE28004B1E02FB0433203ADBB2534303F5FC4389
:10EE38005FFA89F9DFF894B14B3303EB49039BF888
:10EE480000101846039302F0F3FD5D4A4FF4B66CC8
:10EE58000CFB04FC11781A22013902FB01C14F484E
:10EE6800494400EB41019BF80000DFF870B1887558
:10EE7800039B9BF80010581C0492CDF814C002F0B4
:10EE8800D7FD4F49049A0B78DDF814C0013B02FB0B
:10EE980003C2424B4A4403EB42029BF80030D3754D
:10EEA8007BE2012308E0DFF8209199F800302BB9C4
:10EEB800012289F80020434A13706EE2F9F736FE02
:10EEC800002389F800302046FFF736FD65E2432924
:10EED8004BD1354A1278002A40F05F82354A1278C1
:10EEE800002A40F05A82B9F1000F00F05682364AE3
:10EEF8001278002A40F05182212B30D01F2B30D0BD
:10EF08002E4B1978012919D9B8F1000F02D1002F19
:10EF180000F043822D4B02391A7852FA01F010F0B2
:10EF2800010F4FF0010004D010FA01F122EA0102AA
:10EF380025E210FA01F141EA020220E200F02D82F6
:10EF480009F1FF312046C9B210F058FC20B9204B16
:10EF58001B78002B40F0218200232B7000E2202335
:10EF680000E01E23CBF80030FAE1232940F0968018
:10EF78000D4B1B78002B40F010820E4B197800299E
:10EF880040F00B82104BB9F1000F50D01A783AB309
:10EF98000C480F2A01700F48017042E1043E00201E
:10EFA800081E0020541D0020561E0020061E0020AA
:10EFB800641E00201F1E0020D41E00200B1E0020EF
:10EFC800121E00205D1D0020071E0020051E0020C7
:10EFD800131E0020861D0020201E0020551E002024
:10EFE80009F1FF312046C9B210F008FCB0B19A4AC5
:10EFF80013787BB1B8F1000F01D0042B08D90EB1FA
:10F00800012B05D9002F00F0C881042B00F2C28122
:10F01800013351E79DF81F000121F6E08F4B1A7864
:10F02800511EC9B208296FD801321A706CE0DFF896
:10F038006CC2132101FB04C1487869F304104870BD
:10F04800022120460492039310F066FB08F034FE78
:10F05800F9F76CFD8249087840F00600087081488D
:10F0680001780139C9B201707F48049A50F821101B
:10F0780011607E4A82F800907D4A82F80090039BD6
:10F08800CBF8009083F800907A4B85F8009083F8CD
:10F098000690794B83F8009000F004BF2A2936D1F6
:10F0A800764B1B78002B40F07881754B1A78002A34
:10F0B80040F0738173490B784BB16C48012B027097
:10F0C8006B48027040F26981013B0B7065E1B9F150
:10F0D800000F00F0628109F1FF312046C9B210F03B
:10F0E8008DFB58B15C4A137823B1012B40F255814E
:10F0F800013BE1E69DF81F00002186E0574A13789E
:10F10800012B01D9013B13700022584B37E14429E8
:10F1180040F08D80594A1278002A40F03E81B9F1BA
:10F12800000F0DD1534B9A79511EC9B2012901D84C
:10F13800013203E0032A40F03081023A9A712CE14F
:10F14800504A1278002A40F02881444A1278002A4E
:10F1580040F023814A4A1278002A58D13E4B1B7846
:10F16800012B09D9002E00F01881474B1A78072A7D
:10F1780000F212810132AAE019D1B8F1000F0BD0C8
:10F18800424A032011789846013191FBF0F000EBD8
:10F198004000091A117000E1002E00F0FE803B4A81
:10F1A8001E461178013101F003011170F5E0314B71
:10F1B800204699794A4610F009FBFF2800F0ED80B7
:10F1C800DBF80030212B00F0E8801F2B00F0E580F1
:10F1D800013028702046FFF7AFFB4FF436626243D8
:10F1E80029783423013903FB0123294A9BF80000BD
:10F1F800D31893F8049049468DF81F90FFF770FBD9
:10F208000146002840F0AC804846224AA6E00D2B73
:10F218000BD19DF81F0010F0A3F930B11E4B1A78DE
:10F228001F2A00F2BA800132A9E00120AAE055297C
:10F2380040F0B380114A1278002A40F0AE80B9F14C
:10F24800000F2DD10B4B9A79012A01D9013A75E7A4
:10F2580040F0A380032271E70B1E0020131E00203C
:10F26800571E0020371E0020441E00205D1D002070
:10F27800861D002067130020091E0020561E00204E
:10F288001F1E0020071E0020051E0020551E0020FE
:10F29800043E0020201E0020D41E0020833A0020B7
:10F2A800894A1278002A78D1884A1278002A74D1BB
:10F2B800874A1278002A56D1864B1A78012A08D92B
:10F2C800002E6AD0844B1A78012A65D9013A1A703F
:10F2D80062E012D1814B197811B1013919705CE0E3
:10F2E800B8F1000F03D002211970904655E0002EA6
:10F2F80053D00321197016464FE0B9F1010F4CD9CC
:10F30800774BA9F1020220469979D2B210F06CFA33
:10F31800FF2842D0DBF80030DFF8D091212B3CD019
:10F328001F2B3AD0013028702046FFF705FB4FF419
:10F338003662624329783423013903FB0123694A81
:10F3480099F80000D31893F804B059468DF81FB007
:10F35800FFF7C6FA014618B958464A46FFF7D0FAE9
:10F36800F9F7E4FB19E00D2B0BD19DF81F0010F005
:10F37800F7F830B15C4B1A78012A0ED9013A1A70A5
:10F388000BE0FF20584910F009F806E000273E4638
:10F39800B84602E0012700E001262978DFF89891B5
:10F3A800002940F0CB8099F8003013F0010205D114
:10F3B80043F0010389F800304C4B1A6000252046C1
:10F3C800294610F09BFC30B172236343484AD15C54
:10F3D80041F00201D1540135382DF0D13A35654359
:10F3E800434E735D13F0020F43F3400015D03F4CBA
:10F3F800206810B93F4900F0C1BC00203E49F9F728
:10F40800D1FA735D13F00C0F43F3810540F04A8580
:10F41800F9F78CFB256000F045BD314DAB79A3B100
:10F42800012B01D1354906E0022B01D1344902E014
:10F43800032B02D13349F9F7B5FAA979204610F020
:10F448000FFA022201463048EDE114B920462F494F
:10F4580001E02F491846F9F7A5FA2E4803786BB949
:10F468002D490A222D48F1F76BFA2D49132303FB86
:10F4780004135A7842F010025A7004E027482949C8
:10F488000A22F1F75DFA284D3821022205F11E0003
:10F49800F9F7AEFA204610F007FA0222014605F104
:10F4A8001900F9F7A5FA214B00221A70204B1B7896
:10F4B80003F08003DBB2002B00F0F4841D4B1B88A3
:10F4C800EB8100F0EFBC00BF071E0020131E0020D8
:10F4D8001F1E00200B1E0020051E0020551E0020A8
:10F4E80067130020043E0020D41E0020201E0020A8
:10F4F800C454002081E20208A2E20208AAE302083A
:10F50800CBE30208ECE3020812020020E4E202085E
:10F5180068E30208541D00200DE40208FA010020E7
:10F52800833A00202EE40208F4010020091E00207E
:10F53800783A0020E1550308571E0020013920467B
:10F54800C9B210F05BF9002800F0F483954B93F8EA
:10F5580000B038230BF1FF3B03FB04BB99F80030E4
:10F568005FFA8BFB13F0010F03D08F4A1378002B3F
:10F5780041D08E48F9F7BCF90BEB0B1101F5E841C6
:10F5880010228B483B3102F06EFA884B11229A7197
:10F59800884B1B6813B91020874921E0012B02D141
:10F5A800102086491CE0022B02D11020844917E064
:10F5B800052B02D11020834912E01E2B02D1102006
:10F5C80081490DE01F2B02D11020804908E0202B33
:10F5D80002D110207E4903E0212B03D17D49102060
:10F5E800F9F7E0F999F800306F4843F0010389F81A
:10F5F800003000230370784B1A78002A00F0AB80A3
:10F608000BEB0B1B0BF5E84909F13B09102273487A
:10F61800494602F028FA00229346704B995C41B1A2
:10F628000BF1010B5FFA8BFB0132BBF1100FF4D128
:10F6380007E06A49C2F1100201EB0B002021F0F744
:10F64800A9FE654A107858450BD90138484402F09C
:10F65800F9F930B9604B202118780138484402F094
:10F66800E7F9DFF894B19BF8003018460393F9F7EF
:10F6780055FADC46039BDFF878B110B9432B44D127
:10F6880001E0432B05D100238BF800304FF0200A0E
:10F6980030E05348534A90F800E053499E450ED154
:10F6A800AEF1300E0A20137800FB0E1E0133DBB2D8
:10F6B8001370734493F8AD307BB913700DE0037089
:10F6C8009BF800304FF0000E82F800E02BB1424862
:10F6D80003780F2B01D80133037040238BF80030D7
:10F6E80013789CF800200A20303A00FB0211C91850
:10F6F80091F8ADA03849394A08785146013802F8DE
:10F7080000A0484402F094F90FE0384B1B7803F04E
:10F718008003DBB24BB19BF8003033B92E482F4938
:10F728000378FF22CB1803F8012C9BF8003013B1A3
:10F738002F4A013B13709BF80030012B10D1264A49
:10F7480013780F2B01D801331370264A00238BF846
:10F758000030137004E004200C21144AF9F7DAF899
:10F76800144A13689346002B48D14FF4366262431B
:10F7780029783424013904FB01241E4AA41861782D
:10F78800164AC1F3C30109B93F2004E0994201D9DF
:10F79800DB2000E0A5200133DBB2907501320A2B93
:10F7A800F1D17FE3121E0020091E0020681E0020F0
:10F7B8006F1E0020201E00202BF0020815E502080D
:10F7C80057E502081DE60208C2E60208E3E6020859
:10F7D80004E7020825E70208071E0020F4010020BC
:10F7E8005A1D0020861D0020346E0208783A002039
:10F7F8005D1D00200C3E0020401D0020012B15D16E
:10F808004FF4366363432A783424013A04FB023404
:10F81800AB4BE418637813F0070300F0438314211B
:10F828005943A8488322F9F7E3F83BE3022B26D192
:10F83800A54A9DF81F30882101FB03232978A34A94
:10F84800D87901390623202502F8015950FA03F521
:10F8580015F0010F10D04FF436656543342606FBCA
:10F8680001559B4E7519ED791D4115F0010F01D019
:10F87800DB2500E0A5255570013BE4D212E3032BFC
:10F8880013D14FF4366363432A783424013A04FBD6
:10F8980002348F4B1C19237A13F0010F02D0102069
:10F8A8008C496BE210208C4968E2042B13D14FF489
:10F8B800366363432A783424013A04FB0234844BC8
:10F8C8001C19237A13F0020F02D01020834955E245
:10F8D8001020834952E2052B15D1162700262B78D4
:10F8E8003422013B53434FF4366202FB0433784A17
:10F8F8007C49D318985DC919013614F0F5FF023711
:10F90800052EECD1CEE2991F062900F2FF809DF862
:10F918001F206D4F02EB0210411807EBC101C968A7
:10F92800714801F1100651F804CBB14240F804CBFC
:10F93800F9D19E1FF6B202EB02129219013207EBBF
:10F94800C202507A92F80AC0684A29781378904619
:10F9580073B94FF4366363433422013902FB013132
:10F96800634BCA5E634B024102EA0C021A7011E053
:10F97800022B0FD1604B01391B784FF0000900931F
:10F988002046C9B204223346CDF8049010F084FC16
:10F9980088F8009098F80030012B29D1574BDFF8F0
:10F9A800589193F800A05046F9F7B8F810B9BAF191
:10F9B800430F1AD10DF11F005149FFF70BF810B191
:10F9C800002389F800309DF81F30DBF8002003EB96
:10F9D80003139B1807EBC303504699F8001013F85C
:10F9E800202CFAF7C5F889F8000099F800A003E080
:10F9F80013B9404B93F800A0BAF1090F07D9BAF12F
:10FA0800630F8CBF4FF003094FF0020901E04FF07C
:10FA180001099DF81F3003EB03139E1907EBC60776
:10FA2800FB685A7BE02A02D12E4A202151779A7B23
:10FA3800E02A02D12B4A20219177DA7BE02A02D1F1
:10FA4800284A2021D17798F800200ABB4FF4366263
:10FA5800624329783424013904FB0124184AA41884
:10FA6800A27812F0080F1BD05A7BE02A02D11D4A57
:10FA78003F2151779A7BE02A02D11A4A3F21917798
:10FA8800DB7BE02B40F00E82164B3F22DA7709E24F
:10FA98001C4B1B7803F08003DBB2002B40F0028282
:10FAA8000DF11F001649FEF76FFF18B15046FEF71B
:10FAB80055FFF7E114485146C9EB00004A46B2E643
:10FAC8000C3E00200F020020840D002013020020AD
:10FAD800043E0020BAE50208DBE5020880E60208D9
:10FAE8005FE60208F401002004020020561E0020F0
:10FAF800093E0020061E0020641E0020401D002034
:10FB0800201E0020783A002014020020A3F10D02E4
:10FB1800042A31D89DF81F30D6B2222202FB036393
:10FB2800984A02EB83035F6C3846F0F783FE394648
:10FB380002469548F0F704FF944B1B786BB1944B41
:10FB48001B7803F08003DBB21BB19248202102220C
:10FB5800EDE0914B8F4819780CE04FF4366363431E
:10FB68002A783424013A04FB02348C4B89481C1946
:10FB7800A619717C822256E6123B0B2B00F2928169
:10FB88009DF81F20DBB2222101FB02317D4A16318C
:10FB980052F821207C4902F110008A4652F804CB21
:10FBA800824241F804CBF9D1DFF83092DFF830B265
:10FBB8002FB199F80020012A15D1013209E096B138
:10FBC80099F80020012A07D97549097803290AD12B
:10FBD800013A89F8002006E005D17149097803291E
:10FBE80008BF8BF8002099F800209AB94FF4B66145
:10FBF8004C432A781A21013A01FB0244674AE31868
:10FC0800083302EB43039A798BF80020DA79644BC6
:10FC18001A7047E1634C202104F118000822F0F71C
:10FC2800B9FBB8F1000F00D1AEB15D4D2B78012BB7
:10FC380001D15D4A01E04BB95C4A136823615368FE
:10FC4800CAF80430B8F1000F21D00BE0022B0CBF2A
:10FC5800574A584AF1E7584A136823615368CAF863
:10FC6800043019E19BF800004E4A3121002350FA74
:10FC780003F515F0010F01D0117701E02D25157757
:10FC8800013301310132042BC9B2F0D12FE0002E2B
:10FC980000F00281202108224848F0F77BFB3D480C
:10FCA8009BF800108222F8F7A3FE394B1B7803F06B
:10FCB8008003DBB21BB199F80030012B02D82B78F6
:10FCC800032B21D1202102223248F0F763FB1BE0ED
:10FCD80050FA03F515F0010F01D0117701E02D2539
:10FCE8001577013301310132042BC9B2F0D1284B09
:10FCF8001B7803F08003DBB233B199F80030012B95
:10FD080002D9E4182023A376214B1B7803F0800343
:10FD1800DBB2002B00F0C68099F80030012B40F0D0
:10FD2800C180002F40F0BE80174820210822F0F73C
:10FD380031FBB7E099F80030214D13F0010F04BFF3
:10FD480043F0010389F800302E78002E4AD12D2186
:10FD58000A221C48F0F71EFB04201B49F8F722FE74
:10FD68001A4B1B78012B02D11020194906E0022BEF
:10FD780002D11020174901E017491020F8F712FEA8
:10FD880090E000BF840D0020040200201F1E002008
:10FD9800783A002012020020D41E0020043E0020E1
:10FDA800551E0020F401002065EF020886EF0208C6
:10FDB800A7EF0208C8EF0208E1EE02080C020020D3
:10FDC800131E0020381E002054F10208091E0020CE
:10FDD8003EE60208FCE502081DE602080B1E0020AC
:10FDE800051E0020314B1C782046F8F797FE304B53
:10FDF800304A00282AD0304F30493878A04216D1EE
:10FE080030380C782E4E00EB80073C19345D04B96D
:10FE18000C700F7800EB8000C4190137FFB2C019CD
:10FE28000F70315C345D59B92448017008E0012035
:10FE3800087019783C7019B1092E9CBF36182E70BD
:10FE48002978511801F8014C40211970197811B11D
:10FE58001748013901701978012909D12978092928
:10FE680002D818480131017000211970134B19701C
:10FE78001168154BC3F816105168C3F81A10128987
:10FE8800DA83124A127802F08002D2B252B12A788A
:10FE98009B1820225A7505E09BF800000A4A312178
:10FEA800002315E709B0BDE8F08F00BF401D002012
:10FEB8005D1D0020381E00205A1D0020861D0020D0
:10FEC800346E0208131E0020F4010020783A002046
:10FED8001FB5044611B100200B4901E008460B4943
:10FEE800F8F760FD217810220139C9B201EB011140
:10FEF80001F5C2414831684601F0B5FD10200146C0
:10FF08006A46FDF7BBF91FBD4CCF02088ECF020829
:10FF18000B4B1B78442B06D0552B037801D013B11B
:10FF28007047013B01E003780133037003780BB994
:10FF3800203302E0212B01D1203B0370FFF7C8BF1B
:10FF4800401D00202DE9F74FDFF8C881DFF8D4A164
:10FF580098F80030554643F0010388F800309AF8C5
:10FF68000130624C23F07F039B46D3B100206049E7
:10FF7800F8F718FD5F482A21F0F78AFA18B12178B6
:10FF88008222F8F735FD2278002A40F0AB802B68F2
:10FF980062F3CF332B60584B1A7842F003021A7081
:10FFA800A0E0DFF85491237099F800304E4603F032
:10FFB8000202D2B20192514F002A40D013F0010838
:10FFC80013D058464E49F8F7EDFC3B78232B20D147
:10FFD8004C4B4D4A4D481A600121FFF779FF3378A1
:10FFE80003F0FE036BF3410312E040464849F8F77B
:08FFF800D9FC3B78232B0CD14E
:020000040801F1
:10000000424B434A43481A600121FFF765FF3378AA
:1000100068F3000368F3410333703B782A2B65D102
:10002000337803F0FE036FF3410333702B6843F41E
:1000300000432B600F232370364B187803B0BDE8C4
:10004000F04F0DF089BF0DF0CBFE054600282DD0F6
:1000500001213048FFF760FF3B78532B12D13378F2
:10006000019A03F0FD0362F300033370DAF8003005
:1000700043F40043CAF800300F232370254B18784F
:100080000DF06AFF3B78232B30D13378002203F048
:10009000FD036FF3000333701E4B1A70F8F74AFD2F
:1000A0001E4A137843F00603137015E01C49F8F755
:1000B0007DFC3B78232B19D199F8003065F341037F
:1000C00065F3000389F80030F8F734FD98F8003044
:1000D00043F0060388F80030124A1378013BDBB284
:1000E0001370114A52F82320084B1A6003B0BDE880
:1000F000F08F00BF26580020D0CF0208F401002066
:10010000173C0020401D0020F1CF0208781D002080
:10011000F46F0208121E002012D00208571E0020A1
:1001200033D00208371E0020441E0020783A0020F9
:100130002DE9FF412C4D2D4C2B7843F001032B7002
:10014000217801F00401C9B211B92948FFF7E4FE92
:10015000284E3378232B21D12378274F13F004081E
:100160000AD0224A6FF382031370244B20483B606D
:100170000021FFF7B1FE11E0F8F7DCFC2B78204AF4
:1001800043F006032B701378013BDBB213701D4A5A
:1001900052F823303B60164B83F800803378532BA2
:1001A0001FD12378052243F004032370104B164916
:1001B0001C78013CE4B204EB840000F5CA408830AE
:1001C00001F04FFC00201149F8F7F0FBFF2300215C
:1001D00000930134162004220B460191029401F091
:1001E000B3FCBDE8FF8100BF571E0020173C002074
:1001F000121E0020401D0020781D002010700208F3
:10020000371E0020441E00202C700208AFCF0208C9
:100210002DE9F041984B04469A7812F0010F00F056
:1002200017811B88002B40F01381944D95F82030E6
:100230003F2B40F2D780012C14D1914B1B7803F057
:100240000203DBB2002B00F0C48095F820208B4B1A
:10025000402A03D1013283F82020FBE0482283F8B2
:100260002020B6E0022C03D1482385F82030B0E0EE
:10027000844E337803F02002D2B28AB195F8202060
:10028000402A0DD1032C0BD07F4B804A03F1100183
:1002900053F8040B8B4242F8040BF9D1412395E04B
:1002A00003F01003DBB28BB195F82030412B0DD158
:1002B000032C0BD0764B754A03F1100153F8040B55
:1002C0008B4242F8040BF9D142237FE0F37813F01C
:1002D000010F0FD095F82020422A0BD16D4B6B4AAD
:1002E00003F1100153F8040B8B4242F8040BF9D1CF
:1002F00043236BE003F00202D2B27AB195F82020DA
:10030000432A0BD1644B614A03F1100153F8040BEB
:100310008B4242F8040BF9D1442357E003F0040266
:10032000D2B27AB195F82020442A0BD15B4B574AC0
:1003300003F1100153F8040B8B4242F8040BF9D17E
:10034000452343E003F00803DBB28BB195F820307E
:10035000452B0DD1032C0BD0514B4C4A03F110010E
:1003600053F8040B8B4242F8040BF9D146232DE0DD
:100370000EF064FBA0B14B4B1B788BB195F820308D
:10038000462B0DD1032C0BD0474B404A03F11001F3
:1003900053F8040B8B4242F8040BF9D1472315E0C4
:1003A000F37803F04003DBB29BB195F82030472B84
:1003B0000FD1032C0DD03D4B344A03F1100153F8FB
:1003C000040B8B4242F8040BF9D1482385F8203006
:1003D00078E095F820300133DBB2472B85F82030E8
:1003E0007FF629AF95F82060472E04D9234B0026CD
:1003F00083F8206001E00136F6B206F14007FFB253
:1004000012E02B48314614F058FA08B1032C04D1FD
:10041000284B9B5D23B1032C02D185F820600FE0AF
:100420000136F6B2BE4203D03F2EEAD9402E07D1A4
:10043000214B1E221A70402385F82030BDE8F08140
:1004400095F820001149652246F69543F8F7FAF928
:10045000012C37D1194B0D4A03F1100153F8040B4D
:100460008B4242F8040BF9D1044B93F820303F2B18
:100470003CD9002012493EE0681E0020F401002013
:100480000D1A0020783A002084D602086F1E002042
:10049000A5D60208C6D60208E7D6020808D7020881
:1004A00029D70208F83D00204AD702088CD7020855
:1004B000A31A0020591A0020141E002084390308B2
:1004C00042D60208104BD87800F02000C0B220B10C
:1004D000022C06D000200D490DE0032C01D10C495F
:1004E00009E00C4B93F820303F2B02D800200A493A
:1004F00001E00A490020F8F759FA1020084A01469D
:10050000BDE8F041F8F70ABA783A00205DCD02085C
:1005100063D60208F401002000D602086BD7020857
:10052000681E002010B5F8F705FB084B1B7803F098
:100530000403DBB22BB106490020BDE81040F8F7F8
:1005400035BA0220BDE81040FFF762BE0D1A002048
:1005500032D4020870B5224B06461B78214CF3B901
:10056000257819E02048294614F0A7F978B12368C6
:100570009D4202D9FF2E02D007E0FF2E02D19D42FC
:1005800008D202E036B91DB913B9256012E00EB9E0
:10059000013500E0AD19EDB23F2DE3D90AE0013B92
:1005A0002021124810222360EFF7F8FE00201049A6
:1005B000F8F7FCF90F48F8F79FF946F695432078CD
:1005C0000D496522F8F73EF9084D216805F1100044
:1005D00001310222F8F710FA2D23AB7470BD00BF71
:1005E000071E0020201E00207E1D0020F401002098
:1005F00000180308681E00206F1E0020F8B5594B34
:10060000F02259481A700378044613F00E051DD1E4
:10061000564A43F00203156000F8013B14F0F2F86B
:100620002C46534BE35C1BB15248214614F02FF982
:100630000134402CF5D1504B01221A700FF03EFAD4
:100640004E4B1A7842F001021A70F8BD13F00C05F7
:1006500043D12E464748294614F02FF908B10136F8
:10066000F6B20135402DF5D11EB9237843F00403CD
:1006700031E0002542482946EFB214F01EF968B176
:100680003B4BEB5C53B13F4B01371F700020FFF732
:1006900061FF237843F00803237002E00135402D09
:1006A000E8D1394D3A212846EFF7F6FE38B1401B24
:1006B000C0B20130281831460222F8F79DF9334BB9
:1006C0001B78532B4CD12F4B00201870FFF742FFA3
:1006D000237843F008032370F8BD6FF341030370E0
:1006E00003F00403DBB2294D23B100202849F8F7B9
:1006F0005DF90EE02B78552B01D1FF2002E0442B51
:1007000002D10120FFF726FF13200D21214AF8F71F
:1007100005F92B78232B23D12478134E04F00204FF
:10072000F4B9154B1C700FF0C9F9337803F0FB03D3
:1007300064F3C30333700D4B1C60F8F7FBF90F4BE8
:100740001A7842F006021A70134A1378013BDBB2A2
:100750001370124A52F82320114B1A60094B1C7077
:10076000F8BD00BF631E00207D1D0020201E00205C
:10077000A02C00207E1D0020A8140020571E002061
:100780000E1A0020071E0020F4010020401D00204A
:1007900046290308681E0020371E0020441E002042
:1007A000781D002070B505460C4616463BB1430047
:1007B0004BF2B94018184018114601F03DF9054BAD
:1007C000182202FB0535F3092C1906F07F06637029
:1007D000E67070BD3C3B002038B510B3A0F141037A
:1007E000DBB2432B1FD9C50900F07F040BD0052CC9
:1007F00019D90021601E0A460AF04CFCD0F1010014
:1008000038BF002038BD082C0FD9601EC0B2294661
:100810002A460AF0A7F850B9202C8CBF00200120EE
:1008200038BD012038BD002038BD284638BD2846D7
:1008300038BD0000F7B5604C312323745F4F01339E
:100840002376053B637463763B784BF2B9405B00DB
:10085000181801F0FBF8C0B220F07F0200F07F0111
:10086000D2B28DF804108DF8002004F1120359B9AA
:10087000534A04F115001188927861829A70202100
:100880000222EFF78BFD0CE0D20904EB8202526AE0
:1008900010886082927804F115009A700222F8F7AD
:1008A000ABF83878400000F53440BA3001F0CEF8AB
:1008B000C0B220F07F0300F07F01DBB28DF805109D
:1008C0008DF801303F4851B93D4B20311A889B7853
:1008D0006283837002220330EFF760FD0BE0DB09D7
:1008E00004EB83035B6A1A8862839B78022283701D
:1008F0000330F8F781F8344B1B7813F0010F5AD00E
:10090000324D02A92A788B1813F8041C13F8086CCE
:100910002F4B1B78232B04D1002A41D1223B2B7073
:100920003EE02A2B04D1002A3AD0013A2A7037E05F
:10093000552B46EA010611D10DE02B7802AAD318F7
:10094000013E13F8081CF6B23046C90913F8042C0E
:10095000FFF742FF98B9002EEFD121E0442B19D1C7
:1009600015E02B7802A9CB18013613F8081CF6B253
:100970003046C90913F8042CFFF72EFF38B1134B8A
:100980003878197832460123FFF70CFF08E0872EEC
:10099000E7D905E0532B03D1533B2B70F9F7CCF883
:1009A0000C4B1B7803F08003DBB223B12B782022A1
:1009B000023304F83320FEBDF4010020071E00209E
:1009C000433503080E020020571E0020121E00208F
:1009D000401D0020783A0020024800210922EFF74C
:1009E000DDBC00BF251E002070B50A46002405E0CE
:1009F0001B19811A2A2501345D54E4B20E4D0F4BA8
:100A0000295D09B19442F3D1801A001918182021E8
:100A1000121BEFF7C3FC0A4B1E785EB1432E04D1C4
:100A20000CB1013CE4B200232B553046F8F77AF8BC
:100A300000B12E5570BD00BF251E0020F40100201E
:100A4000401D002038B5184C184DA07800F010005B
:100A5000C0B250B91649F7F7A9FFFFF7BDFF2368E9
:100A600043F4801323600F232B702A782AB923685C
:100A7000FF2062F31453236038BD0E48C5792DB9A9
:100A80001C200821FFF7B0FF284638BD23680A491B
:100A90006FF3145308222360EFF700FF00280CBF08
:100AA0000120FF2038BD00BF783A0020661E0020DC
:100AB00095D40208251E0020A4540308F0B55C4C10
:100AC00085B0667806F01006F6B2002E3ED1594B7E
:100AD0001A78594B013A53F82230584A934204D1BC
:100AE000574B1A7842F0020207E002F11C018B42D8
:100AF00008D1534B1A7842F00402022161F3C70275
:100B00001A7019E03832934216D1FFF79BFF002884
:100B100000F08C8001284A4D06D12B78022243F048
:100B2000010362F3C70306E030464649F7F73EFF8C
:100B30002B7866F3C7032B70434B1A7842F00102FF
:100B40001A70236843F4805323606FE03C4D2B7888
:100B500013F0F80606D03D49002005B0BDE8F0408E
:100B6000F7F724BF13F0070F41D003F00202D7B20A
:100B70004FB11220314610F0D7F8FF2300930196B1
:100B8000029643202AE003F00406F6B2A6B13946E5
:100B9000384610F0C9F8382102200EF0A3FC09F005
:100BA0000BFD0DF045F9FF230093019702974420B8
:100BB000394604223B4614E013F0010F13D0012103
:100BC00043F6206010F0B0F83046F5F7E5FA204B18
:100BD00045201E80FF230093019602963146042291
:100BE000334600F0B1FF00201A49F7F7DFFE2B78FB
:100BF00003F0FA036FF341032B70174B1B78232B81
:100C000014D123686FF30C332360F7F793FF0E4B77
:100C10001A7842F006021A70064A1378013BDBB2DA
:100C20001370054A52F823200C4B1A6005B0F0BD32
:100C3000783A0020371E0020441E0020347002083D
:100C4000A8550020B6D40208571E0020E22C030845
:100C5000561D0020C12C0308401D0020781D0020D7
:100C60001FB50446F5F784FBA8B14B2001F036FB15
:100C7000FF2300930121FF3B0193392004220B46FF
:100C80000134029400F060FF064B01205A7842F0D4
:100C900004025A7004E0044B1888003818BF012081
:100CA00004B010BD043C00203C580020F0B5204E9C
:100CB0000024337A0546013385B00F463372102085
:100CC0002146012223460094F1F71CFD55B9FF236C
:100CD00000934F20294604222B460195029700F0ED
:100CE00033FF0EE0012D0CD1FF230093502023464B
:100CF000214604220194029700F026FF337A013B3B
:100D00003372337A052B11D1FA3301210024009379
:100D100027200B4604220194029400F015FF044B97
:100D20001C7205B0BDE8F04001F0AABA05B0F0BDF4
:100D3000161E0020074B182202FB00335B7913F0CC
:100D4000100F05D0044B173ADA715A7009329A70B5
:100D5000704700BF3C3B0020671300202DE9F04F97
:100D60009A4B87B01A78074699461AB1012A40F083
:100D7000E68130E0964B1A68964B9A4200F0E1818A
:100D8000F4F774FF944B5B7803F00203DBB253B9C2
:100D9000924B5B7803F08003DBB223B901F096FA43
:100DA00008B909F009FC8E4B1A686FF310421A60FB
:100DB0008C4B1878F7F7B6FE002800F0C281FFF7D9
:100DC0000BFE894B3C221A70F7F7F8FC99F80030BB
:100DD000013389F80030844B1C7874B9834B791C3B
:100DE0001A78204664F3C30264F304121A70C9B27D
:100DF000FFF75CFF89F80040A3E17D4D384609F01C
:100E0000FBFBF7F7CFFC00207A49F7F7CFFDDFF8BF
:100E1000F4812B78AA46434413F8313C23B91B20B4
:100E20000621FFF7E1FD8CE1704A0B21137804A83D
:100E3000C3F3C004C3F3001603F0F7036FF3041306
:100E40001370002389F80030062200F010FE2A7883
:100E5000414604A8303AEFF7C7F9804628B14FF071
:100E600000084FF0120945462AE04AF26B7000F084
:100E7000EDFD0028F3D0604D85F80880F5F75EF8A9
:100E80000446002840F05D815C4A514B21461A60BF
:100E9000FF2300930190029004220820234600F0D3
:100EA00053FE012223460E2021460094F1F72AFC2E
:100EB000534B1A7842F004021A700123AB7140E1DF
:100EC0004946062204A800F0D2FD9AF8002004A8A2
:100ED0004C49303AEFF788F9002840F02181284644
:100EE000FFF7BEFE002840F02C81DFF80CB1012195
:100EF0008BF808002846F5F72FF88146F5F71EF81D
:100F0000DA46002840F0B58048463F49EFF74AFBF3
:100F1000B0B901F0EDF82E4B14B916B93B4A23E0F5
:100F200036B13B4A1A603B4B1A786FF3410205E039
:100F3000394A1A60374B1A7866F341021A70D7E0C3
:100F400048463649EFF72EFB20B148463449EFF7C3
:100F500029FB70B9002C40F0F480002E40F0F180A5
:100F600001F0C6F82F4A1A4B1A603846FFF7E2FE26
:100F7000BEE048462C49EFF715FB50B94AF26970BC
:100F8000012100F059FD164A136843F40053136021
:100F9000E0E748462549EFF705FB38B9002C40F05B
:100FA000D080002E40F0CD80214A0CE048462149F7
:100FB000EFF7F8FA002841D1002C40F0C280002E53
:100FC00040F0BF801C4A024B1A6091E0741D002063
:100FD000781D00208870020862340020133C002035
:100FE000783A0020401D0020661E0020241E0020AC
:100FF0005C1D00203CCD0208161E0020A4700208D3
:1010000071260020251E00202D560308F0720208CC
:1010100078740208571E002094740208A95503082A
:1010200039580308B0740208E4550308E65503086C
:10103000E8740208F65703083C750208484642491E
:10104000EFF7B0FA002853D101F052F83CB13F4A13
:101050003F4B1A603F4B1A786FF3410270E0002E4D
:101060006FD03D4A3A4B1A603A4B1A7864F341020A
:1010700066E048463449EFF795FA064620B901F094
:1010800037F8002C5DD01BE048463449EFF78AFA68
:10109000002856D048463249EFF784FA38B9002C78
:1010A0004FD1304A2A4B8BF807501A6049E0484626
:1010B0002D49EFF777FA064650B9A4B101F018F8B8
:1010C000224A234B1A60234B1A7866F3410237E019
:1010D00048462649EFF766FA20B148462449EFF71B
:1010E00061FA00B96CBB234A194B1A6001F000F891
:1010F00008F56A507C308AF8075000F0A7FC8AF89F
:1011000000009AF8070000F5D640693000F09EFC18
:101110008AF801001848F5F757F8202D11D108E09A
:101120000135EDB2202D08F1010809F107097FF41E
:10113000C7AE791C0020C9B2FFF7B8FD01E000225C
:101140001A7007B0BDE8F08FE855030894740208E0
:10115000781D0020571E002078740208E655030809
:10116000F65703083C7502082D560308A9550308D5
:10117000E455030858750208161E002010B52148D2
:10118000214903680A789C7B944203D99C8914F016
:10119000200F18D09A8912F0800F01D105E01C3B76
:1011A0009A8912F0400FFAD000E01C33036000234C
:1011B0000B7003689B8913F0200F16D0134BDA795C
:1011C000114B1A7011E00132D2B20A70986843F6DE
:1011D0000953984209D101E00132D2B2162A03D84C
:1011E0000B4853B29840F7D40A700A4A136843F484
:1011F00080731360F7F7E2FA074B1A7842F00602A1
:101200001A7010BD781D0020071E0020161E002039
:1012100000060088783A0020571E002010B52349A8
:10122000234A0B78D3B11068848914F0200F15D1AC
:10123000013BDBB20B70846843F60952944228D11B
:1012400004E013B1013BDBB200E0837B162B03D833
:10125000184C5AB29440F4D40B701AE01368988971
:1012600010F0400F01D106E01C33988910F0800F78
:10127000FAD0136002E00E481C3B036013689A7BAF
:101280000A709B8913F0200F03D00B4BDA79074BC0
:101290001A700A4A136843F480731360F7F78EFAE2
:1012A000074B1A7842F006021A7010BD071E002084
:1012B000781D002000060088161E0020783A0020C5
:1012C000571E0020084B1A68084B9A4204D003F5B9
:1012D00080630C339A4205D1054B1878003818BF4B
:1012E0000120704700207047781D00208870020898
:1012F0000C1A0020074B084A1B68934202D0383270
:10130000934205D1054B1878003818BF012070476B
:1013100000207047781D00203C7502080C1A002040
:101320002DE9F04F814B824D1970A0F11103DBB212
:10133000012B87B00E46287006D8122801D111382B
:1013400000E00020F4F786FF2B78522B0DD1F1F747
:10135000F3FE28B9F1F7E4FE10B9F1F705FF20B16B
:10136000744B1A7842F008021A70734B734C1B7856
:10137000002B2FD12168724A91422BD0714A2360F1
:101380001370714A71481178037063F3C30163F3FA
:10139000000163F3071111706D4A117863F30101C5
:1013A00011706C4A117863F3C50111706A4A1370A9
:1013B0006A4A117863F3410163F3000163F3820128
:1013C0001170674A116863F30C311160654A13703C
:1013D000654A93712368002B40F05F81604F7B78F2
:1013E00003F02003DBB273B1604B93F80080B8F1D7
:1013F000000F08D14AF26970414600F01DFB3B68BE
:1014000068F34D333B605A4B187810F01E0002D041
:101410000020584907E0544B93F808909846B9F1DA
:10142000000F05D0544907B0BDE8F04FF7F7BEBA3A
:10143000524F97F801B0BA46BBF1000F2DD0BBF167
:10144000070F15D94E48F7F757FA4E49B878652275
:1014500046F69553F7F7F6F93878072310F00300AE
:101460007B700EBF484948464849F7F79FFA0CE0A1
:10147000BBF1020F09D84248437823B1F7F73CFA91
:1014800087F80190B4E202237B7010203C4A0146A9
:1014900007B0BDE8F04FF7F741BA3D4FBB795BB1FC
:1014A00087F806B000F034FC8E20594601225B46D6
:1014B000CDF800B0F1F726F90020F1F79FFF224A9E
:1014C00020491378334843F00603137000230B7050
:1014D000314923600B7088F8033088F801300370BD
:1014E000183303FB06FC2D49934611F80CC08946BE
:1014F0001CF0080F04D130460593FFF72FFC059B25
:1015000003FB06935B7913F0100F04D02A78133A8B
:10151000D2B2032A46D913F0200F79D02B78442B6E
:1015200040D03DD8232B3DD02A2B3AE00A1E002084
:10153000401D00204B1A0020631E0020781D002053
:10154000D86F0208371E0020571E0020121E0020F0
:10155000591D00200D1E0020151E0020241E0020F5
:10156000783A0020621E0020671300200C1A002029
:10157000255800209FCD0208FEFE02080F1E002005
:10158000681E00206F1E0020A7CE020886CE02082B
:10159000161E00200C1E0020071E00203C3B0020D1
:1015A000552B35D18C4B1B78002B31D18B4B93F8BD
:1015B0000090B9F1000F2BD143F6DB2000F046FA82
:1015C000012825D11F23FB7188F8030043F61B3047
:1015D00000F03CFA3870F87900F5D640693000F038
:1015E00035FA78707E48F4F7EFFD9BF8003030460E
:1015F00069F341038BF8003008F0FEFFF7F79AFA21
:10160000784B79482360794BC3F800902B780370AE
:101610002B78432B0AD1714B1B783BB9013388F8E7
:101620000330734B3046236008F0E6FF2878173804
:10163000C3B2072B27D86F49FF220AF0BDFD9AF8E5
:1016400000106D4B60F301018AF8001001F00301F6
:10165000022918D00122032041B1009001929B7809
:1016600068309B1802930021033206E0009001923B
:101670009B786C200133029304220B4600F064FA3D
:10168000FF238AF8013098F80730002B00F0B08172
:1016900052232B70594B0022DA712268544B9A4224
:1016A00050D12878A0F14303DAB2122A22D8544A42
:1016B0005BB29A401ED5432840F09A81464B1B7876
:1016C000002B40F0958100F01DFD4E4B48B11A787B
:1016D00003201109013191FBF0F000EB4000091AE1
:1016E00004E01A781109013101F0070161F30712D2
:1016F0001A707DE1F7F716FA002823D0414F3A78A7
:1017000012F0F00308D163F307123A7023603E4BE6
:101710001A7842F008020EE0102B13D100F0F2FC10
:1017200080B13B786FF307133B7000232360364B87
:101730001A7842F0100230461A7007B0BDE8F04F38
:10174000FFF70CBB314B1E211A78264F61F346027E
:101750001A702B78232B1CD12368BB4219D12C4B38
:10176000182202FB0636737913F0100F11D0294BA3
:101770001B7873B11A4EF7F7DDF9FCF783FAF079AD
:1017800000F56A507C3000F061F93070AA20F1F762
:1017900035FE1C4E337813F0010F43D02368BB4253
:1017A0000BD01D4A934208D0FFF78CFD28B9FFF7F4
:1017B000A1FD10B9AA30F1F721FE2268174B9A4219
:1017C00002D10020F1F71AFE2B78522B40F0D58081
:1017D0005322134BC9E000BF0C1A0020741D0020D7
:1017E000161E0020587502080C1E0020441E002002
:1017F00088700208111E00200F1E002067130020B1
:10180000002000C0571E0020241E0020D51E0020EE
:101810003C3B0020371E0020D86F0208907502085C
:10182000401D00202368BB420BD0734A934208D06E
:10183000FFF748FD28B9FFF75DFD10B9AA30F1F7B1
:10184000DDFD2B78552B1ED1FFF7E8FC33786B4874
:1018500043F0060333708378694F03F00203DBB271
:101860004BB1F7F749F823681868FAF7CDF93B78D8
:101870006FF341033B706348837803F00203DBB2EC
:101880000BB1F7F739F82B78442B1ED1FFF776FC14
:1018900033785A4843F0060333708378584F03F087
:1018A0000203DBB24BB1F7F727F823681868FAF7A1
:1018B000ABF93B786FF341033B705248837803F0F8
:1018C0000203DBB20BB1F7F717F82B78522B09D1D3
:1018D0003378002243F0010333704B4B1A704B4BAB
:1018E00045321A704A4B00271F702B78232B44D1A6
:1018F000484B42481F70484B1F70F6F7FDFF4148A8
:10190000F6F7FAFF3378454943F0060333700B7856
:101910003B4A002B2BD0424A013B1770414ADBB2B5
:101920000B7052F8233023603F4B1A7812B11F70AE
:101930000EF0C4F823683D4A9B68934202D109F037
:10194000D3FE1AE002F59A718B4203D002F5E071E2
:101950008B4204D10120014606F0BAFF0DE002F5EA
:10196000EE72934209D1324B00221A7005E01178D1
:1019700063F30711117023603AE02E4BDB7813B14B
:101980000020F1F73BFD23681F7B17F00F0702D102
:10199000FBF720FB1BE0012F02D1F8F77BFA16E0E2
:1019A000022F02D1F9F7E6F911E0082F05D84FF020
:1019B0009C53BB4001D5F9F7A3FC042F03D1236846
:1019C0009B69984703E0052F01D1F8F751FF337861
:1019D00003F00203DBB21BB123681868FAF714F9AD
:1019E00033786FF3410333702B780BB1084A1370CF
:1019F00007B0BDE8F08F00BFD86F0208681E002056
:101A0000571E0020881D0020121E0020401D0020AF
:101A10005A1D0020151E0020621E0020371E0020C7
:101A2000071E0020441E0020A8140020AC750208E8
:101A3000871D00206713002007B502AB03F8011DC6
:101A400019460122002305F09DFB0EBD07B50023BA
:101A500002A901F8013D012205F0FCFB9DF80700F9
:101A60000EBD08B5002305F08DFB002008BD034620
:101A700010B508461446194605F0ECFBE0B210BD5F
:101A800010B50346002484540846194605F0E2FBCD
:101A9000204610BD37B50546002400E0144601225B
:101AA00060190DF1070105F0D5FB9DF80730621CA8
:101AB000203BDBB25A2BF1D920463EBDF8B50025BC
:101AC0002C461E4B1C21585D01FB0431400000F5E3
:101AD00074506630043102220134FFF7C2FF1C3516
:101AE0005C2CEED143F6C43420B2042205341449F0
:101AF000FFF7B7FFA4B243F6D8339C42F4D10025D8
:101B000049F668572C4615E007EB460004EB440104
:101B100000B259180222FFF7A4FF0136F6B2094BB2
:101B20005A199278B242EFD8013480370335142C19
:101B3000BFB201D00026F2E7F8BD00BFA4A00208A2
:101B4000AB550308B4AA02082DE9F347044615462D
:101B50008A46022243F61E610DF106001E46BDF9BB
:101B600030909DF828809DF82C70FFF780FF2F4B58
:101B70002F499A78BDF906008A705A7800EBC000A8
:101B8000CA701A7900F578500A715A7920304A7172
:101B90009A791B7845EAC6158A710C7081F8019014
:101BA000CB710D7200B20922FFF75BFF1EB1214B12
:101BB0001A8801321A80BDF8063001339BB2B3F5A2
:101BC0007A7FADF8063002D30023ADF8063002224A
:101BD0000DF1060143F61E60FFF743FFBDF8060056
:101BE000154B188000B200EBC00000F5785000F1F2
:101BF0002005283000B2FFF729FF10F0800F03D036
